:020000040800F2
:100000000050002049240008F92400080D3600089B
:10001000F9240008F9240008F92400080000000071
:10002000000000000000000000000000F9240008AB
:10003000F924000800000000F924000875540008A5
:10004000F9240008F9240008F9240008F92400081C
:10005000F9240008F9240008F9240008F92400080C
:10006000F9240008F9240008F9240008F9240008FC
:10007000F9240008F924000889530008F92400082D
:10008000F9240008F9240008F9240008F9240008DC
:10009000F9240008F9240008F9240008F9240008CC
:1000A000F9240008F9240008F92400081D24000898
:1000B00029240008312400083D240008714B000861
:1000C000F14E0008754B0008ED4E0008F9240008B9
:1000D000F9240008BD530008F9530008F92400086A
:1000E000F9240008F9240008F924000800000000A1
:1000F0000000000000000000000000000000000000
:0C01000000000000000000005FF808F1A3
:1001100010B5054C237833B9044810B10448AFF347
:1001200000800121217010BD9C050020000000000E
:10013000E80F010808B5064B1BB106480649AFF3A6
:1001400000800648016811B1054A02B1904708BD18
:1001500000000000E80F0108A00500209C05002019
:100160000000000081F0004102E000BF83F0004386
:1001700030B54FEA41044FEA430594EA050F08BF42
:1001800090EA020F1FBF54EA000C55EA020C7FEA06
:10019000645C7FEA655C00F0E2804FEA5454D4EB83
:1001A0005555B8BF6D420CDD2C4480EA020281EA4D
:1001B000030382EA000083EA010180EA020281EA85
:1001C0000303362D88BF30BD11F0004F4FEA0131D7
:1001D0004FF4801C4CEA113102D0404261EB4101E6
:1001E00013F0004F4FEA03334CEA133302D052426C
:1001F00063EB430394EA050F00F0A780A4F1010428
:10020000D5F1200E0DDB02FA0EFC22FA05F2801861
:1002100041F1000103FA0EF2801843FA05F3594147
:100220000EE0A5F120050EF1200E012A03FA0EFCC6
:1002300028BF4CF0020C43FA05F3C01851EBE371F0
:1002400001F0004507D54FF0000EDCF1000C7EEB0D
:1002500000006EEB0101B1F5801F1BD3B1F5001F4B
:100260000CD349085FEA30004FEA3C0C04F101046A
:100270004FEA445212F5800F80F09A80BCF1004F93
:1002800008BF5FEA500C50F1000041EB045141EA15
:10029000050130BD5FEA4C0C404141EB010111F416
:1002A000801FA4F10104E9D191F0000F04BF0146C1
:1002B0000020B1FA81F308BF2033A3F10B03B3F19F
:1002C00020020CDA0C3208DD02F1140CC2F10C022F
:1002D00001FA0CF021FA02F10CE002F11402D8BF8D
:1002E000C2F1200C01FA02F120FA0CFCDCBF41EA59
:1002F0000C019040E41AA2BF01EB0451294330BD28
:100300006FEA04041F3C1CDA0C340EDC04F1140404
:10031000C4F1200220FA04F001FA02F340EA0300DB
:1003200021FA04F345EA030130BDC4F10C04C4F121
:10033000200220FA02F001FA04F340EA0300294601
:1003400030BD21FA04F0294630BD94F0000F83F44B
:10035000801306BF81F480110134013D4EE77FEA2E
:10036000645C18BF7FEA655C29D094EA050F08BF7A
:1003700090EA020F05D054EA000C04BF194610465B
:1003800030BD91EA030F1EBF0021002030BD5FEA9F
:10039000545C05D14000494128BF41F0004130BDC7
:1003A00014F580043CBF01F5801130BD01F000451B
:1003B00045F0FE4141F470014FF0000030BD7FEA8E
:1003C000645C1ABF194610467FEA655C1CBF0B4689
:1003D000024650EA013406BF52EA033591EA030FA0
:1003E00041F4002130BD00BF90F0000F04BF002198
:1003F000704730B54FF4806404F132044FF00005CB
:100400004FF0000150E700BF90F0000F04BF002143
:10041000704730B54FF4806404F1320410F00045A9
:1004200048BF40424FF000013EE700BF42004FEAA4
:10043000E2014FEA31014FEA02701FBF12F07F4321
:1004400093F07F4F81F06051704792F0000F14BF1E
:1004500093F07F4F704730B54FF4607401F0004562
:1004600021F0004120E700BF50EA010208BF7047B9
:1004700030B54FF000050AE050EA010208BF7047AE
:1004800030B511F0004502D5404261EB41014FF417
:10049000806404F132045FEA915C3FF4DCAE4FF01B
:1004A00003025FEADC0C18BF03325FEADC0C18BF02
:1004B000033202EBDC02C2F1200300FA03FC20FA53
:1004C00002F001FA03FE40EA0E0021FA02F11444A0
:1004D000C1E600BF70B54FF0FF0C4CF4E06C1CEAB5
:1004E00011541DBF1CEA135594EA0C0F95EA0C0F2A
:1004F00000F0DEF82C4481EA030621EA4C5123EA9D
:100500004C5350EA013518BF52EA033541F48011CB
:1005100043F4801338D0A0FB02CE4FF00005E1FB7E
:1005200002E506F00042E0FB03E54FF00006E1FBC8
:1005300003569CF0000F18BF4EF0010EA4F1FF040B
:10054000B6F5007F64F5407404D25FEA4E0E6D414B
:1005500046EB060642EAC62141EA55514FEAC5205C
:1005600040EA5E504FEACE2EB4F1FD0C88BFBCF5D8
:10057000E06F1ED8BEF1004F08BF5FEA500E50F189
:10058000000041EB045170BD06F0004646EA01014F
:1005900040EA020081EA0301B4EB5C04C2BFD4EB81
:1005A0000C0541EA045170BD41F480114FF0000E7A
:1005B000013C00F3AB8014F1360FDEBF002001F0E8
:1005C000004170BDC4F10004203C35DA0C341BDC62
:1005D00004F11404C4F1200500FA05F320FA04F034
:1005E00001FA05F240EA020001F0004221F0004168
:1005F00010EBD37021FA04F642EB06015EEA430EDB
:1006000008BF20EAD37070BDC4F10C04C4F120050A
:1006100000FA04F320FA05F001FA04F240EA0200BD
:1006200001F0004110EBD37041F100015EEA430E8E
:1006300008BF20EAD37070BDC4F1200500FA05F2AE
:100640004EEA020E20FA04F301FA05F243EA02032D
:1006500021FA04F001F0004121FA04F220EA02003C
:1006600000EBD3705EEA430E08BF20EAD37070BD82
:1006700094F0000F0FD101F00046400041EB010162
:1006800011F4801F08BF013CF7D041EA060195F044
:10069000000F18BF704703F00046520043EB0303FE
:1006A00013F4801F08BF013DF7D043EA06037047EB
:1006B00094EA0C0F0CEA135518BF95EA0C0F0CD0F6
:1006C00050EA410618BF52EA4306D1D181EA03013C
:1006D00001F000414FF0000070BD50EA410606BF36
:1006E0001046194652EA430619D094EA0C0F02D17B
:1006F00050EA013613D195EA0C0F05D152EA0336C0
:100700001CBF104619460AD181EA030101F00041DD
:1007100041F0FE4141F470014FF0000070BD41F026
:10072000FE4141F4780170BD70B54FF0FF0C4CF400
:10073000E06C1CEA11541DBF1CEA135594EA0C0F1F
:1007400095EA0C0F00F0A7F8A4EB050481EA030E6C
:1007500052EA03354FEA013100F088804FEA033353
:100760004FF0805545EA131343EA12634FEA022221
:1007700045EA111545EA10654FEA00260EF00041E2
:100780009D4208BF964244F1FD0404F5407402D234
:100790005B084FEA3202B61A65EB03055B084FEAC5
:1007A00032024FF480104FF4002CB6EB020E75EBC2
:1007B000030E22BFB61A754640EA0C005B084FEAEA
:1007C0003202B6EB020E75EB030E22BFB61A754667
:1007D00040EA5C005B084FEA3202B6EB020E75EBB2
:1007E000030E22BFB61A754640EA9C005B084FEA2A
:1007F0003202B6EB020E75EB030E22BFB61A754637
:1008000040EADC0055EA060E18D04FEA051545EA25
:1008100016754FEA06164FEAC30343EA52734FEACE
:10082000C2025FEA1C1CC0D111F4801F0BD141EA47
:1008300000014FF000004FF0004CB6E711F4801FAC
:1008400004BF01430020B4F1FD0C88BFBCF5E06F8C
:100850003FF6AFAEB5EB030C04BFB6EB020C5FEA9C
:10086000500C50F1000041EB045170BD0EF0004EF1
:100870004EEA113114EB5C04C2BFD4EB0C0541EA23
:10088000045170BD41F480114FF0000E013C90E620
:1008900045EA060E8DE60CEA135594EA0C0F08BFE4
:1008A00095EA0C0F3FF43BAF94EA0C0F0AD150EAE3
:1008B00001347FF434AF95EA0C0F7FF425AF104676
:1008C00019462CE795EA0C0F06D152EA03353FF49E
:1008D000FDAE1046194622E750EA410618BF52EA1B
:1008E00043067FF4C5AE50EA41047FF40DAF52EAEF
:1008F00043057FF4EBAE12E74FEA4102B2F1E04369
:1009000024BFB3F5001CDCF1FE5C0DD901F0004CF6
:100910004FEAC0024CEA5070B2F1004F40EB830046
:1009200008BF20F00100704711F0804F21D113F172
:100930003872BCBF01F00040704741F480114FEAAB
:100940005252C2F11802C2F1200C10FA0CF320FA34
:1009500002F018BF40F001004FEAC1234FEAD32351
:1009600003FA0CFC40EA0C0023FA02F34FEA4303BB
:10097000CCE77FEA625307D150EA01331EBF4FF044
:10098000FE4040F44000704701F0004040F0FE405F
:1009900040F40000704700BF80F0004002E000BF5C
:1009A00081F0004142001FBF5FEA410392EA030F5A
:1009B0007FEA226C7FEA236C6AD04FEA1262D2EBA4
:1009C0001363C1BFD218414048404140B8BF5B42A9
:1009D000192B88BF704710F0004F40F4000020F042
:1009E0007F4018BF404211F0004F41F4000121F058
:1009F0007F4118BF494292EA030F3FD0A2F10102A2
:100A000041FA03FC10EB0C00C3F1200301FA03F1DF
:100A100000F0004302D5494260EB4000B0F5000F02
:100A200013D3B0F1807F06D340084FEA310102F1C1
:100A30000102FE2A51D2B1F1004F40EBC25008BF73
:100A400020F0010040EA03007047490040EB00003D
:100A500010F4000FA2F10102EDD1B0FA80FCACF16C
:100A6000080CB2EB0C0200FA0CF0AABF00EBC2506B
:100A700052421843BCBFD0401843704792F0000F59
:100A800081F4000106BF80F400000132013BB5E7AC
:100A90004FEA41037FEA226C18BF7FEA236C21D022
:100AA00092EA030F04D092F0000F08BF0846704787
:100AB00090EA010F1CBF0020704712F07F4F04D155
:100AC000400028BF40F00040704712F100723CBF68
:100AD00000F50000704700F0004343F0FE4040F492
:100AE000000070477FEA226216BF08467FEA236350
:100AF0000146420206BF5FEA412390EA010F40F43B
:100B0000800070474FF0000304E000BF10F0004386
:100B100048BF40425FEA000C08BF704743F096436D
:100B200001464FF000001CE050EA010208BF704788
:100B30004FF000030AE000BF50EA010208BF70470F
:100B400011F0004302D5404261EB41015FEA010C24
:100B500002BF84460146002043F0B64308BFA3F11C
:100B60008053A3F50003BCFA8CF2083AA3EBC253FE
:100B700010DB01FA02FC634400FA02FCC2F120021D
:100B8000BCF1004F20FA02F243EB020008BF20F054
:100B90000100704702F1200201FA02FCC2F12002BA
:100BA00050EA4C0021FA02F243EB020008BF20EAAF
:100BB000DC7070474FF0FF0C1CEAD0521EBF1CEADD
:100BC000D15392EA0C0F93EA0C0F6FD01A4480EACB
:100BD000010C400218BF5FEA41211ED04FF00063B4
:100BE00043EA501043EA5111A0FB01310CF00040E0
:100BF000B1F5000F3EBF490041EAD3715B0040EA06
:100C0000010062F17F02FD2A1DD8B3F1004F40EBD5
:100C1000C25008BF20F00100704790F0000F0CF0A8
:100C2000004C08BF49024CEA502040EA51207F3A6C
:100C3000C2BFD2F1FF0340EAC250704740F4000047
:100C40004FF00003013A5DDC12F1190FDCBF00F038
:100C500000407047C2F10002410021FA02F1C2F1E6
:100C6000200200FA02FC5FEA310040F1000053EA82
:100C70004C0308BF20EADC70704792F0000F00F0D0
:100C8000004C02BF400010F4000F013AF9D040EAD6
:100C90000C0093F0000F01F0004C02BF490011F46A
:100CA000000F013BF9D041EA0C018FE70CEAD15368
:100CB00092EA0C0F18BF93EA0C0F0AD030F0004CE8
:100CC00018BF31F0004CD8D180EA010000F000409C
:100CD000704790F0000F17BF90F0004F084691F05A
:100CE000000F91F0004F14D092EA0C0F01D1420294
:100CF0000FD193EA0C0F03D14B0218BF084608D15D
:100D000080EA010000F0004040F0FE4040F40000A6
:100D1000704740F0FE4040F4400070474FF0FF0C39
:100D20001CEAD0521EBF1CEAD15392EA0C0F93EA80
:100D30000C0F69D0A2EB030280EA010C49024FEAD2
:100D4000402037D04FF0805343EA111143EA10138B
:100D50000CF000408B4238BF5B0042F17D024FF443
:100D6000000C8B4224BF5B1A40EA0C00B3EB510F1E
:100D700024BFA3EB510340EA5C00B3EB910F24BF07
:100D8000A3EB910340EA9C00B3EBD10F24BFA3EB8C
:100D9000D10340EADC001B0118BF5FEA1C1CE0D154
:100DA000FD2A3FF650AF8B4240EBC25008BF20F007
:100DB000010070470CF0004C4CEA50207F32C2BF5B
:100DC000D2F1FF0340EAC250704740F400004FF0F8
:100DD0000003013A37E792F0000F00F0004C02BF29
:100DE000400010F4000F013AF9D040EA0C0093F0F3
:100DF000000F01F0004C02BF490011F4000F013B4D
:100E0000F9D041EA0C0195E70CEAD15392EA0C0FB4
:100E100008D142027FF47DAF93EA0C0F7FF470AFEC
:100E2000084676E793EA0C0F04D14B023FF44CAF2F
:100E300008466EE730F0004C18BF31F0004CCAD1C4
:100E400030F000427FF45CAF31F000437FF43CAF00
:100E50005FE700BF4FF0FF3C06E000BF4FF0010C22
:100E600002E000BF4FF0010C4DF804CD4FEA400204
:100E70004FEA41037FEA226C18BF7FEA236C11D04E
:100E800001B052EA530C18BF90EA010F58BFB2EB01
:100E9000030088BFC81738BF6FEAE17018BF40F081
:100EA000010070477FEA226C02D15FEA402C05D135
:100EB0007FEA236CE4D15FEA412CE1D05DF8040BBA
:100EC000704700BF844608466146FFE70FB5FFF74D
:100ED000C9FF002848BF10F1000F0FBD4DF808ED05
:100EE000FFF7F4FF0CBF012000205DF808FB00BFF6
:100EF0004DF808EDFFF7EAFF34BF012000205DF850
:100F000008FB00BF4DF808EDFFF7E0FF94BF01209C
:100F100000205DF808FB00BF4DF808EDFFF7D2FF99
:100F200094BF012000205DF808FB00BF4DF808EDDC
:100F3000FFF7C8FF34BF012000205DF808FB00BFA9
:100F40004FEA4002B2F1FE4F0FD34FF09E03B3EBD6
:100F500012620DD94FEA002343F0004310F0004F16
:100F600023FA02F018BF404270474FF0000070476C
:100F700012F1610F01D1420205D110F0004008BF0B
:100F80006FF0004070474FF00000704742000ED2F3
:100F9000B2F1FE4F0BD34FF09E03B3EB126209D4B4
:100FA0004FEA002343F0004323FA02F070474FF06A
:100FB0000000704712F1610F01D1420202D14FF0DF
:100FC000FF3070474FF00000704700BF2DE9FF4130
:100FD000334B8046187800283BD00024254626460F
:100FE0002746082232210DEB0203532003F05CFE5A
:100FF0009DF809109DF80800013400EB01239DF8CD
:101000000B109DF80A001AB200EB01239DF80D1099
:101010009DF80C00E4B2BF181AB200EB01239DF852
:101020000F10B618202C1AB2154401F07F0001D021
:101030000028D6D11B4B97FBF4F796FBF4F695FBF3
:10104000F4F5ADF80070ADF80260ADF804501C7016
:101050001DE03221062202AB532003F025FE9DF84D
:1010600009209DF808109DF80B0001EB02239DF864
:101070000A20ADF8003002EB00219DF80C309DF8FD
:101080000D00ADF8021003EB0022ADF80420064A73
:1010900068464146127801F055FBBDE8FF8100BF6C
:1010A000B8050020B905002000000020154B10B540
:1010B0001B7804462D21532008227BB103F0B8FE93
:1010C00031210A22532003F0B3FE2C210C2253209D
:1010D00003F0AEFE53203821902209E003F0A8FE71
:1010E00031210A22532003F0A3FE53202C210A228F
:1010F00003F09EFE044840F2091202800CB103493D
:101100000C7010BDB8050020120000200000002067
:1011100037B5104B05461A680F480C46002182422D
:101120008DF8071001D1002013E0532001220DF1AA
:10113000070303F0B9FD0028F5D09DF80710E52955
:10114000F1D12A780548064B064920601A70616083
:1011500001203EBD4C010020001BB700AD1000086F
:10116000B8050020CD0F000813B5022204461B214C
:1011700001AB682003F098FD9DF804209DF8053030
:1011800043EA022000F54E5110314FF48C7291FB6E
:10119000F2F3233323801CBD1FB504461D21062214
:1011A0006B46682003F080FD9DF800209DF801301B
:1011B00043EA022001B2042391FBF3F29DF80200FE
:1011C0009DF80310ADF8082041EA002210B290FB10
:1011D000F3F19DF805209DF80400ADF80A1042EAED
:1011E0000021064A08B290FBF3F3214602A81278C8
:1011F000ADF80C3001F0A6FA1FBD00BF02000020C0
:1012000010B50446192004F068F968201521002261
:1012100003F00EFE10B9032004F0D0F90D4B162197
:101220001A78682042F0180203F002FE172100220B
:10123000682003F0FDFD3D210122682003F0F8FD48
:1012400068203E21012203F0F3FD0CB10248047036
:1012500010BD00BF010000200200002038B5054687
:1012600019200C4604F039F968201521002203F0FA
:10127000DFFD18B3124B13481349144A622C2B603C
:101280006860A960EA60124B0FD004D80A2C12D013
:10129000142C0CD10DE0BC2C04D0B4F5807F06D109
:1012A000002009E00120187038BD022004E003206E
:1012B00002E0042000E005201870012038BD00BFC6
:1012C00001120008991100086911000818449231B0
:1012D00001000020074B197821B1012906D14FF4F4
:1012E000805201E04FF40062034B1A8008B10349B9
:1012F00008707047BA05002012000020030000208B
:101300001FB50446432106226B46682003F0CCFC3F
:101310009DF800209DF8013043EA022001B2042329
:1013200091FBF3F29DF802009DF80310ADF8082040
:1013300041EA002210B290FBF3F19DF805209DF8E0
:101340000400ADF80A1042EA0021064A08B290FBF8
:10135000F3F3214602A81278ADF80C3001F0F2F94F
:101360001FBD00BF050000201FB504463B2106221B
:101370006B46682003F098FC9DF800209DF8013032
:101380009DF8021043EA02209DF80320ADF8080002
:1013900042EA01239DF804009DF80510ADF80A30DB
:1013A000054B41EA0022ADF80C2002A821461A782C
:1013B00001F0C8F91FBD00BF0300002013B5224A89
:1013C0004FF4005304460220ADF804308DF80700B6
:1013D00013681E48042183428DF8061001D11C4871
:1013E00003E01C498B4203D11B4801A903F088FD8F
:1013F0006B218022682003F01BFD052004F06DF8AE
:1014000019210022682003F013FD6B2103226820BC
:1014100003F00EFD37210222682003F009FD0F4A78
:101420001A211278682003F003FD1B21182268207E
:1014300003F0FEFC68201C21102203F0F9FC0CB123
:10144000074B1C701CBD00BF4C01002000127A002D
:10145000000C0140001BB7000010014004000020F8
:10146000050000202DE9FF41064623200D461446C5
:1014700004F033F86820752101220DF1070303F011
:1014800013FC00286DD09DF80780B8F1680F67D174
:1014900006210A4602AB404603F006FC9DF80B30DD
:1014A0009DF80D7003F0010107F001004A0042EAC7
:1014B00080079DF8090000F001031F4307D0012FAA
:1014C000294801D1002318E0022F0CD114E00C218F
:1014D000012240460DF1070303F0E6FB9DF80710DB
:1014E00011F00F0203D1052004F068F806E0042A89
:1014F0001D4801D1077001E0012303701A481B4900
:1015000003781B4A31607260002B14BF6E216F217B
:10151000184A1948194B142C31742A606860EB6022
:10152000174915D004D8052C16D00A2C0ED111E07D
:10153000BC2C08D0B4F5807F03D0622C06D10222E7
:101540000BE0002209E0012008700AE0032204E019
:10155000042202E0052200E006220A70012000E0D9
:10156000002004B0BDE8F081BA050020D5120008C3
:1015700069130008BD1300080113000819449231D3
:10158000040000201FB50446A82106226B466820EF
:1015900003F08AFB9DF800209DF8013043EA022009
:1015A00001B2042391FBF3F29DF802009DF80310B1
:1015B000ADF8082041EA002210B290FBF3F19DF84B
:1015C00005209DF80400ADF80A1042EA0021064A01
:1015D00008B290FBF3F3214602A81278ADF80C3064
:1015E00001F0B0F81FBD00BF0600002010B5044692
:1015F000642003F072FF68202321F02203F018FC1E
:1016000010B9032003F0DAFF052003F066FF064B54
:1016100068201A78202142F00F0203F009FC0CB177
:101620000248047010BD00BFBB050020060000206A
:1016300037B5054619200C4603F04FFF68200F21EF
:1016400001220DF1070303F02FFB9DF80730D32B88
:1016500016D10C480C490D4A4E2C28606960EA608E
:101660000B4B07D05D2C09D0362C01D0002002E0B6
:10167000402000E080201870012002E0C020FAE73E
:1016800000203EBDED15000885150008DDE9A731F5
:10169000BB0500202DE9F041057890B000350646E5
:1016A000334818BF012509F0CBFF00243148A5427B
:1016B000314B0CBF2146802106904FF400500CBFE7
:1016C0004FF001084FF002084FF4807205930A9121
:1016D00020234FF480670E9005A925480B920D93A7
:1016E0000C970794CDF8208009940F940AF020F805
:1016F0001F4801210AF049F84FF4602101270291A7
:101700001E48694600948DF804508DF805700394C6
:101710008DF8108009F03AF9184804213A4603235D
:1017200009F085F92DB1154831780222032309F01B
:101730007EF91248012109F056F91048012109F0FB
:1017400049F90E4809F058F90C4809F05AF90028EF
:10175000FAD10A4809F059F9084809F05BF900285C
:10176000FAD10648012109F059F910B0BDE8F0811D
:1017700008000240BC0500204C2401400024014028
:10178000024B33F8100080B2704700BFBC05002048
:10179000F8B5134B05469B890E461446ECB116B1BD
:1017A00016F8017B00E0FF270D48022109F0E8F858
:1017B0000028F9D00A48394609F0DDF80848012127
:1017C00009F0DEF80028F9D0054809F0D6F8C0B2D3
:1017D0000DB105F8010B013CE0E70120F8BD00BFA9
:1017E000003800402DE9F047012188B04FF48040D7
:1017F00009F022FE374C01214FF4804009F034FEFD
:1018000003214FF420401823ADF800008DF8031099
:10181000204669468DF802304FF0040803F070FB53
:101820002D4E4FF4804220466946ADF800204FF41B
:1018300080554FF0100A8DF8028003F061FB694675
:101840002046ADF800508DF802A003F059FB304659
:1018500009F034F807214FF4007000230222ADF89C
:101860001600ADF81C104FF00109304603A94FF4E3
:101870008277ADF80C30ADF81030ADF81A30ADF815
:101880001220ADF80E70ADF814901F46ADF818A0F8
:1018900009F046F83046494609F061F89F238DF873
:1018A00004308DF805708DF806708DF807700DEB1B
:1018B00008014246656102A8FFF76AFF25619DF8AD
:1018C0000900B0F1EF014A4252EB010008B0BDE857
:1018D000F08700BF000C014000380040074BA1F525
:1018E0007A7153F82000838802684B434FF47A7072
:1018F00093FBF0F18BB21380704700BFC00600204D
:10190000024B53F82000026811807047C006002087
:101910002DE9F04FDFF828814FEA001558F805400F
:101920008E468BB008EB050711468346924620464B
:101930007246019300F0C0FCB96807F108024FF04D
:10194000020C18237868ADF8141005A98DF816302C
:101950008DF817C00392CDF808C003F0D1FA0398B0
:10196000364E077906A809F0AEFA70220198DDF824
:1019700008C0ADF81820012100234FF4807206EB57
:101980000509ADF81A10ADF81C30ADF81E00ADF821
:1019900020C0ADF824200C2F2BD8DFE807F0072A51
:1019A0002A2A102A2A2A192A2A2A2200204606A987
:1019B00009F082F92046082109F0BAFA19E0204618
:1019C00006A909F0BDF92046082109F0B9FA10E08E
:1019D000204606A909F0F8F92046082109F0BAFACC
:1019E00007E0204606A909F031FA2046082109F04F
:1019F000B9FA08EB0B118B7B1BB12046012109F0D2
:101A000080FA2046012109F070FA0C2F10D8DFE887
:101A100007F0070F0F0F090F0F0F0B0F0F0F0D0020
:101A2000343404E0383402E03C3400E04034745193
:101A3000A9F804A048460BB0BDE8F08FD4050020FB
:101A400070E900081B4A1C4813881180C91A89B222
:101A500040F68C2291420380184B02D900221A7062
:101A60007047A1F2EF2080B240F2DA52904218D8CB
:101A70001B78072B15D81248032B20F81310114A96
:101A800009D811480088884205D2012101FA03F3E0
:101A900010780343137012780F2A02D1094B0021EA
:101AA00019700648094B0278511C017000201880FB
:101AB000704700BFC0050020B6060020D2050020F8
:101AC000C2050020B8060020080000206A07002098
:101AD0007FB5044601A80D46164609F0FEF9002020
:101AE0000123ADF80A00ADF80C0001A92046ADF8BD
:101AF0000450ADF80660ADF8083009F06FFA7FBD0C
:101B00002DE9F743DFF858800501144E05EB080472
:101B1000A3688946761928210746B27160680222B7
:101B20008DF8061001A9ADF804308DF8072003F0F8
:101B3000E7F955F80800217B0022FFF7C9FF20468E
:101B400001224FF6FF7100F0D9FB204639464A4684
:101B500000F094FB3046BDE8FE8300BFD4050020B2
:101B600070E9000810B5134B00011B18DA795AB957
:101B700001221981DA71104B02221918097B1858B9
:101B8000BDE81040FFF7A4BF1C8959810B4A091B0F
:101B90009C7989B222F8141000249981DC71064BDB
:101BA00022461918097B1858FFF792FF0448048051
:101BB00010BD00BFD405002070E90008C205002058
:101BC0006A0700202DE9F0410446028A484B8079DB
:101BD00061781A80002814BF0225002501B1013563
:101BE000444F57F8257000257A5DFF2A02F00F0058
:101BF00002F0F00309D122893F484049B2F5FA7F4B
:101C0000016071D93E4B03606EE0A17811B1811E75
:101C1000012965D9E17811B1011F032960D9E17962
:101C200009B181425CD012F0300F03D02278002A33
:101C300008BF0023217931B1A27922B9A0F10801AE
:101C4000012998BF802362792AB1A17919B9021FAD
:101C5000032A98BF802303F01001CAB23AB10022D0
:101C60002849FFF74DFF284B08221A7038E003F08F
:101C70002001CAB242B1244E24493278FFF740FF16
:101C80003078411C31702BE003F04001CAB292B1B0
:101C900023891F4AB3F5FA7F94BF012108214A43E3
:101CA0001C4EB2FBF3F39AB2A38996F80080FFF7BB
:101CB0002FFE194B0EE01B0612D563891449174EEF
:101CC00091FBF3F292B2E389012196F80080FFF7CD
:101CD0001FFE134B43F8280008F1010886F8008026
:101CE00001350E2D80D186E70020BDE8F08100BFD0
:101CF0000800002038E90008BC060020011900088F
:101D0000DD180008451A0008B4060020651B00080D
:101D100040420F00B5060020C0060020B906002092
:101D2000F006002008B5044B1A78824202D9034B12
:101D30001A68904708BD00BFB5060020BC06002009
:101D4000044B1A78824204D9034B53F820000268EE
:101D500011807047B9060020F0060020014B33F8CF
:101D600010007047C2050020704701717047426A39
:101D7000806A131A594251EB03007047037913F03C
:101D800001010BD0026AC3699A4205D09CBFC068AA
:101D90001218D01AC0B2704700207047084670472A
:101DA000037910B513F0010104460ED0FFF7E6FFEA
:101DB00060B1E3696269E168D05C4A1E934201D276
:101DC000013300E00023E36110BD084610BD037934
:101DD0009A070AD5436A8269D154416A03694A1C49
:101DE000B2FBF3F103FB11224262704790F84232DA
:101DF0001BB1D1F1010138BF0021D0F83401426894
:101E0000836809B1136170475361704707B5034692
:101E100099684822ADF804100223406801A98DF8A2
:101E200006208DF8073003F06BF80EBD58B50E4B49
:101E3000044618680E460346B3FBF2F1B1F5803F45
:101E400003D3012BF8D95B08F6E7084A89B2B0FB47
:101E5000F2F3DAB2204600F051FA054A2046314644
:101E6000BDE8584000F00ABA5001002040420F007F
:101E7000E52100087FB5044601A80D46164609F085
:101E80002CF800200123ADF80A00ADF80C0001A9E0
:101E90002046ADF80450ADF80660ADF8083009F002
:101EA0009DF87FBD38B504460D46002A0CBF0222BE
:101EB0000022217B0068FFF7DDFF034A2046294608
:101EC000BDE8384000F0DAB97920000807B50346CC
:101ED00099681022ADF804100223406801A98DF81A
:101EE00006208DF8073003F00BF80EBD00F1340327
:101EF0004FF48072436100F59C710023C26003625D
:101F0000C361816102618362436270472DE9F041E0
:101F10001D46194B0E46032103600171044690468D
:101F20000127FFF7E3FF002084F83C0284F8390220
:101F3000A4F84402A4F8460284F83872D4F83401B4
:101F400084F84252FFF7C2FF206BFFF75FFF39466C
:101F50002046FFF74BFF322003F0BFFAD4F83401DC
:101F600031464246FFF762FF206B31462A46BDE804
:101F7000F041FFF797BF00BF58E9000810B5084AC5
:101F8000044608480B4602631032C0F83421002191
:101F90002246FFF7BBFF044B01201C60187110BDE7
:101FA000B0E900087011002010070020034607491F
:101FB0000748084AC0F8781212681031C0F87C133C
:101FC00000F512700121FFF7A1BF00BFD0E90008A2
:101FD0007011002010070020C268036A511E8B4256
:101FE00001D3002300E001330362704710B590F87D
:101FF0003C220446AAB9836A416A994225D0806985
:102000002169C05C01338B42A36228BFA2624200F7
:102010000A2342F4007084F83D32A4F83E02012302
:1020200011E090F93D3273B1B0F83E124A08A0F8C1
:102030003E2201F00101FFF7D9FE94F83D02431E54
:1020400084F83D3210BD84F83C3210BD90F83B322C
:1020500010B583B990F83A3290F8392293420AD2F7
:10206000012101FA03F1B0F8404201332143A0F805
:102070004012DBB2F2E710BD2D4B10B54FF41274D5
:1020800004FB00342079C10751D594F8381221B3EC
:10209000236B0021186808F06FFF94F83C1221B1FF
:1020A000B4F84402421CA4F84422236B94F8422260
:1020B0001868197B002A14BF02220022FFF7DAFEFB
:1020C0000020012184F83B1284F8390284F83A0296
:1020D000A4F8400284F8380210BD94F83B22204650
:1020E000012A04BF94F8392284F83A22FFF7AEFFA0
:1020F00094F83B02236B58B9012094F8422284F8EB
:102100003B021868197B002A14BF022200220AE051
:10211000002184F83B1294F842221868197B002AA7
:102120000CBF02220022BDE81040FFF7A3BE10BD85
:102130007011002090F83B1200230122012980F841
:10214000393280F838220CD180F83B32036B90F89A
:102150004222197B1868002A0CBF02220022FFF7D6
:1021600089BE704702790346D20713D5B0F84022E2
:1021700002F4007189B209B9D10705D4B3F8460257
:10218000421CA3F8462270474169036A5208CA54A8
:10219000FFF722BF704710B590F838320446002B85
:1021A0001ED190F839124A1CD3B2092B80F839326B
:1021B00003D1BDE81040FFF749BF0A2B10D190F8BA
:1021C0003B0228B9B4F8401241F00102A4F84022C1
:1021D0002046FFF7C7FF2046BDE81040FFF7AABF23
:1021E00010BD0000064B10B54FF4127404FB003410
:1021F0002046FFF7FBFE2046BDE81040FFF7CBBFAF
:102200007011002030B500240E4D55F82450854241
:1022100002D00134E4B2F7E7A400E4B200200A4D92
:102220002D5C8D4202D0451CE8B2F8E70019C0B21F
:102230000F2805D8054C04EB001083600171027370
:1022400030BD00BF50EA000860EA00080016002018
:102250000C2912D8DFE801F0071111110911111131
:102260000B1111110D00022104E0042102E00821EC
:1022700000E01021012208F052BE704738B5044634
:102280000D461346217B00682A46FFF7BBFF2068F6
:10229000217BBDE83840FFF7DBBF07B58DF80400B0
:1022A000012000238DF806008DF8070001A88DF8A5
:1022B000053008F013FC0EBD7FB5044601A80D469D
:1022C000164608F0F7FD0B4B0B485E4301680023F0
:1022D000B1FBF6F2013D561E204601A9ADF80850AB
:1022E000ADF80460ADF80A30ADF8063008F09AFC9D
:1022F0007FBD00BF40420F005001002010B50446D2
:102300000068FFF7D9FF2068012108F0EEFD607B2F
:10231000BDE81040FFF7C1BF00230C4A52F823204C
:10232000824202D05A1CD3B2F7E79B00D8B20023F6
:10233000074AD25C8A4202D05A1CD3B2F8E7181876
:10234000044BC1B203EB0110704700BF50EA000814
:1023500060EA00080016002070B5044600262E4BE7
:10236000F55C95B90221204608F0E1FE01284FD125
:102370002046022108F0E6FE29462046FFF7CCFF62
:102380000546204608F0C6FE3DE0042D12D1204649
:10239000294608F0CCFE01283AD12046294608F00B
:1023A000D1FE29462046FFF7B7FF0546204608F034
:1023B000B4FE28E0082D12D12046294608F0B7FEC9
:1023C000012825D12046294608F0BCFE2946204692
:1023D000FFF7A2FF0546204608F0A2FE13E00C2DF1
:1023E00016D11021204608F0A2FE012810D1204667
:1023F000102108F0A7FE29462046FFF78DFF05466D
:10240000204608F090FEAA6801460AB1287B904752
:102410000136042EA3D170BD60EA00080148FFF721
:102420009BBF00BF002C01404FF08040FFF794BFDE
:102430000148FFF791BF00BF000400400148FFF7CB
:102440008BBF00BF000800401D481E4902680060A5
:102450008A4200F01F80002100F004B81A4B5B583C
:102460004350043119481A4B42189A42FFF4F6AF10
:10247000184A00F003B8002342F8043B164B9A4276
:10248000FFF4F9AF08F00CF90BF04AF900F0BCFFCB
:10249000FFF7FEBF114E124830601248016821F06C
:1024A00070610160410201600F4C182020600F49EB
:1024B0000F4808600F48D0F800D04068004700007F
:1024C000F04F0020EFBEADDE0C1001080000002030
:1024D0009C0500209C050020601D00201810024073
:1024E0000900000004000140140C0140000C0140F0
:1024F0004434434400F0FF1FFFF7FEBF014B186850
:1025000002F039BD501D00200149002000F048BEF6
:10251000FD24000810B5FEF7F9FA0A49FEF74AFB58
:102520000949FEF7FBFB094B044618680078FEF7E3
:10253000EDFA01462046FEF73DFBFEF727FD80B28F
:1025400010BD00BF3333534000F07F452C070020FF
:1025500038B50D4C00202578FFF712F90B4A05F02D
:10256000070322F813000135002325701846D15ABD
:1025700002334018102B80B2F9D1C008FFF7CAFF10
:10258000034A107038BD00BF180700201A0700204A
:1025900000170020074B084A19781088884207D393
:1025A000064B1A68907888428CBF00200120704743
:1025B0000020704700170020021700202C07002081
:1025C000124B70B51860202400250020FFF7D8F8C2
:1025D0002D180A2002F081FF013CF6D1C5F34F10FF
:1025E000FFF798FF094902230A6851784D006619E0
:1025F000B04203D30133062B0C44F8D1044892783F
:102600000370534303490B8070BD00BF2C070020AB
:102610000A000020021700202DE9F04F0446008830
:1026200085B048B9B4F9023043B9B4F90420D2F105
:10263000010138BF002102E0002100E0014611F055
:10264000010377D13D4D00B22B7000F0D9FC064656
:10265000B4F9020000F0D4FC0546B4F9040000F01F
:10266000CFFC0446304609F0B3F80746304609F07F
:1026700023F98046284609F0ABF80646284609F0BB
:102680001BF90546204609F0A3F88246204609F0CA
:1026900013F9394681465046FEF78CFA394683468F
:1026A0004846FEF787FA514601904046FEF782FA07
:1026B000494602904046FEF77DFA31460390504667
:1026C000FEF778FA1E4C4946206006F10040FEF7FE
:1026D00071FA29466060A5600298FEF76BFA014620
:1026E0000198FEF75FF92946E0600398FEF762FA69
:1026F00001465846FEF754F93146206108F1004082
:10270000FEF758FA294660615846FEF753FA01462B
:102710000398FEF745F92946A0610198FEF74AFAA9
:1027200001460298FEF73EF93946E0613046FEF771
:1027300041FA206205B0BDE8F08F00BF0B00002019
:1027400030070020013A2DE9F8430C46072A30D81B
:10275000DFE802F004080F14191E222601882180E8
:10276000428803E043880B8002885242628082885C
:102770001EE00388594221804288F6E74388594287
:1027800021800288F2E703885942218041880CE0C9
:1027900042880A80018808E003880B80428803E0B1
:1027A0004388594221800288514261808088424298
:1027B000A28030480278002A5AD1B4F90000FEF70E
:1027C000A5F98046B4F90200FEF7A0F90746B4F96E
:1027D0000400FEF79BF9284D064629684046FEF79F
:1027E000E9F9E96881463846FEF7E4F901464846CA
:1027F000FEF7D8F8A96981463046FEF7DBF90146B5
:102800004846FEF7CFF809F017F86968208040467F
:10281000FEF7D0F9296981463846FEF7CBF9014623
:102820004846FEF7BFF8E96981463046FEF7C2F92F
:1028300001464846FEF7B6F808F0FEFFA96860803A
:102840004046FEF7B7F9696980463846FEF7B2F9A7
:1028500001464046FEF7A6F8296A07463046FEF7CD
:10286000A9F901463846FEF79DF808F0E5FFA0807B
:10287000BDE8F8830B00002030070020F8B5154CA8
:1028800006462378274663B902F016FE124D2A68E1
:102890003232904205D30123237002F00DFE2860EE
:1028A000F8BD3878A0B102F007FE0B4C2168731810
:1028B00098420DD307480022027002F0FDFD07493F
:1028C00020600B780BB15A1E0A7005490120087070
:1028D000F8BD00BF540700205C0700205607002009
:1028E0005707002037B58DF805101F498DF80730C0
:1028F0000B788DF8040002A88DF80620C21812F893
:10290000044C0D46443CE0B20A2828D81749022B53
:1029100031F8104003D814B12046FFF7AFFF2B78F1
:10292000022B0BD9124D2D6802F0C6FD021B9542F9
:1029300004D20D490F4B0020087018700E48027821
:102940000146012A00D074B9074B1878022801D833
:10295000421C1A7000230B7008490B7003E03224EC
:10296000022BD9D9DBE73EBD5907002064EA0008F5
:102970005C0700205607002057070020540700205E
:1029800070B5374B04465A7B364802B101220270BB
:102990004FF4007000F032F9F0B133494B78181C55
:1029A00018BF012000F0CEFC38B1304D0120287056
:1029B00000F0D4FC08B102222A7000F0B1FC28B16A
:1029C00029494B7813B9294A0220107000F09EFC67
:1029D00010B1264B00211970202005F0AFF860B12E
:1029E0001F482349827A0AB9C37A23B11E48C27AA2
:1029F0000AB9012300E000230B701C490878022863
:102A000002D14C204E211DE0012807D14D21532039
:102A10004C220B46BDE87040FFF764BF144A1378A0
:102A2000012B03D1532001464E2206E00D490878C0
:102A3000012804D15320014602464D23EAE724B180
:102A400053204D210A464423E4E70A4A137823B170
:102A50003220BDE87040FFF711BF07490C7070BD10
:102A6000DC1C002055070020CB1C00205A0700204A
:102A70005807002056070020540700200E4B1A78F4
:102A8000402A16D15888B0F5667F12D11979BE292F
:102A90000FD193F895230020EF2A0CD113F8011BD6
:102AA000064A48409342F9D1D0F1010038BF0020D6
:102AB000704700207047704700F8010898FB010834
:102AC00038B5FFF7DBFF10B90A2002F077FD164C8E
:102AD000164920464FF466720AF06CFE94F894335F
:102AE000022B02D9002084F8940394F89413CC228A
:102AF00002FB01430E4D03F5987128460AF05AFE79
:102B000005F11F0005F0D0F805F11F00B4F8D01052
:102B1000B4F8D22005F0E2F8287801F01DF9BDE8FC
:102B2000384003F0F9BF00BFD417002000F80108B7
:102B3000081700202C4B70B5402206464FF46670F3
:102B40001A705880BE25EF2200201D7183F895234E
:102B500083F8960349B193F89413CC2202FB013316
:102B6000224903F598700AF025FE00210D461E4A01
:102B7000885C0131B1F5667F85EA0005F7D182F8FE
:102B80009653002508F06AFB342008F07BFB1848B8
:102B900008F0CEFB042811D1154C164B2046E15805
:102BA00008F09CFB042805D0013508F063FB032DD9
:102BB000E8D103E0104A04349442EED108F05AFB05
:102BC000032D02D0FFF75AFF10B90A2002F0F6FCDD
:102BD000FFF776FF36B10F2014210122BDE87040C7
:102BE00007F044BD70BD00BFD417002008170020B7
:102BF00000F80108D41FFE1798FB0108034B9968E1
:102C000008420CBF00200120704700BFD4170020ED
:102C1000024B9A6810439860704700BFD417002099
:102C20002DE9F3470446FFF729FF10B1002C00F00F
:102C30007081B94AB94D10685168B94C6B4603C3ED
:102C40004FF46672002128460AF062FECC22002171
:102C500020460AF05DFE40200321287002206971A1
:102C6000FFF7D6FFFA22A5F8F2202A236E22A5F854
:102C7000EE304FF4FA7085F804212B2340F24C42D9
:102C8000A5F8F60085F80531212002F548732021CA
:102C900085F80601A5F8163140F27E404FF47A73AC
:102CA00000274FF001094FF4167685F8F410A5F8C7
:102CB000142140F2DC5100F52F72A5F8D00003F585
:102CC000CB70A5F8F060A5F81211A5F8D22085F810
:102CD0009473A5F8F870A5F8FA70A5F8FC7085F85B
:102CE000E27085F8E37085F8E470A5F8E670A5F861
:102CF000E870A5F8EA7085F8ED7085F8EC9085F835
:102D0000077185F82C7185F82D7185F82E7185F87D
:102D1000107185F8187185F8197185F81A91A5F860
:102D2000D430A5F8D6006C30A5F8D8004FF4C870A0
:102D3000A5F8DE004FF41650322340F2B452C5F825
:102D4000240140F6AC50A5F8DA20A5F8DC301A468C
:102D5000A5F8E030A8814FF4E1331E20C5F82031FA
:102D6000E07252232073552085F82A31E070172332
:102D70000B204FF028086375A37560712D23142074
:102D80004FF0080E63732271A07184F810E085F88B
:102D90001C7185F81D7185F8287185F8297185F8F1
:102DA0001B71277084F8018084F80280E775A7738F
:102DB0002776E7736776A37660745020E076E18427
:102DC0005A20042120722375E077412384F82E10C5
:102DD000544855494FF00E0A84F82030534B84F87C
:102DE00007A04FF0640C4FF00A0A4FF0780E84F8F9
:102DF000212060631522E1634D4805F5847184F854
:102E00003120A36384F812A084F81CC084F80980E0
:102E100084F80AE084F81E9084F8237084F8247003
:102E200084F8257084F822706785A785278584F843
:102E30002F8084F8308084F8409004F08DFF4FF4A8
:102E40004872C8204FF4966340F2D9313E4684F868
:102E50006C7084F86D7084F86E8084F86F9084F8DC
:102E60007270A4F8702084F8B4A084F8B500A4F8B7
:102E7000B630A4F8B8104FF47F724FF4FA601DF822
:102E80000710A4F87420A0F5FA73FF220137A4F804
:102E90007600A4F8783084F87A1084F87B2008341F
:102EA000082FE8D11E4C0120C823142184F8BA0051
:102EB00084F8BB0084F8BC00A4F8BE3084F8C010CD
:102EC00084F8C2001E2264204FF49673282184F8EF
:102ED000C120A4F8C400A4F8C630A4F8C810002487
:102EE0000E4A0023A0181034C02C0361F8D100242E
:102EF0001049CC2260180A49CC340AF05BFCB4F5C6
:102F0000197FF5D10020014602B0BDE8F047FFF778
:102F100011BE02B0BDE8F08708E90008D417002010
:102F2000081700209A99193F3D0A773FF6287C3F01
:102F30007AEA000804190020024B9A6822EA00008D
:102F400098607047D4170020014B9868704700BF05
:102F5000D4170020884203DB8242B4BF11460146E9
:102F6000084670470023036170472DE9F041066968
:102F700004460136012E0D46066105D1002361602D
:102F800021608360BDE8F081D0F8008008464146AA
:102F9000FDF706FD07463046FDF7B8FD0146384609
:102FA000FDF7BCFE01464046FDF7FCFC06466060AE
:102FB00031462846FDF7F4FC01463846FDF7FAFD98
:102FC000A168FDF7EFFC2660E060A060BDE8F0813D
:102FD00010B504460069012807DD0138FDF796FDAC
:102FE0000146E068FDF79AFE10BD002010BD08B54F
:102FF000FFF7EEFFBDE8084008F0ECBC0000000061
:1030000008B5FDF701FA04A3D3E90023FDF762FA3E
:10301000FDF772FC08BD00BF399D52A246DF913F0B
:103020002DE9F041069C06460F46002B0CBF4FF0E1
:1030300020084FF03008204610F8013B0BB9154628
:1030400003E0002AFBDD013AF6E7002D04DD3046FF
:103050004146B847013DF8E714F8011B11B130466D
:10306000B847F9E7BDE8F0812DE9F04389B006469D
:103070000F4603921C46039A134613F8011B039351
:10308000002900F08A80252901D0304683E0002005
:1030900004905578911C302D039105D19578033219
:1030A00003924FF0010800E08046A5F13003D8B24A
:1030B000092806D8284603A90A2204AB00F00CF917
:1030C00005466C2D05D10399012211F8015B03918E
:1030D00000E00022642D2FD010D8582D3AD006D809
:1030E000002D5AD0252DC6D13046294653E0632DF8
:1030F000C1D130462178251DB8474AE0752D0DD045
:10310000782D27D0732DB6D1251D24683046009424
:103110003946049A0023FFF783FF3AE0251D206813
:103120000A2122B1002205AB00F060F802E005ABF5
:1031300000F08CF82C4623E005AD04F1040920686A
:10314000294612B100F077F801E000F0A4F84C46EF
:10315000009517E004F104092068102142B1B5F18F
:103160005804634253EB040205AB00F03FF806E05D
:10317000B5F158035A425A4105AB00F067F84C4686
:1031800005A8009030463946049A4346FFF748FFA9
:1031900071E72C466FE7B8476DE709B0BDE8F083EB
:1031A000024B196002490860704700BF60070020A9
:1031B000640700200FB407B5094904AB0868094942
:1031C00053F8042B09680193FFF74EFF064B18686C
:1031D00001F0F0FE0028F9D0BDE80E4004B07047C1
:1031E0006407002060070020501D0020F0B5012476
:1031F000B0FBF4F58D4201D34C43F9E70026C4B18E
:10320000B0FBF4F504FB1500B4FBF1F41EB9002D7E
:1032100001DC002CF4D1092DEFB204DD002A0CBF33
:103220005725372500E03025ED1903F8015B0136FD
:10323000E5E71C70F0BD00280B4603DA2D22404262
:1032400003F8012B0A210022FFF7D0BFF0B50124BB
:10325000B0FBF4F58D4201D34C43F9E70026C4B12D
:10326000B0FBF4F504FB1500B4FBF1F41EB9002D1E
:1032700001DC002CF4D1092DEFB204DD002A0CBFD3
:103280005725372500E03025ED1903F8015B01369D
:10329000E5E71C70F0BD00280B4603DA2D22404202
:1032A00003F8012B0A210022FFF7D0BFA0F1300361
:1032B000DAB2092A01D818467047A0F16101052940
:1032C00001D857387047A0F14103052B01D8373892
:1032D00070474FF0FF3070472DE9F8430D68044602
:1032E0000F469046994600262046FFF7DFFF00284C
:1032F00006DB404504DC08FB060615F8014BF3E746
:103300003D602046C9F80060BDE8F883034BB3F97F
:103310000000D0F1010038BF002070476A0700208C
:10332000064B0749B3F9000091F8B4300522534326
:103330009842D4BF00200120704700BF6A070020D8
:103340000817002010B50446FFF7EAFF002814BF55
:103350002046002000F0010010BD00000749084B86
:1033600091F8B420B3F9000091F8B530D1180522D6
:1033700051438842D4BF0020012070470817002025
:103380006A07002008B504F0F9FB024B00221A700E
:1033900008BD00BFCB1C002010B54FF40070FFF734
:1033A0002DFC18B3FFF7BCFFE0B1114B5C78201C7B
:1033B00018BF0120FFF7C6FF70B10E480E4BB0F8E2
:1033C00012210E49B3F8B6000A804A808A80C8806C
:1033D0000B490A88531C0B80FFF7C0FF00B90CB9DA
:1033E000FFF7D0FF074801884A1C028010BD00BFCC
:1033F000CB1C0020D4170020081700200C1D002033
:10340000680700206A07002010B586B002F070F847
:10341000FFF77AF80020FFF703FCFFF751FB6F4A34
:1034200092F8073133B1012B01D0092B02D18DF86D
:10343000003004E000208DF8000082F807016846A3
:10344000FEF728F96648FFF7E7F8022004F080FB52
:1034500002F08AFD61494C790E2C01D0082C01D173
:10346000012200E000224FF480708DF80A20FFF75F
:10347000C5FB18B90820FFF7C1FB00E0012000F0F0
:10348000010340208DF80630FFF7B8FB8DF80700E8
:103490000120FFF7B3FB8DF805000820FFF7AEFB16
:1034A00080F001008DF8040003F0AEF94D498DF86D
:1034B000080091F8BC404FF47A71C4F38002474C85
:1034C0008DF80920B4F8E000B4F8DE30ADF80E0055
:1034D0004FF48040ADF80C30ADF81010FFF78EFBC4
:1034E00018B1B4F8DA20ADF81020BDF80C30B3F5FF
:1034F000FA7F02D90020ADF810003A4AB4F8121150
:1035000094F80741B2F8B830012CADF81210ADF8BC
:10351000143004D0092C01D1072400E0002401A8B4
:103520008DF80B40FEF74EFB2F4804F047FB4FF49D
:103530008070FFF763FB40B10820FFF75FFB20B905
:10354000264890F81D0103F039FB0A24192001F0E8
:10355000C4FF192001F0C1FF611E11F0FF04F5D175
:1035600001F0DCF802F0C4F80220FFF747FB10B1CD
:103570001E48FFF725F81E4805F0B0F94020FFF778
:103580003DFB50B1154CD4F8240194F82811FEF7F6
:10359000F5FC94F82901FEF709FD4FF40060FFF7F0
:1035A0002DFB10B1134804F07DFE01F06BFF124AB1
:1035B0000A4B10605879052803D1104C4FF4C8719C
:1035C00021800F4B4FF47A721A800E490E4AC820A0
:1035D00001240880547300F0CDFBFCE7D4170020D1
:1035E000BA18002008170020DC180020D818002086
:1035F000F4180020501D0020B00700200C08002007
:103600007208002070080020CB1C002008B5034B76
:10361000B3F9D40002F0C4FDFEE700BFD4170020C8
:103620002DE9F04F794B0024B3F902A0B3F9000063
:1036300087B0BAF1000FB8BFCAF1000A0028B8BFBE
:1036400040428245B8BF82462546A046274605949B
:10365000A14626466E49CA7812B90B79002B40D094
:10366000022E3ED06B4B6C486849B0F8F620685E7D
:10367000E95EDFF8B4B101EB40005142FFF76AFCAC
:10368000664A05EB0B0335F902C0B3F92A10CCEBFF
:1036900000009BF8082000EB010902FB09F09BF8F1
:1036A0001C30642190FBF1F005226FF004015943B6
:1036B0005A43CDF81090FFF74DFC594BDDF810C080
:1036C000E258584981460CEB020042F21072049312
:1036D000FFF740FC04999BF81230605058430013E8
:1036E00005904B49CA781AB10B790BB9022E30D12B
:1036F000464F4D48EF5F5021794306EB000B9BF896
:1037000001204A4BDFF83C8191FBF2F0E95E54F86E
:103710000820401A801846494FF47A520493FFF764
:1037200019FC049B48F80400E95E0029B8BF49422F
:10373000B1F5207F02DD002048F8040058F804208D
:103740007D239BF80B1092FBF3FE01FB0EFC4FEA6E
:10375000AC182F480279A2B1022E12D00AFB07F151
:10376000CAF5FA7303FB09104FF4FA7190FBF1F2FA
:103770000AFB08F0DDF814B003FB0B0393FBF1F335
:1037800008E0C3780BB1022E02D143463A4601E06D
:10379000059B4A462549DFF8B0C0695A16F80CB0B7
:1037A00008B20BFB00FB6FF04F0C9BFBFCFB934440
:1037B000204ACDF804B035F902C0A952CCEB000084
:1037C0001D4ADFF888C0029054F80C10A058401829
:1037D000029903904018A15844F80C100299A15086
:1037E000164A0434B15C202201FB00F090FBF2F198
:1037F0005B1A134A9B44013625F802B00235032EAA
:103800007FF428AF07B0BDE8F08F00BFA01B0020F9
:10381000CB1C0020E0070020D41700202C0C002037
:10382000E8070020F0D8FFFF081700201C0C00203C
:1038300080C1FFFFF2070020C0070020EE1B002020
:10384000A81B002070070020F11B0020800700202B
:103850002DE9F74F002425462646A246474BDA7845
:103860000AB91879C8B1022E19D0454B45484649C6
:10387000B0F8F6206F5EE85E514200EB4700FFF7BC
:1038800069FB424A424F35F902A0EB19CAEB00012D
:10389000B3F92A0001EB000A0BE0022E09D13C49E2
:1038A000394B91F82470B3F904201B3757437B112F
:1038B00016E03249364ACF7877B9334892F8237008
:1038C0002B5E1B375F4309793B1149B1927C02FBA8
:1038D0000AF703EB272303E0137A03FB0AF0031133
:1038E0002C48DFF8C8B0295EBBF800005F1A284BEF
:1038F000784306EB030898F80120DFF8B4907A4388
:1039000098F80B104FEAE21C54F80920C31201FB8F
:103910000320214944F809004FF40012CDF804C0F7
:10392000FFF718FB1D4B4FF6FF72E158E750791A6D
:10393000BBF8007044F809003B09B2FBF3F74F43B2
:10394000174A184B54F80290E158BF11A750494448
:1039500098F81520C9194A43DDF804C012490CEB48
:10396000603044F80390013600EB22236B5204349C
:103970000235032E7FF472AFBDE8FE8FCB1C002012
:10398000E0070020D4170020A01B00202C0C0020F2
:10399000081700201C0C00200000E0FFD0070020CA
:1039A000900700209C070020A81B0020E4070020AF
:1039B000700700200B4B0C481A8852B9817841B12E
:1039C00042786AB9012141700848094B02881A807F
:1039D0007047437823B90220FF21012206F046BE3A
:1039E000704700BF72080020CB1C0020361C00204E
:1039F000EC1B00202DE9F04FA94BAA4AB3F90600B1
:103A0000D18C85B088420FDBB0F5FA6F92F8254073
:103A100007DA451A6C43A1F5FA6694FBF6F46434B0
:103A200003E0C4F1640400E064249F4A9D4BB2F8B3
:103A3000127192F9EC2093F823100097574293F8F3
:103A40006C50019193F86D60B9B293F824300291F3
:103A5000002103930A46924FDDF8008031F907C038
:103A600040F2E637C8EB0C0303F2F31EBE4503D861
:103A7000002BB8BF5B4201E04FF4FA73022ADFF873
:103A800034822CD025B1AB42CCBFC5EB030300235D
:103A90006427DFF84CA293FBF7FE6FF0630B3AF854
:103AA0001E900BFB0E3B0EF1010E3AF91EA00FFA11
:103AB00089FECEEB0A0E0EFB0BFE9EFBF7FEF144D9
:103AC00028F80190DDF8048003FB08FE774B9EFB8D
:103AD000F3F3DB199BB2634393FBF7F712E026B1D4
:103AE000B342CCBFC6EB03030023029F5F43A8F899
:103AF0000470039F002BB8BF5B427B436B4F93FB6B
:103B0000F7F76437674B02EB030E9EF801906423CE
:103B100007FB09F898FBF3F9DFF8C88102F8089071
:103B20009EF80B909EF815E007FB09F807FB0EF7CF
:103B300098FBF3F9DFF8B08197FBF3F302F80890F4
:103B4000DDF800805A4FC445D35503DA594BCF5A9C
:103B50007F42CF5201320231032A7FF47CAF524CB4
:103B60004FF4FA62B4F81411FFF7F4F9B4F81461E1
:103B70004FF47A75801B4543C6F5FA63B5FBF3F540
:103B800064214D4895FBF1F36FF0630630F8132084
:103B900006FB0355013330F9130013B2C01A454335
:103BA000464B444C95FBF1F1587A8A18E280002884
:103BB00038D0434F434D3E882988721A10B2FFF720
:103BC0001FFA074607F004FE0646384607F074FE63
:103BD0000546B4F90200FCF799FF0746B4F9000066
:103BE000FCF794FF31468046FCF7E4FF2946814606
:103BF0003846FCF7DFFF01464846FCF7D1FEFDF7EB
:103C00009FF9314620803846FCF7D4FF2946064606
:103C10004046FCF7CFFF01463046FCF7C3FEFDF7F8
:103C20008FF960800220FEF7E9FF90B12648062256
:103C30000378591CCBB20370B3FBF2F002FB1031D6
:103C400011F0FF0F05D1FEF783FCFEF7A3FC1F4B1D
:103C500018701E4A1078003018BF0120FEF790FE41
:103C60001B490B882BB91B4A108838B904F0F6FAA7
:103C700004E0022003F062FF0028F4D01649174A3E
:103C800009681368C81A002832DB0C4B587B68BBE4
:103C9000987001F5F42303F59070106028E000BFE0
:103CA0000C1D002008170020D41700200CFEFFFF79
:103CB000EE1B0020A01B0020F41C0020CB1C0020C9
:103CC000361C0020EC1B00206C070020AF070020F2
:103CD0000C08002072080020F8070020A807002028
:103CE000301D0020F11B0020E41B002001219970F1
:103CF00004F000FE124A117831B94FF40060FEF76B
:103D00007DFF08B104F0F2FA202003F017FF78B12C
:103D10000C4B18680C4B1A68811A002908DB0B4AF7
:103D20001178042904D900F5123000F5F8721A60F0
:103D3000074B996809B10748884705B0BDE8F08F7F
:103D4000D8100020F8070020DC070020EA1B002024
:103D5000201C0020801B00200128034B14BF034AB5
:103D6000034A1A60704700BF0C000020213600088B
:103D70005138000838B50820FEF740FF90B19F4B3E
:103D800093F8100103280CD8DFE800F002020508C0
:103D900004F012FA06E004F06DF803E004F020F9F4
:103DA00000E000209649974A0B681168591A0029CB
:103DB00002DA002800F0618203F59C449248203426
:103DC0009249146003F018FF4FF48040FEF716FF8D
:103DD00020B18F4D2B780BB903F0D0FE874A92F8B3
:103DE0001B11B1B18B4CC81C34F910504FF47A72CE
:103DF0000021A5F57A70FFF7ADF8FCF787FE86493C
:103E0000FCF78CFF8549FCF7D5FEFDF7BFF8844B26
:103E10001880FFF7C1FA794AB2F81401B2F81641D6
:103E2000002215467B49AD08535E8342C4BF65F04E
:103E30007F05EDB2A342B8BF45F040050232082A23
:103E4000F0D17848784A04780346AC4204D110781F
:103E5000F92803D8411C00E0002111704FF4804084
:103E60001D70FEF7CBFE68B1644B6A4DB3F81211BA
:103E7000B3F8DC20B5F90640881A844202DD8D18BB
:103E8000AC420CDB4FF48040FEF7B8FEF8B9614C51
:103E90005A4BB4F90610B3F81421914217DA63496A
:103EA0006348644CB1F84230002505604560856088
:103EB000256065605BB1564A5F4D1078002800F0C0
:103EC0006D822C78002C00F06982FFF773FD564B51
:103ED0001A78142A40F0D58057484478ECB1534CF6
:103EE000B4F842202AB94F4D29785F2901D103F057
:103EF00045FE424890F81831002B00F0C2804B4C30
:103F0000B4F84220002A40F0BC80464D29787D2933
:103F100040F0B78003F032FEB3E0424D29785729D4
:103F200018D1464C4FF47A724FF480702280FEF71D
:103F300065FE08B102F09EFD042003F0FFFD10B104
:103F40003F490A250D80082003F0F8FDD8B93D4B04
:103F5000188018E00420FEF751FEA0B12B785A2BF0
:103F600011D1394802781AB10470384B012009E0A8
:103F7000374C384B257885F00101217009B10220BA
:103F800000E003201870274802785D2A00F00D82B7
:103F90005B2A00F00C825E2A00F00B822348B0F806
:103FA000422032B91F4C25786F2D02D1FFF702FD58
:103FB00015E012491B4B91F8180118B112B91A7883
:103FC0007E2AF3D01C78972C04D1234B4FF4C87071
:103FD000188004E0A72C02D1174901258D73114ADE
:103FE0001478BB2C03D1114CA18D8D1C04E0B72C8F
:103FF00034D10E4CA28D951EA5853BE0D417002030
:10400000F80700207C070020DC180020F21C0020AC
:10401000DC1C00200C1D002000007A4400C07F44FE
:10402000E81B0020AD070020F00700200817002043
:1040300070070020E8070020CB1C00207208002039
:1040400070080020361C0020B40700208C070020D8
:10405000AC070020560700200C080020BE2C03D11E
:104060008A4D6B8D981C04E0BD2C0AD1874D698D5B
:10407000881E688501200146FEF75CFD844B002008
:1040800018700420FEF7BAFD00282CD0814B187858
:1040900088B1814C627872B1804D8148B5F90610C3
:1040A000B0F81441A14206DD7E4A15781DB97E495B
:1040B000322008801D707B4B5C7C54B17B4B1D789B
:1040C0002DB97B4A107810B9774C32212180012418
:1040D00008E0774D2A7832B16F48417819B9754BAD
:1040E000297001241C700023734C1A4634F8020F07
:1040F00040F2135501B2A942CCBF0025012505FAB3
:1041000003F5A0F21550B0F5C77F8CBF0020012049
:104110002A435D1C00FA05F0024340F2A46081428C
:10412000D4BF00210121981C01FA00F103330A4396
:104130000C2B92B2DAD1002354485A4900EB4300C9
:10414000B0F8420002420CBF002001205854013355
:10415000152BF1D14A7822B1022003F0EFFC28B9E7
:104160000DE0FFF7DDF80028F6D108E04A4AD378E1
:1041700043B9524901200B604B60D07002E04648C1
:104180000021C170474A444B917839B11879002118
:10419000D97020B9494A0121106050601971414B12
:1041A000187810B93C4901220A70202003F0C6FC9F
:1041B000002852D0384BD87A1A46002848D04049B7
:1041C0000878042844D93748817A79B1DA79002A05
:1041D00043D13C480121D9711A723B4B011D1A7021
:1041E00002F044FD394A0220107036E0C27AD971DB
:1041F0001AB326483649B0F8C820B1F900000028A3
:10420000B8BF4042904218DAB1F902100029B8BF95
:104210004942914211DA187AF8B901241C722A4BEA
:104220002C4918702C480A684B68011D02604360D5
:1042300002F01CFD254804700FE02348164B01785E
:1042400000221A7249B90122027002F037FC04E020
:104250000023D37113721D4A137012490E4B087B51
:1042600000B101200E4A98725179082901D00E2917
:1042700051D1094B002058724DE018480368042BB7
:1042800049D8DFE803F02D2F323541000817002010
:10429000F0070020AC070020CB1C00200C1D0020E4
:1042A000D4170020DC1C0020BC070020E6070020FB
:1042B000B40700208C070020121D0020E807002012
:1042C000EA1B0020B01B0020100000208D070020FA
:1042D000A01B0020CC1B0020901B0020CC0700203E
:1042E0000122026001684B1C03600268511C0160DE
:1042F000384803685A1C02604FF48070FEF77EFC59
:1043000010B102F04DFD06E03248002101604FF48B
:104310000050FEF773FC01F0B5F82F4A2F491060EA
:104320008A892F4B1AB11968411A002951DB80186C
:10433000186001F0EDFBFFF75DFB01F0A3F8294BDE
:10434000254A196810601860421A2748274990F8D2
:1043500072300A8053B12649CA780AB9087928B15F
:10436000244B2549DA8808888118D980202003F059
:10437000E5FB40B11E4BD87908B91A7A1AB1197BFE
:1043800009B103F055FB1D4B1868804701F01AFF77
:1043900001F096FEBDE8384001F0EEBE69780029D4
:1043A0003FF495AD03F0EAFB91E5012402E002241D
:1043B00000E00324E5B2094B0020691E83F8941342
:1043C0000146FEF7B7FB022028212A4606F04EF9E7
:1043D000E4E538BDCC070020F8070020D417002002
:1043E000B8070020B007002008170020E4070020CD
:1043F000CB1C0020A01B0020400C00200C00002043
:10440000F8B5614B188800283BD000231A46B0F558
:10441000C87F5E4901D100248C505D4C8E581F5FCF
:104420005A4DF6198E50002119535A4C04321E1958
:104430000233062BA6F8F810E9D101281DD12A680D
:104440004FF4C87302F1C80292FBF3F2A4F8F8200B
:104450006A68C83292FBF3F2A4F8FA20AA68C8325C
:1044600092FBF3F34C4A12889B1A4C4AA4F8FC3096
:10447000518591850146FEF75DFB434801884B1E3F
:1044800003800420FEF7BAFB00286BD0444A128850
:10449000322A11D13F4C434DB4F8F860B4F8FA0019
:1044A000B4F8FC102E806880A9803C4D3E4B6C8D8A
:1044B000AE8D1C805E8001E0002A32D000231946B8
:1044C000322A3A4801D100254550314D44585E5FAB
:1044D000A61946502F4800245C531D18023304319E
:1044E000062B2646A5F8F840EAD1012A16D1304B12
:1044F00030491A70304B0C7002211970294B198801
:10450000A0F8F81059889B88A0F8FA102649A0F85E
:10451000FC30224B0888498858859985204B013A00
:104520001A8026480178E9B1002303701F48194A10
:104530000468322194FBF1F4A2F8F84044688068E2
:1045400094FBF1F490FBF1F11348A2F8FA400088D3
:10455000091AA2F8FC100120104A014653859385E0
:10456000FEF7E8FA0A4B0B4A1888B2F8F810401A1E
:104570001880B2F8FA105888B2F8FC20401A9988CE
:104580005880881A9880F8BD0C0800201008002078
:10459000541C0020D417002012000020081700200F
:1045A000BC0700201C080020240800200008002070
:1045B000B4070020E6070020560700208C070020E3
:1045C00008B5044B044859688847BDE80840FFF720
:1045D00017BF00BF041C0020541C00202DE9F84F19
:1045E000414B188800286ED00024254626463E49B7
:1045F0000A88B2F57A7F08D13C4B3D490027142048
:10460000EF5000FB0610FEF7ADFCDFF8F0A0374FCF
:104610003AF90400EA59DFF8D8901318EB51FCF787
:1046200075FA4FF0140B0BFB069B01464FF0000888
:104630005846FEF79AFC24F80A80DFF8ACA02D4813
:10464000BAF8001024F80080012933D15846FEF74B
:10465000CEFC294A834692F8F400E0B1FCF756FA02
:1046600001465846FCF762FCA8B14FF47A714846FF
:10467000AAF80010FEF776FC09F11400FEF772FCB0
:1046800009F12800FEF76EFCC7F80880C7F804801F
:10469000C7F800800EE0154B4FF47A72E858154BBE
:1046A00000F5FA7191FBF2F0E0520F210A2001228D
:1046B00005F0DCFF013604350234032E97D10A4899
:1046C0000288531E03800D4B0A4A18881188401A2D
:1046D0001880518858889288401A99885880881A7A
:1046E0009880BDE8F88F00BF7208002064080020A1
:1046F00028080020220C0020D41700203C1C002099
:1047000008B5044B044859688847BDE80840FFF7DE
:1047100065BF00BF201C00203C1C00202DE9F34198
:10472000444C45484549B4F8EE20FCF79BFE98B947
:104730004248B4F8EE10FCF77BFF08B100270CE00C
:104740003E48B4F8EE10FCF789FD07460028F5D185
:10475000032000F033FF00E00127364B93F8ED0013
:10476000052827D8DFE800F007071B2626030220CC
:1047700003F0F6F91EE000218DF804104FF44872A2
:1047800001A82D49ADF80620FCF7C2FC10B12C4B56
:1047900001241C70274890F8ED1001290AD04FB170
:1047A000244A25482549B2F8EE20FCF75BFE244B4D
:1047B00002241C70224802784AB91E4C94F8ED106D
:1047C00011B184F8ED20C8E7022003F0C9F90220F6
:1047D00003F0B4F9174F20B1174B97F8E3001A68AC
:1047E00090471648046897F8E200A047154908204A
:1047F0000F8D03F0A3F9144CC0B13FB2642697FBB0
:10480000F6F52846FCF782F906FB1572804610B2D1
:10481000FCF77CF90D49FCF7CDF901464046FCF761
:10482000C1F80B49FCF7C6F9206001E000232360C2
:10483000BDE8FC81D4170020041C0020201C0020AF
:104840002208002008170020440C00208988883C9A
:10485000000020412DE9F84F9C4C2068838A9BB2D0
:1048600013F0010239D0018821F400631A04110CFD
:104870000180012106F0C2FE954A964B1178002076
:104880001870D9B1944803781BB9944A1178FF295C
:1048900014D10123037092480278022A06D18B4971
:1048A0000B68188882B242F4006119808D4B8748EA
:1048B00019780068012206F0BBFE2FE18948834B7E
:1048C00001780022186806F0B3FE844A1178FF29A7
:1048D00000F02481FF207F4BDEE003F00201C9B22B
:1048E00000293DD0BFF35F8F7D4D2E78012E3546D8
:1048F00016D177490B789BB177490B7883B1114674
:1049000006F07CFEBFF35F8F20683146038B06F014
:1049100069FE754A206816704FF480613246FBE0EC
:10492000038BBFF35F8F6E490A78022A09D1684B67
:104930001A7832B1684B1A781AB1002106F05EFE7F
:10494000E5E00978032907D1614B1A7822B1624961
:104950000B78002B40F0DD804FF480610122DBE01A
:1049600003F00406F6B2002E71D0594BDFF87881BF
:104970001A78012688F80060574B002A4DD01A7823
:10498000002A4AD0564D2F78524D022F574F29D921
:1049900006F034FE206895F80090D7F800A006F0E5
:1049A00044FE4FFA89FB0AF80B0009EB060031467A
:1049B0002870206806F016FE206888F800603F68BE
:1049C00095F8008006F031FE4FFA88F907F80900E3
:1049D000B04420684FF48061324685F8008006F0CC
:1049E00019FE2BE0314606F0FDFD20682E78D7F841
:1049F000008006F01AFE4FFA86F9731C08F80900C9
:104A0000D9B220684FFA81F83F68297006F00DFE90
:104A1000033607F808002E7010E01B78012113B947
:104A2000334A13782BB106F0DDFD2A480278511C79
:104A300003E006F0CBFD284801210170234A1168EC
:104A40000B8803F4807082B2002AF9D166E003F08B
:104A500040010F461F4D09B3244B2F78D3F8008037
:104A600006F0E3FD4FFA87F908F80900781CC1B297
:104A700029701B4D4FB22A780337BA4205D12068FE
:104A80004FF48061324606F0C5FD124B28781A7843
:104A900051B2884242D1501C18703FE01B063DD5F0
:104AA0002B785EB2721C27D0124901330A682B7032
:104AB000915D06F0B8FD0A4895F900200178914211
:104AC0002CD120684FF480613A4625E08C08002004
:104AD0008A08002088080020890800207708002024
:104AE0007808002091080020760800207C0800202B
:104AF0008008002084080020154A2970117806F0EB
:104B000092FD1448017811B9134B1A7832B9134841
:104B100000684FF48061002206F07CFD0E4A104BC5
:104B2000117893F900004A1C90420ED10D4B0E49AA
:104B3000187800220A7028B1084908684FF44071BB
:104B400006F068FD094B00221A70BDE8F88F00BF1F
:104B5000770800208A080020780800208C080020B0
:104B6000880800207608002089080020900800208E
:104B7000FFF770BEFFF76EBEF0B5484C89B04FF43A
:104B800040651C2307460226204602A9ADF80850BE
:104B90008DF80A308DF80B6000F0B2F9404814210E
:104BA00007608DF80E10204603A9ADF80C508DF863
:104BB0000F6000F0A5F925610825384CA268520560
:104BC00003D40A2000F07EFCF7E74FF480660A2049
:104BD000666100F077FC6F1E0A20266100F072FC0F
:104BE00017F0FF05E9D14FF4006767610A2000F074
:104BF00069FC66610A2000F065FC26610A2000F06D
:104C000061FC022027611C218DF80F002046244CF6
:104C10004FF440638DF80E1003A9ADF80C3000F08E
:104C20006FF9206806F034FC04A806F0B5FC206893
:104C30002A464FF4407106F0EDFC1A484FF48043C9
:104C40004BF6FF72049001212068ADF81C30ADF8DE
:104C50001620ADF8145006F0ADFC04A9206806F04B
:104C600031FC4FF4A06005F02FFF2221012201A8A2
:104C70008DF804108DF805508DF806508DF807203A
:104C800005F02CFF212301A82E468DF804308DF865
:104C9000055005F023FF09B0F0BD00BF000C014036
:104CA0008C080020801A060010B54000244CC0B2C9
:104CB00020702448244C017000212170234C0120D5
:104CC0002070234C2360234C2360234B1A70234A0B
:104CD00010702348017023490868838803F4007228
:104CE00091B2A1B9038803F4807291B241B90388EB
:104CF00003F4007291B20029F9D1012106F066FC9B
:104D000018484FF440710068012206F083FC47F216
:104D10003053124A117811B1013BFAD100E053B976
:104D200011490A88501C83B20B800E490868FFF7AE
:104D300023FF002010BD0A4B187880F0010010BD41
:104D40009108002077080020800800208A080020B1
:104D50007C080020840800207808002090080020AB
:104D6000810800208C0800207408002010B5400045
:104D7000244CC0B220702448244C017024490120E6
:104D8000087000212170234C2360234C2360234BA7
:104D90001A70234A107023480170234908688388D9
:104DA00003F4007291B2A1B9038803F4807291B246
:104DB00041B9038803F4007291B20029F9D10121AD
:104DC00006F004FC18484FF440710068012206F018
:104DD00021FC47F23053124A117811B1013BFAD14C
:104DE00000E053B911490A88501C83B20B800E4968
:104DF0000868FFF7C1FE002010BD0A4B187880F04C
:104E0000010010BD91080020770800208A080020CA
:104E100080080020840800207C08002078080020FA
:104E200090080020810800208C08002074080020D1
:104E300007B502AB03F8012D0122FFF797FF0EBD66
:104E4000274B37B51868818A8AB20192019B13F407
:104E5000706F02D0234A01211170019B13F4E06F9F
:104E600031D04FF480610022038B06F0D3FB019810
:104E7000810528D41A4D2868018801F4007293B284
:104E80000BBB048804F480718CB29CB1028802F4DC
:104E9000807399B20029F9D1012106F0A3FB1048D3
:104EA0000068028802F4007399B20029F9D1FFF773
:104EB00063FE08E0012106F095FB28684FF440717D
:104EC000224606F0A7FB06480268938A23F4706125
:104ED0000804030C0449938200220A703EBD00BFFF
:104EE0008C0800208108002090080020FFF7A8BF50
:104EF000FFF7A6BF014B188880B2704774080020E6
:104F00002DE9F0410F88002347FA03F2D2072DD58F
:104F10008A7803F00705DC08AD0012F0100F18BF07
:104F200091F803C002F00F0618BF46EA0C064FF0D6
:104F30000F0C0CFA05FC06FA05F550F82480282A17
:104F400028EA0C0C45EA0C0540F8245006D1012251
:104F500002FA03F2C46824EA020206E0482A05D1F4
:104F6000012202FA03F2C4682243C2600133102B0B
:104F7000CAD1BDE8F08108B503681A68904708BD3A
:104F800038B505460C4614F8011B19B12846FFF741
:104F9000F2FFF8E738BD08B503685968884708BDCF
:104FA00008B503689968884708BD08B50368DA68DA
:104FB000904708BD08B503681969884708BD08B55A
:104FC00003685A69904708BD7047036B13B15A686C
:104FD000006C01E0026AC069101A18BF0120704716
:104FE000436B13B190F844007047826A406A111A0B
:104FF0004B4253EB01007047836A8169426BC918C9
:10500000D160416A994203D9CB1A5360816204E0AE
:105010000169CB1A536000228262002180F844109B
:10502000406B012106F0B1BB30B50446007985B074
:1050300000230D460091C107ADF80430ADF80630ED
:10504000ADF80830ADF80C30ADF80A3002D50422C6
:10505000ADF80A20820705D5BDF80A1041F0080313
:10506000ADF80A30A06C694606F070F8A56005B08E
:1050700030BD026B034610B5406942B11A6CD96865
:105080008C1A013A18BF1146005D196410BD196AE7
:10509000DA68405C0131B1FBF2F402FB14111962D1
:1050A00010BD10B5426A8469A154416A0269013198
:1050B000B1FBF2F402FB1411426B416232B113688E
:1050C000DB070BD4BDE81040FFF796BF806C40F2C1
:1050D00027710122BDE8104006F09CB810BD000009
:1050E000214B13B5986021480C4658612048214A4D
:1050F0002149186314381A6099614FF4807258631B
:1051000001214FF48040DA601A6106F089F94FF40A
:10511000007102231822ADF80010A1078DF80330AA
:105120008DF8022003D515486946FFF7E9FE4823AC
:105130004FF48060E207ADF800008DF8023003D52F
:105140000E486946FFF7DCFE01220E2101A88DF80A
:1051500004108DF805208DF806208DF8072005F045
:10516000BDFC01481CBD00BF540B0020520A0020AA
:105170005800024084EA0008D208002000080140DC
:105180001F4B13B51F4A98600C4680204021D86001
:1051900019611D481D491A601D4A986199644FF4B0
:1051A000003001215A6106F047F902230422182039
:1051B0008DF80330A307ADF800208DF8020003D569
:1051C00014486946FFF79CFE08214823E007ADF824
:1051D00000108DF8023003D50E486946FFF790FEA7
:1051E000012026228DF8050002218DF8070001A874
:1051F0008DF804208DF8061005F070FC00481CBDE9
:10520000A00B002084EA000892080020004400401F
:10521000D2090020000801402DE9F0411E46584BFC
:1052200090B0984205468846174604D1104631464C
:10523000FFF756FF07E053480024854204D110468B
:105240003146FFF79DFF0446002106F00402267157
:10525000A7600197A5642162E161A1626162C4F85F
:105260002C80ADF8081002F0FF0732B14FF4005364
:10527000ADF80A304FF4806701E0ADF80A70002005
:10528000ADF80C7016F00107ADF8100002D1ADF8C2
:105290000E7002E00421ADF80E1006F0020606F0D2
:1052A000FF082EB1BDF80E2042F00803ADF80E3015
:1052B000284601A905F04AFF0121284605F09EFF76
:1052C00005A806F055FA0023281D4FF480518022CE
:1052D00005900E910F9309930B930A920C9317B3B9
:1052E000206BD0B16269E168079320230D93069289
:1052F000089106F0A5F9206B05A906F019FA206BB4
:10530000012106F042FA28464021012205F09CFFC7
:10531000206B06F04FFA206405E0284640F2255144
:10532000012205F077FFB8F1000F24D0606BE0B1E7
:10533000266910210896002607910D9606F080F93F
:10534000606B05A906F0F4F90122606B022106F0FA
:1053500027FA606B314606F02BFA606B80214660BD
:105360000122284605F070FF05E0284640F227712B
:10537000012205F04FFF204610B0BDE8F08100BFCC
:10538000003801400044004010B50B4C4FF4005071
:1053900006F014FA0021606B06F0F7F9626AA36A5E
:1053A0009A4204D02046BDE81040FFF725BE0120F8
:1053B00084F8440010BD00BF540B00200D4B986CC6
:1053C000028802F080018AB29AB19A6A596A8A42C6
:1053D0000AD09969895C013281801969B2FBF1F0C8
:1053E00001FB10229A62704740F22771002205F0FB
:1053F00011BF7047540B00201C4B10B59A6C1488D9
:10540000A4B204F0200188B290B1D96A19B193888E
:1054100098B288470CE09288D9695869D2B2425450
:10542000D869DA68411CB1FBF2F002FB1011D961B6
:1054300004F08004A4B2C4B10C4B9A6A586A824248
:105440000BD09869996C805C013288801969B2FB35
:10545000F1F001FB10229A6210BD986C40F22771A6
:105460000022BDE8104005F0D5BE10BDA00B002005
:1054700070470000024B1A68501C1860704700BF4C
:10548000EC0B002010B5094A094913688C681068B4
:105490008342F8D1074A106811684FF47A7250437A
:1054A000001BB0FBF1F102FB031010BDEC0B002060
:1054B00010E000E0F00B0020014B1868704700BFBF
:1054C000EC0B002038B50446FFF7DCFF0546FFF77C
:1054D000D9FF401BA042FAD338BD10B504462CB109
:1054E0004FF47A70FFF7EEFF013CF8E710BD0000C3
:1054F00010B586B005F034F90121254805F09CFF70
:10550000012144F61D2005F08BFF0120014605F026
:105510007BFF002405F0B4FF4FF6FF7369461D487A
:10552000ADF800308DF80240FFF7EAFC69461A48F2
:10553000FFF7E6FC69461948FFF7E2FC18484268A5
:1055400042F000714160FFF793FF01A805F00EFFE4
:10555000019B1448144AB3FBF0F114481160016830
:105560004FF47A73B1FBF3F2114B501E114A58609D
:10557000F021072082F823109C6018600E48FFF786
:10558000FBFAFCF72FF96420FFF7A7FF06B010BD68
:105590000700400000080140000C014000100140DD
:1055A0000000014040420F00F00B0020500100209D
:1055B00010E000E000ED00E00058004010B540F2BF
:1055C000DB146043841E2046FFF787FF1920FFF796
:1055D00084FFF8E710B1034A034B1A6003480449FB
:1055E000C8607047EFBEADDEF04F00200400FA0542
:1055F00000ED00E0000000002DE9F84F384E0446B1
:105600003768384606F0E4F80546384606F054F99F
:1056100076688046304606F0DBF88346304606F072
:105620004BF9D4F80490064629464846FBF7C2FADF
:10563000A768824641463846FBF7BCFA0146504609
:10564000FBF7AEF9216882465846FBF7B3FA4146AC
:1056500004464846FBF7AEFA3146FBF7ABFA014683
:105660002046FBF79FF9314604463846FBF7A2FA7D
:105670002946FBF79FFA01462046FBF793F90146BE
:10568000504606F0A5F91749FBF794FAFAF7CEFE53
:1056900011A3D3E90023FBF747F8134B044618681E
:1056A0000D46FAF7C3FE02460B4620462946FAF796
:1056B0005FFD00220D4BFBF737F8FBF71DF906F0F5
:1056C000BBF881B20A0444BF00F5B47189B208B2D4
:1056D000BDE8F88FAFF30080182D4454FB2109403A
:1056E000140C00200000E144440C00200000244081
:1056F00010B5194C2088FBF709FA1849FBF75AFA3C
:1057000006F09AF8164B18802088FBF7FFF901463F
:105710001448FBF703FB1449FBF700FB134908602F
:105720001348B0F87000FBF7F1F901461148FBF798
:10573000F5FAFAF77BFE06A3D3E90023FAF7CAFECF
:10574000FBF7DAF80C4A106010BD00BFAFF3008021
:105750003B597E90A9E7814012000020C903683FB1
:10576000100C00200AE81C4100401C46501C002080
:1057700008170020000061446C1C0020AFF300807B
:105780002DE9F041044600680D460146FBF712FA88
:10579000D4F80480064641464046FBF70BFA014622
:1057A0003046FBF7FFF8A768064639463846FBF750
:1057B00001FA01463046FBF7F5F806F00BF9002137
:1057C0000646FBF78BFB70B920683146FBF7A6FA5B
:1057D000314628606068FBF7A1FA31466860A0682E
:1057E000FBF79CFAA860BDE8F0812DE9F04F0C684A
:1057F000836889B0D0F800A0D0F80480064620461F
:1058000003938B4605F0E4FF0746204606F054F864
:10581000DBF804408146204605F0DAFF05462046C5
:1058200006F04AF8DBF8082004461046019205F01D
:10583000CFFF8346019806F03FF83946029058465C
:10584000FBF7B8F9394604900298FBF7B3F95946CB
:1058500005904846FBF7AEF9029906904846FBF7DB
:10586000A9F9294607905846FBF7A4F90146504686
:10587000FBF7A0F9214683460698FBF79BF9014602
:105880000598FBF78FF801464046FBF793F9014670
:105890005846FBF787F8214683460498FBF78AF9B8
:1058A00001460798FBF77CF801460398FBF782F95D
:1058B00001465846FBF776F83060029905F1004042
:1058C000FBF778F901465046FBF774F92146834609
:1058D0000798FBF76FF901460498FBF761F801465A
:1058E0004046FBF767F901465846FBF75BF821464F
:1058F00083460598FBF75EF901460698FBF752F8D8
:1059000001460398FBF756F901465846FBF74AF85B
:10591000214670605046FBF74DF92946044609F1CF
:105920000040FBF747F901464046FBF743F90146C3
:105930002046FBF737F8394604462846FBF73AF984
:1059400001460398FBF736F901462046FBF72AF893
:10595000B06009B0BDE8F08F1FB50B684A68896870
:105960000193039101A90292FFF73FFF05B000BD2B
:1059700080EAE073A3EBE0738B4206DB002801DDD5
:10598000401A704702D0401870470020704700004E
:105990002DE9F041524B86B01A685B6802F1004273
:1059A00003F1004301934F4B0646B3F90000009208
:1059B000FBF7ACF800F10040FAF738FD46A3D3E955
:1059C0000023FAF787FDFAF797FF474C0290B4F9E6
:1059D0000000FBF79BF80390B4F90200FBF796F880
:1059E0000490B4F90400FBF791F86946059003A808
:1059F000FFF7FBFE3D4B93F84030012B16D13C489E
:105A0000417869B93B4C4025226892FBF5F7D01BE1
:105A1000FBF77CF80599FAF7C5FFFBF791FA2060D0
:105A2000344B4021186890FBF1F001E0324B1888AC
:105A3000FBF76CF801460598FAF7B2FF059030467F
:105A4000FBF760F82D490746FAF7ACFF01463846E8
:105A5000FBF764F92A4D07462C6805982146FAF7AA
:105A60009FFF01463846FBF7A5F801462046FAF7A6
:105A700099FF244C28601D4D07460398D4F80080F8
:105A800005F0DAFE95F83010FFF772FF08EB000220
:105A900004982260D4F8048005F0CEFE95F830100A
:105AA000FFF766FF08EB000338466360D4F8088010
:105AB00005F0C2FE95F82F10FFF75AFF1249134B5D
:105AC0000A684044A0601868B6180E60411C19604E
:105AD00006B0BDE8F08100BF399D52A246DF913F7C
:105AE000140C0020361C0020641C00200817002025
:105AF000CB1C0020F40B0020120000203661823CF9
:105B0000340C0020441C0020280C0020380C0020FD
:105B10002DE9F04F87B0FEF7F3FD022002F00EF8FA
:105B2000002800F0A781FEF74BFDFFF7ABFCAA4C65
:105B300005462768C71B3846FAF7E4FFA749C96836
:105B4000FBF738F88346A648256090F82E8000259C
:105B50002C462E46A34A105FFAF7D8FF5946FBF7AA
:105B600029F803AB5851B8F1000F27D04046FAF797
:105B7000CDFF01464FF07E50FBF7D0F8DFF8A4923E
:105B8000824651464FF07E50FAF70AFF55F8091049
:105B9000FBF710F894490346085F0193FAF7B6FF44
:105BA0005146FBF707F801460198FAF7FBFE49F862
:105BB0000500FBF7C5F98D4A105303E08A498B4A6B
:105BC000605AA052894B0435E15E0234062C01FB79
:105BD0000166BFD1864A6420138846435B438548EB
:105BE00003A996FBF3F6FFF7B7FE082001F0A6FF26
:105BF00020B1814803A9FFF7AFFE07E07F4803A962
:105C0000FFF7AAFE7D480146FFF7BAFD493EB1B253
:105C10003B2904D9082001F091FF48BB50E0784CA3
:105C2000B4F8F000FAF76EFF4FF07E518046FAF7B5
:105C3000B9FE01464FF07E50FBF770F8002406468F
:105C40006C4D404655F81410FAF7B4FF814667488A
:105C5000005FFAF75BFF01464846FAF7A3FE3146BC
:105C6000FAF7A8FF45F814000234062CE8D1D1E772
:105C7000634A0024B2F8F200FAF744FF4FF07E5175
:105C80008046FAF78FFE01464FF07E50FBF746F84C
:105C90000646594D404655F81410FAF78BFF594BFC
:105CA0008146185FFAF732FF01464846FAF77AFE56
:105CB0003146FAF77FFF45F814000234062CE8D18C
:105CC00051494C4DB1F90000FAF720FFAC6801468C
:105CD00020460126FBF72AF900B906464B48214623
:105CE0004673686805F074FE494C2A68206068684D
:105CF00002F100460146FAF75DFFD5F80880054637
:105D000041464046FAF756FF01462846FAF74AFE52
:105D100005F060FE0146304605F05AFE60602068DE
:105D2000FAF784FB2AA3D3E90023FAF7D3FBFAF7A7
:105D3000E3FD05F081FD374D28806068FAF776FBBA
:105D400023A3D3E90023FAF7C5FBFAF7D5FD05F045
:105D500073FD6880082001F0F1FE2F4C08B1264841
:105D600000E02648FFF748FC1D4D20803846FFF72D
:105D70000FFE95F87230002B00F080801D490868F6
:105D80008C684F680146FAF715FF394606463846D3
:105D9000FAF710FF01463046FAF704FE21460646A0
:105DA0002046FAF707FF01463046FAF7FBFD05F0FB
:105DB00011FE01462046FAF7B1FF18490446FBF7E9
:105DC000A1F888B3164A0020108057E0AFF3008096
:105DD0003B597E90A9E781403C0C0020201C00200C
:105DE000081700203C1C0020541C0020641C0020CC
:105DF00012000020701C0020F80B0020140000206E
:105E0000D4170020181C0020100C0020CB1C0020F0
:105E1000140C00202C0C0020361C00208FC2753C76
:105E2000400C0020040C0020204605F081FD264B8C
:105E30001968FAF7BFFE05F0FFFCB0F5617FA8BF57
:105E40004FF46170FAF7E0FA1DA3D3E90023FAF7E3
:105E50006BFCFAF751FD05F02FFD044695F8720032
:105E6000FAF754FE2146FAF7A5FE05F0E5FC174BBC
:105E7000188003E0164B188058809880154B59798C
:105E8000154B012907D015481A8859889B8802802C
:105E90004180838011E01249B3F90420B1F9000078
:105EA00002EB4000032290FBF2F080B20B4A088024
:105EB00019885B8890801180538007B0BDE8F08F0F
:105EC000A2EB0FE5DD1696406C1C0020400C002074
:105ED000541C0020D41700203C1C00201C0C002067
:105EE000420C0020AFF3008010B5054C0020218843
:105EF000FBF726FF61880120BDE81040FBF720BFBB
:105F0000200000200A4A02EBC00393F87B10FF290F
:105F100004D019B1074830F8110007E00728DABFAC
:105F200002EBC000B0F8780040F2DC5000B27047DD
:105F3000081700200C1D002010B500244FF48040ED
:105F4000FCF75CFE064B10B1B3F8DA0001E0B3F8E1
:105F5000D400044AA0520234182CEFD110BD00BF67
:105F6000D4170020941C0020F8B53B4D3B4E6B79B4
:105F70003B4C06EBC300417820202160FCF73EFE3D
:105F8000324608B1012626606B79162B1CD10024FD
:105F9000314E0021A6193069FAF7A0FF28B14FF45D
:105FA0008040FCF72BFE50BB23E02E4B06F1100087
:105FB0001D190FC885E80F002B4910340A78531CAF
:105FC000C02C0B70E4D1EAE7274F12F8336002EBE4
:105FD000C3003E704768002FE1D00024B442DEDAEF
:105FE000204D21016D187A180FCA013485E80F0081
:105FF000F4E719481D4B4179082923D124E01A4EB2
:106000003678012EF5D91A4C00251034B542F0DA55
:1060100054F8100C4FF07C51FAF7CCFD4FF07C5146
:1060200044F8100C54F8140CFAF7C4FD4FF07C51EE
:1060300044F8140C54F80C0CFAF7BCFD013544F884
:106040000C0CE2E70E2901D1012200E000221A74B3
:10605000BDE8F840FFF770BFD41700200CEC000833
:10606000500C0020580C00204C0C0020CB1C0020B1
:10607000600C0020F0B50023461C0E4A0021981841
:106080001033C02B0161F8D10B4F07EBC6035F68DB
:1060900007B9F0BD0024084A12F83600844208DA35
:1060A000064D21014D197B180FCB013485E80F00F7
:1060B000F1E7F0BDD41700200CEC0008E417002035
:1060C000284B10B5186800284AD027494A79531E32
:1060D000142B3DD8DFE803F00B3C3C24403C3C1C37
:1060E0003C3C3C3C3C2C3C3C3C3C3C242C001F4875
:1060F00090F8BB1031B11E4B00205989BDE810400B
:10610000FBF71EBE1B4A50780028F4D10146F5E784
:10611000174C0020E188FBF713FE01202189EDE7F1
:10612000134C00202189FBF70BFE01206189E5E774
:106130000F4C0020E188FBF703FE01202189FBF7CB
:10614000FFFD02206189FBF7FBFD0320A189D5E754
:106150002020FCF753FD18B1BDE81040FFF7C4BE86
:1061600010BD00BF500C0020D417002008170020DD
:1061700020000020CB1C002010B50024064B18780E
:10618000A04208D90549204631F814100134FBF724
:10619000C9FDE4B2F2E710BD4C0C00207C1C0020CD
:1061A000064B1A780023D9B2914204D2044921F84F
:1061B00013000133F7E7FFF7DFBF00BF4C0C0020EF
:1061C0007C1C00202DE9F84FB24B187803280FD91A
:1061D000B149B24CB1F904206FF06305002AB8BF91
:1061E0005242A91AB4F904006432FCF7B3FEA0804D
:1061F000A84A1678012E1DD8A94EAA4C75796A1E98
:10620000142A00F2F981DFE812F0C200F701F70169
:106210008400D500F701F7017101F701F701F701DB
:10622000F701F701F100F701F701F701F701F701B5
:106230005E00C7019B48994B90F9BA90964FB3F90D
:106240000440C9F10001B7F806A004FB01F95F881A
:10625000B3F80080944C00251034B542CCD20FFA2C
:106260008AF0FAF753FC54F8101CFAF7A3FC8346A3
:1062700038B2FAF74BFC54F8081CFAF79BFC0146BD
:106280005846FAF78FFB83460FFA88F0FAF73EFC80
:1062900054F80C1CFAF78EFC01465846FAF782FBBC
:1062A00083464846FAF732FC54F8041CFAF782FC9D
:1062B00001465846FAF776FBFAF742FE7B4B23F885
:1062C00015000135C8E794F89A20744D12F0010FBB
:1062D0006B880CBF01264FF0FF365E43744CB7B29B
:1062E00004202781FFF70EFE29886E4D381895F897
:1062F000A230208113F0010F0CBF01224FF0FF32BA
:106300004A43052096B26681FFF7FCFD3718678186
:1063100072E194F89A50614805F002084FFA88F645
:10632000002E0CBF01214FF0FF3115F0010F458801
:106330000CBF01224FF0FF326A438688042001FB24
:1063400006F497B2FFF7DEFD1FFA84F808EB0003AE
:106350005448F91890F8A270554C07F0020253B255
:106360002181002B0CBF01214FF0FF314E4317F06C
:10637000010F0CBF01204FF0FF3045430520FFF710
:10638000C1FDB6B2ADB23718EA19628134E14349B2
:1063900094F8A2408E8814F0010F0CBF01234FF037
:1063A000FF3305205E43FFF7ADFDB5B2404F28181F
:1063B000788121E10020FFF7A5FD3E4F94F97A3066
:1063C000B7F902603A4D7343322693FBF6F1401859
:1063D00028800120FFF796FDB7F9002094F982404C
:1063E000544394FBF6F3C7186F8005E1324C607894
:1063F00020B9B6F8D4202E4BDA810AE02649B6F847
:10640000D220B1F90600B6F8D010FCF7A3FD284D54
:10641000E881274E254CF7892780214F97F81901ED
:1064200030B3204D0220FFF76DFDB5F98410B5F9AA
:106430008620FCF78FFD214BB7F812111A880C1A31
:1064400016B220B2864203DA97F81961B41803E055
:1064500003DD97F81971D41B1C8095F98A50B3F9A4
:10646000003064226B43124F93FBF2F00918B9809D
:10647000114C0F4DA67A56B1074B1A880324EA80B7
:106480002A81988868815988A981094D18E0034BB1
:10649000F3E700BF4C0C0020A01B0020A81B00202D
:1064A000D417002008170020580C00207C1C002066
:1064B000200000202C0C0020CB1C0020540C0020BD
:1064C000AA4FB5F9062007EBC40696F97A30642086
:1064D0005A4392FBF0F7EF802046FFF713FD01349B
:1064E0003918E9800235072CEAD185E0A04B5A78AB
:1064F00022B9B6F8D4709F49CF810AE09E48B6F819
:10650000D010B6F8D220B0F90600FCF723FD994E62
:10651000F081964E974B964A96F89270974DDC898B
:10652000907A17F0010F2C800CBF01254FF0FF353A
:1065300008B1914900E09249488807F002044543B8
:1065400096F89A60098862B2002A0CBF01274FF0C2
:10655000FF3716F0010F0CBF01244FF0FF3407FB8B
:106560000155604306F0020257B2DD80002F0CBFD8
:1065700001254FF0FF3505FB010018810320FFF7CF
:10658000C1FC7C4EF388C1180420F180FFF7BAFCEF
:106590003489021932812FE0794F0324BF88734B6D
:1065A00003EBC40090F87A60C4F1060306F0020120
:1065B0004DB2002D0CBF01224FF0FF327A437049DB
:1065C000580831F8105016F0010F0CBF01264FF09B
:1065D000FF3606FB0522674D96B225F8146020466B
:1065E000FFF790FC331825F814300134072CD6D16E
:1065F000614F6249F88808802020FCF7FFFA0028E4
:1066000041D00020FFF77EFC5A4C05462080012037
:10661000FFF778FC5B4A6080137AA3B3534F5A4A62
:1066200097F8BC1001F00206F3B2CBB1B2F900301A
:1066300097F9821097F97A70B2F9022059437B4298
:106640005343322691FBF6F16FF0310789B293FB89
:10665000F7F28F187D1993FBF6F625808E1910E05E
:1066600097F97A10B2F9026097F982704E43B2F945
:1066700000203221574396FBF1F3ED18258097FB5C
:10668000F1F680196080414C384D04F11006B4F9E0
:106690000200B5F97410B5F97620FCF75BFC24F81C
:1066A000020F0835B442F2D1304991F8BC3003F002
:1066B0000402D7B22FB93148354B07881C78012224
:1066C0001CE0344D68790E280AD0082808D0324CD6
:1066D00004EBC0014B78002B14BF0225002500E01D
:1066E000042500242D4F621907EB4401D0B209891B
:1066F0000134FBF725FB042CF4D1DCE7A24209D2DC
:106700001E483FB230F912100132B942A8BF0F46FD
:10671000BFB2F3E70024A0461D4A1178884567D22E
:106720001C4D3BB2B5F8D200834204DD134DC21BB1
:10673000615B501860534FF48040FCF75FFA0F4DD7
:1067400070B3164B40F2DC51B3F90620114B8A426C
:10675000285FC7BFB3F8D810B3F8D220B3F8D4106D
:10676000B3F8D620FCF7F6FB285336E008170020D4
:10677000CB1C002020000020A01B00207C1C00203F
:10678000A81B0020DC1C00202C0C00201E00002078
:106790004C0C0020D41700200CEC00080C1D00202D
:1067A000144E285FB6F8D010B6F8D220FCF7D2FB12
:1067B000114BB6F81411B3F9062005EB04098A420F
:1067C00028530ADA1020FCF719FA10B9B6F8D000ED
:1067D00001E0B6F8D400A9F80000084A507818B9CA
:1067E0000749084B625AE25208F10108023493E764
:1067F000BDE8F88FD41700200C1D0020CB1C002012
:10680000941C00207C1C0020024B1868003018BF2C
:1068100001207047500C002044F25063984203DD81
:10682000A0F50C40A038704703498842BCBF00F572
:106830000C40A030704700BFB0B9FFFF10B5FAF7A9
:1068400065F900210446FAF771FB08B1204601E022
:1068500004F100400549FAF761FA0549FAF7AAF987
:1068600004F0B6FF034B186010BD00BF8096184BB4
:1068700035FA8E3C3000002010B5044C0023207007
:106880002361FEF719FE606110BD00BFB01C00203F
:10689000F8B51D4614460E46FAF738F96968FAF756
:1068A00089F93146FAF786F92168FAF77BF8206012
:1068B000FAF746FBED68074605F10040FAF740FBA2
:1068C00006462846FAF73CFB314602463846FCF7B6
:1068D00041FBFAF71BF92060FAF732FBF8BD000024
:1068E000F8B5101A0C461F46FAF710F90546381B82
:1068F000FAF70CF9174B079E1968FAF75BF9294666
:1069000004462846FAF756F9214607462046FAF784
:1069100051F901463846FAF745F805F05BF80E499B
:10692000FAF748F9FAF732FB06990860214605F1B3
:10693000004005F04DF80949FAF73CF90849FAF723
:1069400031F8FAF7FDFA0028BCBF00F50C40A03082
:106950003060F8BD300000202C7D8E3FA00CB34588
:1069600000A00C4610B50446002003460D49CA5C41
:10697000A2B12E2A04D1013394B1C91800220A55BC
:10698000084A0A21D25C4843A2F13001092901D802
:10699000303880180E2B02D80133E7E710BD0020F5
:1069A00010BD00BF800D0020F8B52D4B93F81C01E1
:1069B00010B1012850D10AE02A4B2B4A58782B4BB2
:1069C00002EB001149685868FEF7EFFA41E0274DE5
:1069D0006868FEF7EFFA00283ED0224C2178264660
:1069E00001291ED1FEF768FD06466069321A632A46
:1069F00035D92169042912D81B4F686807EB0113A8
:106A00005968FEF7D2FA607807EB0017B968686832
:106A1000FEF7B6FA22696661511C21611CE0022072
:106A200018E022693AB964780F4B686803EB0411E7
:106A30004968FEF7BAFA33690A4C8B2B09D80C4A1D
:106A40000A48D15C4068FEF796FA21694B1C236125
:106A500002E00320FFF710FF024A00205060F8BD5B
:106A6000D4170020B01C00202CF10008501D00207D
:106A70009EF0000810B50B4CE37A8BB10A48017800
:106A800004290DD9094A0A4B1068516818605960E9
:106A9000FFF7D4FE0748084B028801211A802173B2
:106AA00010BD00BFCB1C0020EA1B0020CC1B002027
:106AB000B01B0020361C0020E20D0020002370B522
:106AC0001C460F4800211952142060430D4A0E4EF7
:106AD0000E4D995200223250595335180C4E6960B0
:106AE000AA60325035180B4E01346960AA60023337
:106AF0003518022C32506960AA60E2D170BD00BF27
:106B0000841B0020E0070020A00D0020881B00202F
:106B1000440D00201C0E002070B5204C204D6079E3
:106B2000F9F7F0FF1F49FAF7F9F82860E07BF9F769
:106B3000E9FF1C49FAF7F2F81B4E6860EE60A07995
:106B4000F9F7E0FF1949FAF7E9F8194D2860207CB8
:106B5000F9F7D8FF1349FAF7E1F86860A07EF9F772
:106B6000D1FF1449FAF7DAF8EE60A860E079F9F796
:106B7000C9FF0E49FAF7D2F80F4D2860607CF9F78B
:106B8000C1FF0849FAF7CAF86860E07EF9F7BAFF72
:106B90000849FAF7C3F8EE60A86070BD0817002036
:106BA000CC0D00200000C8420000FA440000204143
:106BB000FC0D002000007A44900D002070B5124CAE
:106BC00005460020FFF758FE6570FEF775FC0F4B79
:106BD000A06093F81C0100266660B0420CBF01243F
:106BE0000324FFF799FF0A49234601EB05156A685C
:106BF00031460848FEF710FB074A50600120BDE807
:106C00007040FFF739BE00BFB01C0020D417002031
:106C10002CF1000800440040501D002038B5114BF5
:106C2000187803281BD1104C6068FEF7B4F938B10E
:106C300060682568FEF7B4F901462846FEF79BF91F
:106C40002068094DFEF7A7F90028ECD095E811005F
:106C5000FEF7A6F901462046FEF78DF9E3E74FF06F
:106C6000FF3038BDB01C0020501D0020F7B5036870
:106C7000164C174D23600968164E61600068FFF7D7
:106C8000DDFD94E80C0014480196009095E803009F
:106C9000FFF726FE6B68114A61683668C81A1660ED
:106CA000F9F734FF0E4A0F4F1168F9F783FFFAF72F
:106CB00047F92968786020680B4A431A0B483B6003
:106CC000B0F8C4100A4B16601980FEBDE80D002014
:106CD000CC1B0020480E0020540E0020E40D0020A4
:106CE00030000020780E0020580E002008170020E9
:106CF000760E0020264BF0B51D68024600F110010B
:106D000016781446AB195B78013203F00403DBB24A
:106D100063B18A42F4D10020F0BD13B10A2253437B
:106D2000DBB210F8011B30395B18DBB2211A0229E3
:106D3000F3DC0021844209D911B10A225143C9B2BE
:106D400010F8012B303A8918C9B2F3E72E2E11D171
:106D50000134042000220A2672432678AF197F7876
:106D600007F00407FFB217B1303A92190134013825
:106D7000F1D100E00022074C6420614300FB0211C6
:106D800006240548B1FBF4F200FB0320F0BD00BF70
:106D90006C01002040420F00809698000000000027
:106DA0002DE9F04F9A4B91B05868C0B9994C2178B1
:106DB0004A1E032A00F20286DFE812F0C605C60565
:106DC000DF05C9056068FEF7EBF89349044691F8C2
:106DD0001C31012B00F0DF8008D3022B06D08C4C35
:106DE0006068FEF7D8F80028ECD1DFE7242C07D143
:106DF0008A4B8B4A8B4C0021197011702170C5E0B1
:106E00002C2C02D02A2C40F08280854D834A297890
:106E1000854B157800205854844AB5B918781570F8
:106E2000472868D15978502965D19878472840F08B
:106E3000B385D978472940F0AF851B79412B40F0C5
:106E4000AB850120107000F0A7BD117801293AD15F
:106E5000022D05D11846FFF74DFF754908604AE03D
:106E6000032D07D11978532945D17148026853423F
:106E7000036040E0042D05D11846FFF73BFF6C4B43
:106E8000586038E0052D07D11B78572B33D168495E
:106E90004A68504248602EE0062D07D119786548AF
:106EA000302994BF00210121C17224E0072D04D1B3
:106EB000FFF758FD604A10701DE0092D1BD1FFF748
:106EC00051FD5E4B16E0022915D1072D0CD1012092
:106ED000FFF748FD41F2184250434FF47A71584B86
:106EE000B0FBF1F0188006E0082D04D10120FFF777
:106EF00039FD544B1880494B4949013500202A2C53
:106F00001D70087039D15048012404703EE00D2CEA
:106F10004D4A01D00A2C26D11478FCB1424C21787C
:106F20006478A1F13000C3B2092B84BFA1F137030B
:106F3000DBB2A4F1300003F00F02C3B21101092B40
:106F400084BFA4F13703DBB2364C03F00F0289187B
:106F50002078CBB2C21A514251EB02043A4B0020C6
:106F600018707CB912E02E490B780E2B03D82E48EE
:106F7000C45401330B70127842B92A4B1A7854402A
:106F80001C7003E0294A1078012800D00020C007B7
:106F900000F1338123E72D4B0022197808293FF6B1
:106FA0001EAFDFE801F00A051119275F7C96A000EB
:106FB000622801D1022105E01A70B52C7FF40FAFD1
:106FC0001C78611C19700AE72149224A03261E70A9
:106FD00008701070204B0BE01E4E0421197032789F
:106FE0001D4BA1181878CAB2101818701B4B3270BC
:106FF0001C70F4E605211970164B174E1A7830787C
:10700000A118CAB210183070154E1A703480E6E616
:10701000501D0020B01C0020D4170020DD0D0020E2
:107020006C0D0020740E0020800D0020400D00200B
:10703000CC1B0020CB1C0020EA1B0020821B002060
:107040008C1B0020FC0700205D0E0020DF0D0020BF
:107050005C0E0020DC0D0020E00D0020410D002022
:107060007E0D00206C4906261E700A786B4BA61810
:107070001878F2B210181870694B0A70198801EB71
:107080000424A6B2B6F5007F01D81E8003E00022DA
:107090001A80644B1A700024634B00F052BC5E49A6
:1070A0005E4E0A783078A318DAB2101830705E4E4F
:1070B0000A7033885A4AC72B98BF5C49108898BF1A
:1070C000CC545C1CA1B2884231807FF488AE072189
:1070D00007E0514A08261E70137883423FF47FAEC2
:1070E0000021504B6EE74D4E1A70337883427FF487
:1070F00076AE4F4C207806283BD005D8022813D016
:1071000003287FF46CAE23E0122847D030287FF4A8
:1071100066AE464A474C1679444A102E88BF102660
:1071200026702178002347E0404C434E6368A068F6
:1071300021697360414B4FF47A723060404C91FB8F
:10714000F2F618783F492680C87201223E4923E0B2
:1071500036494A7912F0010004D00E79F41E6342D8
:1071600053EB040035490870002839D1354AD072F4
:1071700036E02E4EF47A14F0010104D0B07AC21E2B
:10718000534253EB02012D4E317009B92D4CE1727F
:1071900026482E4990F82F200A7021E023482C49D8
:1071A0008669426942F210742A4B96FBF4F00A8019
:1071B000188001222849EFE70C328B4210DA12F8CE
:1071C000046C264812F8034C1E54254E25489C5545
:1071D00012F8014C16781C54234C1E550133EBE772
:1071E00019490A78002A3FF4FAAD1B4B1E78002E8D
:1071F0003FF4F5AD00240C701C701C4CA068E060DE
:10720000FEF75AF9A060202000F0A2FC18490A7885
:10721000012A2FD100232EE0DC0D0020E00D0020FC
:107220007E0D0020DF0D0020C80D0020840E002000
:10723000410D0020EB1B0020CC1B0020680E00201D
:10724000821B0020CB1C0020DE0D0020EA1B00204A
:107250008C1B0020FC0700205E0E0020701B00200D
:10726000BA1B0020D41B0020F41B0020B01C0020FF
:10727000AE07002001237E4C0B70E07A00283FF41B
:10728000AEAD7C490A78042A7FF6A9AD677807B9C4
:107290002773257B15B90FB1FFF7ECFB764E05215F
:1072A0003378764F5C1C94FBF1F001FB1042327096
:1072B000734E97F800C0734D06EB82020023724CA8
:1072C00072491F59DFF810E27148724E5F5097FB08
:1072D000FEF1195006FB0170DFF8009203EB040A7F
:1072E00042F2107490FBF4F71668BCB253F80970C0
:1072F0001060C6EB07084044052643F8090090FBE0
:10730000F6F00EFB01016448BCF1010F25F8024FB5
:10731000195005D1023CB4F5797F98BFCAF8001026
:1073200004331432082BCAD1FEF7C6F85B4D5C4C0F
:107330002A68801AF9F7E6FB5A49F9F7EFFC206052
:10734000FEF7BAF8286025684FF07E512846F9F715
:10735000CFFD08B94FF07E5525600CA90DAC4A4809
:10736000514B0194009103C80CCBFFF7B9FA0C9A6A
:1073700064234E49B2FBF3F008800D9A3C4892FB1F
:10738000F3F34B4C027B23800AB90A8022804949DF
:107390000C78002C36D0424F4FF07E503968F9F708
:1073A000BDFC454D384E2B6804463068C01AF9F7CD
:1073B000ADFB2146F9F7FEFBF9F7C2FD726869687B
:1073C0003E4D0746501AF9F7A1FB2968F9F7F2FB81
:1073D0002146F9F7EFFBF9F7B3FD04B2384802256F
:1073E000B0F902303FB2E21892FBF5F1B0F900209B
:1073F0008BB2B918334C91FBF5F291B263802180C6
:10740000438001802B4B01201F4C1870184B616882
:10741000294A20681C7A516010601CB9DA79002A68
:107420003FF4DDAC284E294D294C01960095164FAE
:1074300094E80C00FFF754FA61687868254E081A42
:10744000F9F764FB1D4B1968F9F7B4FBF9F778FD00
:1074500070600A48226890F900303C68012BC4EB48
:10746000020131603CD0022B7FF4B9ACF2E000BFE6
:10747000CB1C0020EA1B0020800E00208D0700207E
:10748000180D0020F40D0020CC1B0020600E002001
:10749000100E0020806967FF740D0020F00D0020A1
:1074A0000C0E002000007A44B01B0020AE1B002010
:1074B000B81B0020F40D00206C0E002030000020CE
:1074C0006E0D0020180E0020480E0020540E0020E3
:1074D000E80D0020780E0020809698004C0E0020C9
:1074E000002634463546DFF874B28B4F5BF82580B2
:1074F000DFF864924046F9F709FB3968F9F75AFB5F
:10750000F9F71EFD34F80910844B421A90B2E0528C
:1075100007B2CDF80890DFF8489238460397F9F79C
:10752000F5FAD9F80010F9F745FBF9F709FD81B232
:107530007B48142202FB0507DFF800A2039B089199
:1075400003EB0800DAF800104B463A46FFF7A0F9C3
:107550000899DFF810820A185BF82500DAF800B005
:1075600024F8082008905846F8F760FFD7F808A0DC
:10757000CDE904015046F8F759FF6A4BCDE9060101
:1075800093F8C000F9F7BEFAF8F750FF60A3D3E90B
:107590000023F8F79FFF02460B4600206249F9F7E7
:1075A000C3F8DDE90423F8F7E3FD0B460246DDE905
:1075B0000401F9F7B9F8089ACDE9040179680135B1
:1075C000501AF9F7A3FA5946F9F7A8FB5146F9F70B
:1075D000E7F9F8F72BFF02460B46DDE90401F8F75F
:1075E00079FF0B460246DDE90601F8F7C1FDF9F720
:1075F00083F9089938617960B860D9F80810F9F70B
:10760000D9FAF9F79DFC49494FF4FA62FBF7A2FC5D
:10761000DDF808C034F8081034F80C20313293B289
:10762000622B98BF0020401882B224F8082010B2C4
:107630003F4940F6B832FBF78DFC394B28F804007F
:1076400099593C48023431501436022D7FF44BAF27
:10765000FFF7C5BB2F68334D374CB5F9C6807E08A0
:10766000B04528BFB04625881FFA88F80FFA88F27F
:1076700029B28A420BDD314831490068F9F79AFA9C
:10768000F9F75EFC43191FFA83F8A4F800802D4E29
:107690002D4D34682A68A61A3046FFF7BDF8002839
:1076A000D8BF404241F293118842CCBF0020012054
:1076B000002859D03046F9F729FA2449F9F77AFA1F
:1076C00004F0FAF805463846F9F71CFA0146284650
:1076D000F9F770FAF9F734FC1D4B1549188040F69C
:1076E000B83200B2FBF736FC201848F6A044A0429E
:1076F00003DDA0F50C40A03804E00028BCBF00F575
:107700000C40A030134A106030E000BFAFF300809F
:10771000182D4454FB211940CC0D0020440E0020AC
:10772000440D0020081700200000F03F30F8FFFF54
:1077300048F4FFFF1C0E0020760E00200C0E0020E7
:107740000000C842480E0020580E0020D3023739EE
:107750007C0D0020E40D0020180E0020780E002083
:10776000FC0D0020881B0020994F3C60984E00259E
:1077700031682C46C1F50C502830F9F7C7F9954906
:10778000F9F718FA074604F023F80F90384604F08A
:1077900093F82F460E900FFA88F0F9F7B7F90EAB71
:1077A00053F82710F9F706FA06468B48DFF86CA263
:1077B000005FF9F7ABF901463046F9F7F1F8F9F750
:1077C000BFFB864924F80A004FF47A7200B2FBF737
:1077D000C1FB82B211B2DFF8489224F80A200846B1
:1077E0000391F9F793F9D9F80010F9F7E3F9F9F7EC
:1077F000A7FB83B27A48142606FB0706DFF824B2FB
:10780000039ADBF80010069310464B463246FFF70A
:107810003FF8DBF800C034F90A1009906046D6F84A
:1078200008A00891CDF808C0F8F700FECDE90401E2
:107830005046F8F7FBFDDFF8F0B1CDE90A019BF8FF
:10784000C000F9F75FF9F8F7F1FD5FA3D3E9002372
:10785000F8F740FE02460B4600206249F8F764FF45
:10786000DDE90423F8F784FC02460B46DDE9040158
:10787000F8F75AFF089BCDE9040170680137181A20
:10788000F9F744F9DDF808C06146F9F747FA5146BF
:10789000F9F786F8F8F7CAFD02460B46DDE9040160
:1078A000F8F718FE02460B46DDE90A01F8F760FC1E
:1078B000F9F722F8089A099B72603061B060069E61
:1078C000D9F80810F618F9F775F9F9F739FB3018F7
:1078D000454E81B2A15308B240F6B8324349FBF796
:1078E00039FB3F4A3053424BA8580234E850143514
:1078F000022F58467FF44FAF90F8C21031B1344A8E
:10790000642413683B4A93FBF4F111803A4BB0F8BE
:10791000BE001C6884420ED9384939480A68036899
:1079200042F21074D01AFEF777FF0028B8BF404229
:10793000A0427FF754AA3348334A012104882D4BD3
:1079400011701C80FFF74BBAFFF72EF836E0626823
:107950006078531C411CCAB263600523B2FBF3F08C
:1079600003FB10216170FDF7A7FD284AA06028489D
:107970000023C372137001200BE0FDF79DFDA36887
:1079800040F6C411C01A884218D9202000F0E8F847
:107990000420FEF771FF11E01E498A78522A7FF415
:1079A000AAAACB784D2B7FF4A6AA087943287FF4A6
:1079B000A2AA194A02211170FFF79DBA11B0BDE8C1
:1079C000F08F00BFAFF30080182D4454FB21194005
:1079D000E40D0020D3023739180E002018FCFFFFF9
:1079E0001C0E00200000F03F881B002048F4FFFF21
:1079F000440D0020341C0020540E0020480E0020AE
:107A0000580E0020E20D00208D070020EA1B002008
:107A1000CB1C0020800D0020400D0020440E0020D3
:107A2000900D00200C0E002008170020AFF30080FE
:107A30003B4B2DE9F047B3F90000F9F767F83949F6
:107A4000F9F7B8F8044603F037FF0646204603F07E
:107A5000BFFEDFF8E490054699F8C180324FB8F1D7
:107A6000000F29D0314CB7F90200B4F802A00FFA88
:107A70008AF1401AFEF7D0FEC8F100014246FBF73A
:107A800069FAB4F80080B7F900700FFA88F300EBD8
:107A90000A02F81A6280FEF7BFFE99F8C12051422F
:107AA000FBF758FA404487B22780B4F90200F9F78F
:107AB0002DF8804638B206E0B7F90200F9F726F84B
:107AC0008046B7F90000F9F721F8294607464046F5
:107AD000F9F770F8314681463846F9F76BF80146F8
:107AE0004846F8F75DFF1249F9F718F9F9F728FA4F
:107AF000104C314620804046F9F75CF8294606468E
:107B00003846F9F757F801463046F8F74BFF084971
:107B1000F9F704F9F9F714FA6080BDE8F08700BFBF
:107B2000361C002035FA8E3C881B0020841B002068
:107B300000002041E007002008170020034B1968CF
:107B400008420CBF00200120704700BF4C0F0020EE
:107B5000024B1A6810431860704700BF4C0F00209A
:107B6000024B1A6822EA0000186070474C0F002090
:107B7000014B1868704700BF4C0F0020024B5A7829
:107B80000AB1002058707047CB1C0020037A032BE9
:107B90000FD8DFE803F00202060A0649064A00F0A1
:107BA000D5BA0449044A00F03BB90249024A00F040
:107BB000FDB97047F21C0020940F002010B500237F
:107BC00004466189094A99520233242BF9D10820CD
:107BD000FBF714F820B12046BDE81040FFF7D6BFF0
:107BE00003480449BDE8104000F0D8B80C1D00203F
:107BF000F21C0020940F00202DE9F84307460820CE
:107C00008846FAF7FBFF70B10024224A4146136808
:107C10003846E2B29847204921F814000134082C74
:107C2000F3D1BDE8F8831D4A1D4D1378591CCCB221
:107C300004F00306147005EB460904460646154891
:107C40004146036832463846984729F824002A8876
:107C50006988AB885018EA88C118881803B2991C43
:107C6000042291FBF2F00C4A0E4BA15EE052CB1EB7
:107C7000984201DA811CA152135FD91C884201DDB0
:107C8000023810530136F6B202340835082ED6D128
:107C9000BDE8F883940F00200C1D0020500F002039
:107CA000520F0020980F002010B544780078002370
:107CB00003FB03F11939614301F6C41159434143F0
:107CC00040F6C41291FBF2F1034A22F8131001337B
:107CD000072BEDD110BD00BF301D00202DE9F04F66
:107CE00085784FF00A0C0CFB05FCC778C5F16408D9
:107CF0006E425FFA88F8C7F16409B6B2002330B269
:107D0000002804DCB8BF2C4602DB012400E0444616
:107D100000FB00FB64430BFB07FB9BFBF4F44C44B0
:107D200044434FF00A0B94FBFBF00CEB000420B231
:107D3000C1EB020A00FB0AF44FF47A7094FBF0F4F2
:107D400004480C191C5202335E44182BB6B2D6D12B
:107D5000BDE8F08FF41C0020F8B505460F46441E20
:107D600014F8011F49B1054E304605F08DFE00287C
:107D7000F6D0861B631BBB55F2E7F8BD7CF100080B
:107D800010B50446805CF9F7E9FFA0F2EE2291B24B
:107D900040F2DC53994288BF608910BD024B0B60F2
:107DA00008210170704700BF817D0008825C044B90
:107DB00053F82200410801F5777290B2704700BF76
:107DC000B40F002038B50446FDF75CFB104B40F6BD
:107DD000C4111A68821A8A421A460E4B01D9002130
:107DE00019701B7810600BB90F2C10D10A480021B4
:107DF0000170084A4BB1094D182B1D4405F8014C80
:107E000003D101230370117038BD0133137038BDE5
:107E1000AC0F0020A80F0020B00F0020D40F0020CE
:107E2000408938B50D4B0D46A0F5777114464A00D0
:107E30001A605A609A60DA601A615A619A61DA616E
:107E400007490848084A0523FDF7E6F90749C860CD
:107E50000CB10748206008222A7038BDB40F0020FA
:107E6000C57D000800440040A0860100501D002090
:107E7000AD7D0008274970B50878002849D0264B09
:107E8000987DC0F3C000002841D1244A10805D785D
:107E90001C78234A05F0070644EA062414609C78FF
:107EA00004F03F06760146EAD5055560DE78B50058
:107EB00045EA94151C7904F0010645EA862595608B
:107EC0005D7905F00F06F60146EA5404D4609C790A
:107ED00004F07F06360146EA15151561DE79750056
:107EE00045EAD4141D7A05F0030644EA4624546199
:107EF0005C7A04F01F06B60146EA950595619B7A07
:107F00000870DB0043EA5414D461012070BD0020E6
:107F1000087070BDB00F0020D40F00206A07002049
:107F2000B40F0020825C034B53F82200C0F3CF0053
:107F3000704700BF0C10002010B50446FDF7A2FAF0
:107F4000154B1A68811AB1F57A6F1A46134B01D98D
:107F5000002119701060187820B9A82C1AD1104B84
:107F6000187006E0022802D10E4A147001E01428AD
:107F700001D80D490C540B490130C3B20878074AA7
:107F80004100481D8342137004D10023044913703B
:107F900001220A7010BD00BF041000202C10002028
:107FA0000810002009100020ED0F002038B5084807
:107FB00001230D46144607494FF4E132FDF72CF931
:107FC000054BD8600CB1054820600821297038BDE8
:107FD00000440040397F0008501D0020257F000824
:107FE000134A10B513780BB9002010BD11490020B9
:107FF00010704A78012AF7D10F4B18800F4801788A
:10800000082901D90822027001780D4A0023D8B24C
:10801000023288420AD212F8010C12F8024C40EAED
:108020000424084840F823400133F0E7012010BD44
:1080300008100020ED0F00206A0700200910002022
:10804000F00F00200C100020124B012210B51A7006
:108050000446FDF717FA104A0146106811600B1A22
:108060000E4841F288318B4203600D4B01D900224A
:108070001A7018780B49E4B20F280C5406D10A493B
:108080000A4B0120002208701A8010BD044A431CCC
:10809000137010BD35100020301000203810002063
:1080A000361000203E1D0020341000206A070020FA
:1080B0001F4B2DE9F0431B7823B31E4C1E4D277830
:1080C00091F800C095F8008002231C4C03F10109CF
:1080D000E65C46FA07F606F00F05EEB266450BD2EF
:1080E0000B2E09D8E65C14F8094006EA080604EBF2
:1080F0000626134C44F825600233102BE5D10C4BB7
:1081000000241C700978914202D90E4B197811B9DC
:108110004089BDE8F0830C4B825C1978084B53F81A
:10812000220001B1400800F5777188B2BDE8F08304
:10813000341000202D1000203C1000203E1D002097
:1081400040100020351000202E10002010B5037ABA
:1081500014465BB1012B13D1104A03201070104A52
:10816000072010700F4803700C2308E00B4A022010
:1081700010700B4A032010700A48037007230B701D
:1081800009490A484FF4E1320123FDF745F808494F
:10819000C8600CB1074A226010BD00BF2D1000203E
:1081A0003C1000202E1000204980000800440040B0
:1081B000501D0020B1800008014B1878704700BFA7
:1081C0003410002008B54FF40060FAF717FD08B925
:1081D000002008BD4020FAF711FD094B20B993F8A3
:1081E0002D21501E0128F3D993F82C01012805D127
:1081F000034991F82D31002BEAD008BD012008BDBC
:10820000D4170020084B93F82D215AB993F82E016A
:1082100010B9064A537801E005490B7D181C18BFB8
:108220000120704701207047D4170020CB1C00208C
:10823000DC1C002010B5084B93F82C211C460AB911
:1082400000F0ACF894F82C01012803D1BDE81040EF
:1082500000F062BA10BD00BFD417002038B50E4B35
:108260001878C0B1FFF7CEFF0C4904460A78824265
:1082700011D060B10A4D95F82C310BB900F098F887
:1082800095F82C01012804D100F03EFA01E0FFF737
:10829000D1FF02490C7038BD711000207010002011
:1082A000D417002038B504464020FAF7A7FC0B4D40
:1082B00008B985F82D01FFF785FF094B187095F86F
:1082C0002D01012801D1074803E002280CBF064810
:1082D0002068A060BDE83840FFF7C0BFD417002079
:1082E0007110002070110020B81300200B4B10B546
:1082F000187888B1FFF786FF70B1094991F82C21F1
:108300000C460AB900F06CF894F82C31012B03D11B
:10831000BDE8104000F008BA10BD00BF7110002089
:10832000D417002038B5064C05465E21A068FCF73E
:1083300022FEA0682946BDE83840FCF71CBE00BFFD
:10834000501D0020024B5E219868FCF714BE00BF50
:10835000501D002010B50A4C5E280146A06805D1CA
:108360005D21FCF708FEA0683E2105E05D2903D1F0
:10837000FCF701FEA0683D21BDE81040FCF7FBBD05
:10838000501D002010B50446C0B2FFF7E3FFC4F350
:108390000720BDE81040FFF7DDBF0000034B93F856
:1083A0002D0108B900F092BA704700BFD417002021
:1083B000044B93F82D0118B94FF4165000F078BA19
:1083C000704700BFD417002008B5044B9868FCF72D
:1083D000E2FDD0F1010038BF002008BD501D002093
:1083E0002DE9F041FFF7F0FF002800F04081FDF794
:1083F00063F8A04B1A68811A7C2940F23881186012
:108400009D480478651C0570002404F12406F0B230
:10841000FFF788FF994B33F91400F8F777FB984A78
:1084200005461088F8F772FB01462846F8F776FCF7
:108430009449F8F7BFFBF8F783FD013400B2FFF76A
:10844000A1FF032CE1D13020FFF76CFF8E49B1F979
:108450000000FFF797FFFFF775FF8748067816F0D3
:10846000030629D1894D1020FFF75CFF2B68642497
:1084700093FBF4F210B2FFF785FF2120FFF752FFC4
:10848000296891FBF4F004FB101484EAE473A3EB75
:10849000E47318B2FFF776FF1420FFF743FF7C4A1E
:1084A000B2F90000FFF76EFF1C20FFF73BFF3046DC
:1084B000FFF768FFFFF746FF6F490878430740F072
:1084C000B080744D0220FFF72DFFB5F900300A256A
:1084D00093FBF5F0FFF756FF0220FAF78FFB002819
:1084E00047D06D4F6D4E3878347840F63401B4FB88
:1084F000F0F26B4C4A4321882A2391FBF0F800FBF1
:108500001810B2FBF3F24FEA001399B241EA022CC1
:108510001FFA8CFEC2F303224EEA02080620FFF780
:1085200001FF0FFA88F0FFF72DFF20883F78431CEA
:108530009AB292FBF7F107FB1120367820806E2467
:108540007443152394FBF3F43A206427FFF7EAFE03
:10855000B4FBF7F63046FFF715FF3B20FFF7E2FECE
:1085600007FB164291B24C1D94FBF5F000B2FFF7E9
:1085700009FF2020FFF7E2FA002850D0494C1320D1
:10858000FFF7D0FE2568484F002DB8BF6D4295FB20
:10859000F7F630B2FFF7F6FE1B20FFF7C3FE2368A5
:1085A0000A26002BB8BF5B4293FBF6F142F210752E
:1085B00091FBF5F205FB121000B2FFF7E3FE23205A
:1085C000FFF7B0FE2368002BACBF4E205320FFF70F
:1085D000D9FE1220FFF7A6FE61680029B8BF494204
:1085E00091FBF7F210B2FFF7CDFE1A20FFF79AFECB
:1085F00060680028B8BF404290FBF6F696FBF5F3A2
:1086000005FB136108B2FFF7BDFE2220FFF78AFECB
:108610006268002AACBF45205720FFF7B3FEFFF782
:1086200091FE15480378282B21D100240470FCF713
:1086300043FF4FF47A753C24B0FBF5F61720FFF7A3
:1086400071FEB6FBF4F5B5FBF4F104FB1152100218
:1086500000B2FFF797FE1820FFF764FE04FB1563D6
:1086600018B2FFF78FFEBDE8F041FFF76BBEBDE823
:10867000F08100BF7410002072100020641C0020E4
:108680001200002000007A44480C0020300C00202A
:10869000361C0020801B00200A000020001700204C
:1086A00078100020CC1B0020A0860100154B2DE97E
:1086B000F04180460F4698680221FCF780FC0024B8
:1086C0002646781E84420F4D0DDA18F80410A8686B
:1086D0008E190134FCF74FFC4FF47A70B6B2FCF7F8
:1086E000F1FEE4B2EDE7F1B2A868FCF744FC4FF408
:1086F0007A70FCF7E7FEA8680121BDE8F041FCF7BD
:108700005EBC00BF501D0020024B01219868FCF7A1
:1087100056BC00BF501D0020024B03219868FCF797
:108720004EBC00BF501D0020F8B5544CA068FCF7AB
:1087300032FC002800F0A080A068FCF731FC054660
:108740000520FCF7CAFE8A2D21D08E2DEDD14C4C90
:1087500000212E22204605F0DBF84A4A7C232370B4
:108760001378E0207D21E07084F82C1014204FF461
:10877000FA71A37723754822782320766076618387
:108780006570628484F8243020462E2171E0202018
:10879000FFF7D4F90028C8D03B4C00212C222046FA
:1087A00005F0B6F8A021E170384B39497C207D22D4
:1087B000207084F82B201878CA7A6570A076002A79
:1087C00052D0344934480F686625FE0F97FBF0FC01
:1087D0006672324E5FFA8CFC06FB0C7284F82950EC
:1087E00006256A4342F21073B2FBF3FE03FB1E2719
:1087F0004968277391FBF0F03F0AC0B26773CF0F4F
:1088000006FB00116943B1FBF3F5642203FB15136A
:10881000E9B202FB0010010AE073214821740188CB
:108820005FFA8EFE63741B0A02FB0CECA374B1FBAF
:10883000F2F224235A4390B21A4A010A1388E071D3
:108840002172180A1849207518480A8801884FEAC9
:108850001C2EE374130A84F80AC084F80BE0A77393
:108860006275A375217702E0202384F82930064839
:108870002C21FFF71BFF58E7F8BD00BF501D00205B
:10888000A6100020001700207A100020EA1B00200C
:10889000CB1C0020CC1B0020A08601006079FEFFCD
:1088A0008C1B0020AE1B0020821B0020B81B002068
:1088B00008B50246032303480021FCF7ADFC024B38
:1088C000186008BD00380140501D0020024B186898
:1088D0000068FFF7EDBF00BFD410002008B5044BBF
:1088E0001860FFF7F3FFBDE8084001F0EFB800BFE4
:1088F000D4100020034B187808B100F0F1BE01F04D
:108900005FB900BFD8100020232801D100F0E8BED5
:10891000044B19688A7A824202D10120FCF75ABEC0
:10892000704700BFD410002070B50646B6FBF2F4C5
:108930000846154614B12046FFF7F6FF05FB146400
:10894000024B195D00F8011B70BD00BF00F3000869
:108950002DE9F041027803460130202AFAD0092A95
:10896000F8D02D2A02D10346414D04E02B2A08BF3E
:1089700003464FF07E551E460024334616F8010B81
:10898000A0F13007F9B209290DD83A492046F8F785
:1089900011F904463846F8F7B9F801462046F8F7C9
:1089A00001F80446E9E72E2817D1324F334616F86E
:1089B000010B3038C2B2092A0FD8F8F7A7F83946A8
:1089C000F8F7ACF901462046F7F7ECFF29490446D1
:1089D0003846F8F7EFF80746E8E71878652801D039
:1089E000452839D15E782D2E02D19F1C012605E045
:1089F0002B2E01D05F1C00E09F1C00267B1E002751
:108A000013F8012F303AD1B2092903D80A2000FB0C
:108A10000727F5E7B7F59A7F28BF4FF49A77B8464E
:108A20004FF07E51B8F1070F07D908461249F8F701
:108A3000C1F8A8F108080146F4E707F0070737B1C5
:108A400008460C49F8F7B6F8013F0146F7E72EB1A2
:108A50002046F8F763F904E04FF07E512046F8F71E
:108A6000A9F801462846F8F7A5F8BDE8F08100BF4F
:108A7000000080BF0000204120BCBE4C10B5441E49
:108A800014F8011F21B1034B1868FCF774FAF7E7DB
:108A900010BD00BF501D00200148FFF7EFBF00BF11
:108AA00025F3000810B50748FFF7E8FF0024064B40
:108AB00006481A19E15852680C34FAF77BFBC02CAF
:108AC000F5D110BD53F3000824F2000869F3000843
:108AD00070B5FCF7F1FC244C244B4FF47A71B0FBD9
:108AE000F1F11A7822482378FAF764FBFFF740F88F
:108AF00005462048204902682048B2FBF1F1FAF708
:108B000059FB00241E4B53F8241051B1012000FAE8
:108B100004F0284202D01B48FAF74CFB0134E4B2BF
:108B2000F0E70220FFF70AF868B1174A174B1178EF
:108B3000174853F82110FAF73DFB1648017C11B194
:108B40001548FAF737FB154C1548FFF797FF2488AF
:108B5000FCF7D0F90246134821464FF46673BDE88E
:108B60007040FAF727BB00BF0A0000200017002062
:108B700071F300085001002040420F00AFF30008DD
:108B800038010108CDF3000822080020E4F20008B3
:108B9000D1F30008041C0020DBF30008E4070020E8
:108BA00090F60008DFF3000838B50C68054620464B
:108BB00005F046F8024628682146BDE8384005F031
:108BC0006FB8000008B50948FFF758FF01210020E1
:108BD000F9F7B0FF0648FFF751FF0A20FCF77DFCCC
:108BE0000020BDE80840FCF7F5BC00BF11F4000808
:108BF0001BF400087FB5044605F022F8082825D1AB
:108C000000231F49E25C086885186E7806F00301AE
:108C1000022908BF203AE2540133082BF1D1002584
:108C2000665D1848314604F02FFF28B10135601900
:108C3000314604F029FF18B11348FFF71FFF1DE06C
:108C4000082DEDD120461149FFF786F81048FFF7AF
:108C500015FF00230F4A04A9981890F808218818D6
:108C6000084A995C0133082B00F80C1CF2D1002053
:108C70008DF80C0001A90848FAF79CFA7FBD00BFE7
:108C80006C0100207CF100082AF40008DC180020A8
:108C90004AF40008D41700206CF3000808B5FDF76B
:108CA000BDFF01300CBF03480348BDE80840FFF793
:108CB000E5BE00BF5FF4000885F400082DE9F0412F
:108CC000054604F0BDFF0446FAF73EF9064694B99E
:108CD0002A48FFF7D3FE2A4951F8241049B101224E
:108CE00002FA04F2324202D02648FAF763FA01345B
:108CF000F1E7254821E028462449224604F0D0FF28
:108D000058B92348FFF7BAFE224C54F8041F002933
:108D1000EFD01C48FAF74EFAF7E72B782D2B04D149
:108D20000135013C4FF0010801E04FF0000800263A
:108D3000134850F8267027B91748BDE8F041FFF7EF
:108D40009DBE28463946224604F0AAFFA0B901205C
:108D500000FA06F0B8F1000F03D0FAF7EDF80F486B
:108D600002E0F9F755FF0E48FFF788FE0D48394637
:108D7000BDE8F041FAF71EBA0136D9E7A3F40008BE
:108D800088F10008CDF3000890F6000842FF0008C3
:108D9000B6F4000884F10008CBF40008E5F40008FC
:108DA000EFF400086CF3000810B504460848FFF71C
:108DB00065FE084A084809490023036013700B70D8
:108DC000FDF7BAF82046BDE81040FFF7FBBE00BF34
:108DD000F8F40008D91000200C110020D810002051
:108DE00008B50848FFF74AFE0120F9F719FF0648C1
:108DF000FFF744FE0A20FCF770FB0020BDE80840A6
:108E0000FCF7E8BB10F500081DF40008F8B50746AC
:108E100004F016FF044638B91A491B4B4A791B481F
:108E2000511E53F8211028E038461949224604F013
:108E300037FF60B91748FFF721FE174C54F8041F9D
:108E400019B11648FAF7B6F9F8E7154805E0002514
:108E50000D4B53F8256026B91248BDE8F840FFF7DE
:108E60000DBE38463146224604F01AFF013500286F
:108E7000EED10448314645710B48BDE8F840FAF799
:108E800099B900BFD4170020C8F100082BF50008DD
:108E900042FF00083FF50008C4F10008CDF30008C8
:108EA00090F6000852F500086AF5000810B504466F
:108EB000204604F0C5FE10F0FF0F07D10B490C4807
:108EC00091F89413BDE81040FAF774B9204604F005
:108ED000D5FB022808D8054B064C83F894030020E4
:108EE0000146F9F727FEE3E710BD00BFD4170020C5
:108EF0007CF50008A0F8000870B5044604F0A0FE58
:108F000008B9204830E020461F4905F011FB002435
:108F10002646254678B12CB1012C06D104F0AEFBD3
:108F2000064602E004F0AAFB05460020164901347B
:108F300005F0FEFAEEE70B2D05D914480C21BDE82B
:108F40007040FAF737B9012C08DC114A114832F9A0
:108F500015202946BDE87040FAF72CB9A6F57A73BA
:108F6000B3F57A7F04D90C48BDE87040FAF722B90E
:108F70000A4829463246FAF71DF9054820F81560D7
:108F800070BD00BF92F500086AF80008CCF5000833
:108F9000941C0020F2F500080AF600082CF60008E0
:108FA00038B5054604F04CFEC0B268B90446124913
:108FB000124801EB4402B2F8422021460134FAF78C
:108FC000F9F8152CF3D138BD284604F057FB1428C6
:108FD00004460BDC2021284604F056FD04F04EFB2D
:108FE000054B03EB4404A4F8420038BD04481521A6
:108FF000BDE83840FAF7DEB80817002045F600084B
:1090000051F60008931E222B88BF0A22031E10B5BA
:109010000C4603DA2D2001F8010B5842FFF784FCBF
:1090200000210170204610BD30B587B005460C46C2
:1090300003A800210C2204F06BFC28460021F7F75E
:1090400075FF20B128462949F7F7ACFC03E0284614
:109050002649F7F7A5FC2649F7F7ACFDF7F770FFAF
:10906000054685EAE570A0EBE5700A226946FFF740
:10907000C9FF002D01DB202300E02D2368468DF879
:109080000C3004F0DDFD012807D130228DF80D20D1
:109090008DF80E208DF80F200CE0022805D130212C
:1090A0008DF80D108DF80E1004E0032802D1302049
:1090B0008DF80D00694603A804F0C0FC03A804F075
:1090C000BFFDC51EEDB22A4603A9204604F056FE98
:1090D000002363552046074904F0B0FC03A920464D
:1090E000491904F0ABFC204607B030BD6F12033ABB
:1090F00000007A4428F4000837B5037904460D4689
:10910000052B34D8DFE803F003060A0D111481683B
:1091100009782DE0806890F9001029E083681988AB
:1091200026E08268B2F9001022E0816809681FE039
:10913000806869460068FFF777FF01461148FAF733
:1091400039F8F5B1E068F7F7E1FC6946FFF76CFF25
:1091500001460D48FAF72EF82069F7F7D7FC694663
:10916000FFF762FF01460848FAF724F809E00021FA
:109170000648FAF71FF825B10548E1682269FAF7B1
:1091800019F83EBDD8F30008D7F300087BF60008B5
:1091900077F600082DE9F047064604F051FD054634
:1091A00020B1012819D133782A2B16D14748FFF76F
:1091B00065FC002414266643454F4648F159F9F7EB
:1091C000F9FFB8192946FFF797FF01344248FFF726
:1091D00055FC6E2CEED1BDE8F08730463D2104F001
:1091E00053FC002857D0441C204604F047FA82461E
:1091F0002046FFF7ADFB0027054614247C43DFF82B
:10920000D09054F80980404604F01AFD41460246C9
:10921000304604F045FD002835D14C44E068F7F7AE
:1092200075FC01462846F7F777FE002829D020690B
:10923000F7F76CFC01462846F7F764FE002820D0BB
:1092400020792279052818BF5546052A0FD8DFE86E
:1092500002F003030606090CA1680D7007E0A2687E
:10926000158004E0A068056001E0A1680D6041463A
:109270001A48F9F79FFF20460021BDE8F047FFF7A5
:109280003BBF174803E001376E2FB6D11548BDE844
:10929000F047FFF7F3BB0446142565430C4F3146F6
:1092A00055F80780404604F0CDFF50B109484146CB
:1092B000F9F780FF78190021FFF71EFF0648F9F73C
:1092C00079FF01346E2CE7D1BDE8F0877EF6000807
:1092D000580101085DF7000890F6000893F60008B1
:1092E0009EF60008C3F600082DE9F043584885B003
:1092F000584CF9F75FFF5848FFF752FE6279574B19
:10930000511E574853F82110F9F754FF20690021E6
:10931000F7F7E4FD002858D10025266900213046E2
:10932000F7F7DCFD00284CD101354E482946D4F82A
:109330001490D4F81880E769F9F73CFF3046002113
:10934000F7F7D6FD10B14848F9F734FF69463046C3
:10935000FFF76AFE01464548F9F72CFF4846002111
:10936000F7F7C6FD10B14048F9F724FF69464846B3
:10937000FFF75AFE01463D48F9F71CFF4046002121
:10938000F7F7B6FD10B13848F9F714FF69464046C3
:10939000FFF74AFE01463548F9F70CFF3846002131
:1093A000F7F7A6FD10B13048F9F704FF69463846D3
:1093B000FFF73AFE01462E48F9F7FCFE10340C2D5B
:1093C000ABD12C48691CF9F7F5FEF9F7BDFD2A4C25
:1093D000064654F8041F19B12848F9F7EBFEF8E7E0
:1093E0000D46274850F8251049B1012202FA05F22E
:1093F000324202D02348F9F7DDFE0135F1E7154B83
:10940000214ACE1896F808418B5C04A80131051951
:10941000082905F8103CF2D100241C4869468DF853
:109420000840F9F7C7FE14256543194E1948A95994
:10943000F9F7C0FE00217019FFF75EFE01341648EF
:10944000FFF71CFB6E2CEED105B0BDE8F08300BF2A
:10945000E0F60008D4170020A0F80008C8F10008C2
:1094600010F700081BF700086AF80008D8F3000896
:109470006CF3000823F7000884F1000835F70008B2
:1094800088F1000843F700087CF1000850F7000855
:109490005801010859F7000890F600082DE9F0433B
:1094A00089B0044604F0CCFBC6B2002E6AD17948DC
:1094B000FFF7E4FA784C20690021F7F70FFD38BB7D
:1094C000013676483146F9F775FE206904A9FFF7A1
:1094D000ABFD01467248F9F76DFE606904A9FFF71C
:1094E000A3FD01466E48F9F765FEA06904A9FFF7E0
:1094F0009BFD01466A48F9F75DFEE06904A9FFF7A4
:1095000093FD01466748F9F755FE10340C2ED2D171
:109510000025654C2F46A8464FF000091034B14590
:1095200014DA404654F8101CF7F73CFA54F80C1CB7
:1095300080462846F7F736FA54F8081C05463846A0
:10954000F7F730FA09F101090746E7E75748CDF880
:10955000048002950397FFF791FA002401A823588D
:10956000534923F00040F7F7E1FC5249524A0434D2
:10957000002814BF10460846FFF780FA0C2CEDD1E6
:109580004E4870E020464E49052204F089FB38B968
:10959000414B0022C1181030C0280A61F8D176E092
:1095A00020464849042204F07BFB0546204605BBC3
:1095B000202104F069FA002869D0461C304604F0E6
:1095C0003FFB2C460746404850F824500DB93F4811
:1095D00049E030462946FAB204F062FB38B9204629
:1095E000FCF748FD3A482946F9F7E4FD47E0013425
:1095F000E9E704F043F8461E0B2E074643DC2046FD
:10960000202104F041FA054640B1451C2846FFF7E9
:109610009FF9214B3F01D851012400E00446284620
:10962000202104F031FA054640B1451C2846FFF7D9
:109630008FF91949013401EB0612506128462021A7
:1096400004F022FA054640B1451C2846FFF780F990
:10965000114B013403EB061188612846202104F0E8
:1096600013FA18B91B48FFF709FA10E00130FFF7A9
:109670006FF9094A032C02EB0616F061F2D1164885
:10968000FFF70CFF03E015480C21F9F793FD09B033
:10969000BDE8F0836BF70008D417002096F70008A8
:1096A0009CF700086CF30008E8170020A0F70008FA
:1096B0000AD7233C67F7000863F7000890F6000814
:1096C000AFF70008B5F70008C8F1000852F5000828
:1096D000BAF70008CDF70008A0F8000807F800085E
:1096E000F0B5694B87B01A783AB90120187067480D
:1096F000FFF7C4F96648FFF7C1F9664C2068FBF72D
:109700004AFC002800F0BD802068FBF749FC0928CE
:109710000146614A01D03F2851D1002517685F4CAE
:109720002E462FB15E4821683A4604F0B9FA10B9C6
:10973000254606B926465B490C348C42F1D3C6B1A6
:109740003468D5F800E03B46E05C1EF80310814227
:109750000DD1534A41B92D2B06D820244E48D4545C
:1097600001330360D15404E0D0540133ECE74A499B
:109770000B60494A14681CB1AE4201D13C4612E06C
:109780004948FFF77BF9AE4209D856F80C0BFFF7B2
:1097900075F9404B09211868FBF7EDFBF3E73C48EE
:1097A000FFF76CF900243C4B18688442A5D2394974
:1097B0003B4A0868115DFBF7DEFB0134F3E71368F1
:1097C0002BB9042838D13648FFF7EEFA59E00C28B7
:1097D00001D136488CE70A2901D00D2948D12E4DF8
:1097E0003348FFF74BF92E4C2A6832490023A35423
:1097F0000493009103A8294910220C23039403F039
:1098000041FF054638B1006804F01AFA0130AA6831
:109810002018904702E02848FFF730F90021302255
:109820001F4804F075F818481B4B02780021196096
:10983000002A7FF45FAF24E00C28CAD07F2903D12F
:109840005BE72F2B3FF659AF1F297FF656AF7E29D6
:109850003FF653AF13B920293FF44FAF104C0E48D9
:109860000C4AE154013303601068FBF784FB44E7C2
:109870007F29E6D10A485C1E0021015514600F487B
:1098800039E707B0F0BD00BFD81000202FF800085E
:1098900067F80008501D00200C11002024F2000879
:1098A000D9100020E4F200086CF8000871F80008F4
:1098B00090F60008A98B00087CF800089DF80008C5
:1098C000F8B5174E174C184D0746C1B230682170D5
:1098D000FBF751FB22782B78C7F3072182EA0300BC
:1098E000287030682170FBF746FB21782A783068B1
:1098F00081EA0203C7F307412B702170FBF73BFBA2
:109900002078297880EA0102390E306821702A70A7
:10991000FBF731FB2B78207880EA03012970F8BD32
:10992000501D00202C11002010110020F8B50D4E04
:109930000D4D0E4CC1B2074630682970FBF71BFB7A
:109940002A782378391282EA03002070297030685F
:10995000C9B2FBF710FB23782A7882EA0300207053
:10996000F8BD00BF501D00202B1100201011002059
:10997000054B10B5044621461868FBF7FCFA03486E
:1099800002785440047010BD501D002010110020BA
:10999000034B04491A78885C01321A70704700BF83
:1099A000121100202E11002010B5FFF7F1FF044620
:1099B000FFF7EEFF04EB002080B210BD10B5FFF7FB
:1099C000F3FF0446FFF7F0FF04EB004010BD00007A
:1099D00038B5044624200D46FFF7CAFF4D20FFF797
:1099E000C7FF002C0CBF3E202120FFF7C1FF064B14
:1099F000002228461A70FFF7BBFF04480078BDE834
:109A00003840FFF7B5BF00BF101100202A11002019
:109A100001460020FFF7DCBF01460120FFF7D8BF59
:109A2000014B1878FFF7A4BF1011002070B5054650
:109A300008460E46FFF7ECFF2C467219D0B2E3B28F
:109A4000984204D014F8010BFFF792FFF5E770BDC0
:109A500010B5441E14F8010F10B1FFF789FFF9E7A4
:109A600010BD00002DE9F843002701240025144B08
:109A7000187885421CDA1349134B15F801800C2223
:109A800002FB0830406804F0DBF881460CB13F1857
:109A90000CE026464E4509DA0B4A0C2101FB08234F
:109AA0005868805DFFF764FF0136F3E70135DEE7B4
:109AB00024B1F8B2FFF7ACFF0024D7E7BDE8F88384
:109AC00013110020151100203400002070B5394D0D
:109AD000FF211522284603F01BFF002302202B70D4
:109AE000FEF72CF8012418B102206C70A870032432
:109AF0000420FEF723F868B12E4E03214FF40050E6
:109B00003155651CF9F77AF818B104227255023400
:109B100000E02C460220FEF711F848B1254B052045
:109B20001E190621072518557170B570033404E01D
:109B30000820FEF703F80028F0D12020F9F75EF89E
:109B400018B11C4B08221A5501344FF48070F9F7F4
:109B500055F830B117480A2601190B2506554D70E6
:109B60000234154A134B5079082801D00E2802D12F
:109B70000C261E5501340D2104201955651CF9F7DA
:109B80003DF818B10B4811224255A51C0A49132370
:109B900091F82E21074E6C1C101C18BF0120735524
:109BA000F9F72CF810B114203055AC1C034B1C7085
:109BB00070BD00BF15110020D41700201311002024
:109BC000F8B5B54C2068FBF7E6F9002800F04185B0
:109BD0002068FBF7E5F9B14A0346117871B9B0F195
:109BE00024014B4253EB01041470002CE9D1AC4A20
:109BF00051780029E5D1FEF787FEE2E7012904D17B
:109C00004D280CBF0223002321E0022904D13C2867
:109C10000CBF032300231AE003290FD140284FF083
:109C2000000401D91470CCE79E489F4903709F48F7
:109C30000C7004709E4C2370042308E0042908D1A2
:109C40009B4C9C48217803704B4023700523137074
:109C5000B7E70529B5D19448924C017822788A4219
:109C6000934A07D914785C401470934A53540131D5
:109C70000170A6E71078984240F0E6848D4B197881
:109C80007B2900F0338300F2C5806E2900F07D83CC
:109C900060D8682900F0468325D8652900F0128233
:109CA00019D8642940F0CB840720844CFFF7B0FE1C
:109CB000E620FFF75DFE6079FFF75AFE0020FFF710
:109CC00057FE94F819017E4B7E4A00280CBF1046BF
:109CD000184600F067BC662900F07282672940F0E0
:109CE000AE8479481FE36B2900F02D8323D86929BE
:109CF00000F01D836A2940F0A2841020FFF788FE3F
:109D00006748724CC07AFFF733FE71490878FFF755
:109D10002FFE2068FFF7D4FD6068FFF7D1FD6D4A84
:109D2000B2F90000FFF702FE6B4BB3F90000FFF73A
:109D3000FDFD6A4A26E36C2900F017836D2940F087
:109D40007E840620FFF764FE65490868FFF7B8FDCA
:109D5000644A17E3732900F085833CD8702900F02A
:109D60004383C0F02383712900F05183722940F0AE
:109D70006684524C1620FFF74BFE0020FFF7D6FDFD
:109D8000B4F9D000FFF7D2FD574DB4F9D200FFF778
:109D9000CDFDB4F9D400FFF7C9FDB5F9B600FFF762
:109DA000C5FD0020FFF7C2FD0020FFF789FDB5F9D2
:109DB00028000A2390FBF3F0FFF7B8FD94F80401A4
:109DC000FFF7D6FD94F80601FFF7D2FD94F80501E0
:109DD000FFF7CEFD75E3762900F04F830DD8742987
:109DE00000F02D83752940F02A842F20FFF710FE04
:109DF0003E48FFF72DFE00F025BC772900F02283B6
:109E0000782940F01C84384C3820FFF701FE04F11B
:109E1000400539E2D02900F0898300F2CA80CA29BE
:109E200000F00F816CD8A42900F0E88310D8A02995
:109E300040F005840C20FFF7EBFD2D492D4C086800
:109E4000FFF73EFD2C4A1068FFF73AFD2068A9E3B2
:109E5000C82900F0ED80C92940F0F183FFF798FD93
:109E60000F4B1A4CD872FFF793FD19490870FFF792
:109E7000A5FD2060FFF7A2FD6060FFF795FD154A84
:109E80001080FFF791FD144B18801C48017841F0B9
:109E900002040470E4E000BF501D002011110020F6
:109EA000CB1C0020141100202D11002012110020C5
:109EB000101100202A1100202E110020D41700209C
:109EC0001C0000801400008020000020CC1B00201B
:109ED000EA1B0020821B00208C1B0020FC070020B6
:109EE0005C1C0020480C002008170020F009010825
:109EF000E8F7FF1FF0F7FF1FECF7FF1FAE0700208A
:109F0000CD2900F01C8322D8CB2900F0AB80CC29CE
:109F100040F09583FFF73CFDC84CE077FFF738FD34
:109F200084F82000FFF734FD84F82300FFF730FDAC
:109F300084F82400FFF72CFD84F82500FFF728FDA6
:109F400084F82100FFF724FD84F8220088E0CE2960
:109F500000F0FF82CF2940F07283FFF725FDFFF765
:109F600023FDB74CB54DA4F8D000FFF71DFDA4F8B4
:109F7000D200FFF719FDA4F8D400FFF715FDA5F8EE
:109F8000B600FFF711FDFFF719FDFFF70DFD0A23DE
:109F900058432885FFF7FCFC84F80401FFF7F8FC20
:109FA00084F80601FFF7F4FC84F80501FFF7F0FCE4
:109FB00056E0D52900F0A8810FD8D2296BD0C0F087
:109FC0008482D32979D0D42940F039839B4C002056
:109FD000FFF71EFD04F140056AE1F02900F0D5828B
:109FE0000CD8D6294ED0EF2940F02983FFF7DCFCAE
:109FF000924CA085FFF7D8FC608531E0FA2900F08B
:10A00000B082FE2940F01B830820FFF701FD8D4C34
:10A010008D488E4B01682068B1FBF3F2B0FBF3F37F
:10A020004FF47A7101FB0234894AD4800024A4E2FF
:10A030000024FFF7B9FC874A10530234102CF8D1E2
:10A040000EE0854C04F10A05FFF7A2FC01346070B4
:10A05000FFF79EFCE072FFF79BFCAC426075F3D10A
:10A06000002087E200247D4801788C42F8D27C4DA4
:10A07000655DFFF799FC714A013402EB4505A5F8CF
:10A080004200F0E70024FFF78FFC764A10530234B9
:10A09000102CF8D1E4E7744C6478002CE0D1FFF781
:10A0A00077FC6749022881F8940388BF81F89443BC
:10A0B00000200146F8F73EFDD2E7FFF775FC6B493B
:10A0C0000880CDE76A4D0B20FFF7A2FCB5F9000030
:10A0D000FFF72CFCFAF70EFF00B2FFF727FC022077
:10A0E000FDF72CFD05460420FDF728FD0446082059
:10A0F000FDF724FD820042EA4401294320208CB26E
:10A10000FDF71CFD44EAC00084B21020FDF716FDE7
:10A1100044EA001318B2FFF709FC534A1079D178CA
:10A1200084005378907944EA4101194341EAC0041C
:10A130005179537A44EA411040EA83144D48C17979
:10A1400044EAC113047A417A43EA042343EA4124EE
:10A15000D379117A44EA8324927A44EAC123417B79
:10A1600043EA0234827B44EA4133017C43EA82348D
:10A17000027944EA0143417C43EA0214827C44EAC6
:10A180004143C17C43EA8244007D44EAC142334BEF
:10A1900042EA00540020197803468B420AD2304D1F
:10A1A00001225D5D02FA05F525421CBF9A4010436D
:10A1B0000133F2E7224CFFF783FB94F8940381E12B
:10A1C0001220FFF725FC2C490C88B4F5806F2B4C2E
:10A1D000B4F9000008D8FFF7A9FBB4F90200FFF7B3
:10A1E000A5FBB4F904000EE0082590FBF5F0FFF79D
:10A1F0009DFBB4F9020090FBF5F0FFF797FBB4F973
:10A20000043093FBF5F01E4CFFF790FBB4F900000F
:10A21000FFF78CFBB4F90200FFF788FBB4F90400E8
:10A22000184CFFF783FBB4F90000FFF77FFBB4F98C
:10A230000200FFF77BFBB4F90400B0E1081700202F
:10A24000D4170020500100204C01002040420F0094
:10A25000981B00200C1D0020071700201311002060
:10A2600015110020941C0020CB1C0020341C002061
:10A27000E4070020DC1C002012000020641C0020E9
:10A280001C0C0020181C0020B4F97400FFF74EFBD2
:10A29000B4F97600FFF74AFBB4F97800FFF746FB04
:10A2A00094F87A000834FFF763FBAC42ECD1C9E1C3
:10A2B000FFF77AFBA4F87400FFF776FBA4F87600AA
:10A2C000FFF772FBA0F57A72072893B298BF84F863
:10A2D0007B00B3F57A7F98BFA4F87800FFF758FBAE
:10A2E00084F87A000834AC42E2D1ABE10820FFF7F1
:10A2F0008FFB0024AD49621892F87B000834FFF709
:10A3000037FB402CF6D19DE10020FFF781FB0024B4
:10A31000FFF73EFBA54962180834402C82F87B0009
:10A32000F6D18FE1A2481021FFF780FB8AE11020CF
:10A33000FFF76EFB00249F48005F0234FFF7F6FA38
:10A34000102CF8D17EE10520FFF762FB9A4BB3F9A0
:10A350000000FFF7EBFA9948B0F90000FFF7E6FAC2
:10A3600097490A7802F00100ACE0964C0620FFF70E
:10A370004FFBB4F90000FFF7D9FAB4F90200FFF778
:10A38000D5FA914AB2F9000009E10720FFF740FB36
:10A390008E480078FFF7ECFA0020FFF7C7FA8C4BE5
:10A3A000B3F90000FFF7C2FA0020F8E07F4C072065
:10A3B000FFF72EFBE07FFFF7DBFA94F82000FFF7B2
:10A3C000D7FA94F82300FFF7D3FA94F82400FFF7A4
:10A3D000CFFA94F82500FFF7CBFA94F82100FFF7A5
:10A3E000C7FA94F822006DE01E20FFF711FB794CAC
:10A3F00004F10A0501346078FFF7BAFAE07AFFF752
:10A40000B7FA607DFFF7B4FAAC42F3D11AE17249B2
:10A410000A78540004F0FE00FFF7FAFA00246E48B0
:10A4200003789C4280F00E816C496048625C013484
:10A4300000EB4203B3F94200FFF778FAEFE7FFF7CA
:10A4400011FBFFE0644900240878FFF7E1FA624A53
:10A450001078844280F0F680604B185DFFF788FA30
:10A460000134F4E70820FFF7D3FA0124E0B2013405
:10A47000FFF77EFA092CF9D1E4E0FFF789FA0646E6
:10A480001220FFF7C5FA0EB9554902E0102E03D18C
:10A4900054490D684C6801E0002425463046FFF71A
:10A4A00067FA2846FFF70CFA2046FFF709FA4E4AEA
:10A4B0001068FFF705FA0020FFF738FA0020FFF7D1
:10A4C00035FA0020FFF754FABCE0FFF761FA0546C1
:10A4D000FFF774FA0746FFF771FA0646FFF76EFAC0
:10A4E0000446FFF761FAFFF75FFAFFF751FA65B923
:10A4F0003B483E49012207604660CD710A73002C3B
:10A500003FF4AEAD384B1C60AAE5102D7FF4A8AD2A
:10A510003448076046600CB1334A1460344B31480C
:10A5200002211970011DFCF7A1FB99E52F48437822
:10A53000002B7FF495AD0120F8F772FB90E52B4CD2
:10A540006378002B7FF48CAD2A494FF4C8700880E3
:10A5500086E52648417800297FF482AD0122827386
:10A560007EE5224B5C78002C69D120460121F8F76A
:10A57000E1FA2046FFF74CFA64E01F48005F02341E
:10A58000FFF7D4F9082CF8D15CE0084C0420FFF761
:10A590003FFAB4F92C00FFF7C9F9B4F92A00FFF724
:10A5A000C5F94FE0FFF78CF94CE000BF0817002019
:10A5B0007C1C00200C1D0020AE1B0020B81B0020BE
:10A5C000AE0700202C0C0020361C002000170020B5
:10A5D000E81B002007170020131100201511002090
:10A5E000B01B0020901B0020601C0020CB1C002012
:10A5F0008D0700200C080020981B0020154C2378A4
:10A600009800411CC8B2FFF703FA2078FFF7B0F9B1
:10A610000024104A13789C4214D20F48005DFFF7C3
:10A62000A7F90E49085DFFF7A3F90D4A105DFFF782
:10A630009FF90C4B185DFFF79BF90134E9E7002007
:10A64000FFF7EAF9FFF7ECF9074B00201870FFF766
:10A65000B8BAF8BDEB1B0020701B0020BA1B00200D
:10A66000D41B0020F41B0020111100202DE9F04123
:10A670000746884616460024B4420ED00025BD4247
:10A6800005D040460135FAF728FFEDB2F7E73C2048
:10A690000134FAF722FFE4B2EEE7BDE8F0810000F2
:10A6A0000F4B1A6842F00100186059680D4A0A40C1
:10A6B0005A60186820F0847121F480321A6018689A
:10A6C00020F4802119605A684FF41F0122F4FE0023
:10A6D00058609960044B4FF000629A60704700BF69
:10A6E000001002400000FFF800ED00E0164A174B92
:10A6F000516801F00C00042803D0082805D0144844
:10A7000001E014490868186011E051685068C1F30D
:10A7100083410231C00301D40F4A06E052680D485C
:10A7200012F4003F026818BF520851431960064BEB
:10A730000A485A68054BC2F30311415C1A6822FAB1
:10A7400001F21A60704700BF001002405001002063
:10A7500000127A004C01002000093D003C0100205D
:10A760001FB500234F494FF4E0100093019302936B
:10A7700003900A6842F480330B60886940F010024D
:10A780008A61484B196801F400300190009A511C0D
:10A79000009101981A4618B9009BB3F5A06FF0D14B
:10A7A0001168404811F4003201D0022216E003681B
:10A7B00043F00101016000923A48026802F002038E
:10A7C000019300994A1C0092019B1BB90099B1F5B5
:10A7D000A06FF1D1006883073CD50122324B029271
:10A7E000196841F0100018601A6822F0030119601E
:10A7F000186840F002021A60A3F580535968596046
:10A80000586858605A6842F48061284A5960106854
:10A8100020F070411160264826490860586820F4ED
:10A820007C105860106840F000401060906820F480
:10A8300000409060043A9268100449BF1E4A4FF4E9
:10A84000E0120A604FF48012039202991548012920
:10A8500001D10AE0FEE702290BD14268039B42EADC
:10A86000030141F48032426003E0596841F4601210
:10A870005A60036843F0807101600A4802689201DF
:10A88000FBD5436823F003014160426842F00203B4
:10A890004360416801F00C02082AFAD1FFF726FF55
:10A8A00005B000BD0010024000200240041001402D
:10A8B00000127A004C010020001BB70008B5154BB0
:10A8C00098420BD101214FF4805000F0C1FD4FF4AC
:10A8D00080500021BDE8084000F0BABD0E49884212
:10A8E00007D14FF48040012100F0BEFD4FF48040BD
:10A8F00009E00A4A90420BD14FF40040012100F0D8
:10A90000B3FD4FF400400021BDE8084000F0ACBDAD
:10A9100008BD00BF0030014000380040003C00404E
:10A920000B8810B54C88028823438C8802F441526E
:10A930002343CC8823430C8923434C8923438C89AC
:10A940002343CC89098A23431A4393B20380828B21
:10A9500022F400631A04130C8383018210BD038860
:10A9600019B199B241F0400303E023F040010A0419
:10A97000130C0380704781817047808980B27047D3
:10A98000038919420CBF002001207047426810B5AE
:10A9900022F470230A6823F4807444EA02030C79D9
:10A9A00043EA04224260CB688A6884681A43084BF1
:10A9B000234013434A7943EA42038360097CC26A15
:10A9C0004B1E22F47002D9B242EA0152C26210BD9B
:10A9D000FDF7F1FF836811B143F0010101E023F0BD
:10A9E000010181607047836811B143F4807101E017
:10A9F00023F4807181607047836843F008018160AF
:10AA000070478068C0F3C0007047836843F004015A
:10AA1000816070478068C0F380007047836811B11F
:10AA200043F4A00101E023F4A001816070470929EB
:10AA300070B54FF003040CD94C4307251E3C05FAB2
:10AA400004F503FA04F3C66826EA05052B43C36040
:10AA50000BE04C43072505FA04F503FA04F30669F5
:10AA600026EA050545EA03040461062A4FF00503BA
:10AA70000DD8013A53431F2202FA03F201FA03F1FF
:10AA8000446B24EA020242EA0103436370BD0C2ACC
:10AA90000DD853431F22233B02FA03F201FA03F1BC
:10AAA000046B24EA020242EA0103036370BD5343CC
:10AAB0001F22413B02FA03F201FA03F1C46A24EABD
:10AAC00002021143C16270BD40F0BF60024B40F40E
:10AAD0000031D960704700BF00ED00E0C37810B5C9
:10AAE00003B3164CE168CB43C3F302244178C4F1AD
:10AAF000040201FA02F10F2222FA04F284780378A8
:10AB000022400A43110103F16043CAB203F56141D7
:10AB100081F800230078012200F01F03410902FAA6
:10AB200003F007E00078012200F01F03410902FA58
:10AB300003F02031024B43F8210010BD00ED00E08E
:10AB400000E100E030B5048C24F001052C04250C54
:10AB50000584048BA5B225F0F3052A4342EA0313CA
:10AB6000114A048C9042A4B29DB215D002F5006344
:10AB7000984211D0B0F1804F0ED0A3F59832904298
:10AB80000AD002F58063984206D003F580629042B5
:10AB900018BF24F00A0401D124F0020444F0010497
:10ABA00021430583018430BD002C014030B5048C65
:10ABB00024F010052C04250C0584048B058C24F44A
:10ABC00040742405240D44EA022242EA0333144A65
:10ABD000ADB290429BB212D002F5006290420ED00C
:10ABE000B0F1804F0BD0A2F59832904207D002F519
:10ABF0008062904203D002F58062904207D125F036
:10AC0000200242F0100545EA011189B204E025F066
:10AC1000A00545F0100529430383018430BD00BF22
:10AC2000002C0140224A038890429BB212D002F5C8
:10AC3000006290420ED0B0F1804F0BD0A2F5983256
:10AC4000904207D002F58062904203D002F5806204
:10AC5000904203D14A8823F070031343154A90426F
:10AC600008D002F58062904204D023F44073CA8871
:10AC70009BB2134303808B880A8883850C4B028523
:10AC800098420FD003F5006290420BD002F540636A
:10AC9000984207D003F58062904203D002F58063AA
:10ACA000984201D1097A018601228282704700BF51
:10ACB000002C014000100040038C70B523F001020D
:10ACC0001404250C0584068C8388028B9CB222F028
:10ACD00073052B040D881A0C26F0020633042A4350
:10ACE0004E880D891B0C3543ADB22B43134DA84242
:10ACF0000FD005F50065A8420BD005F54065A842C8
:10AD000007D005F58065A84203D005F58065A84207
:10AD10000ED123F008064B898D881E4326F00403CC
:10AD20002B43CE898D8924F440743543ADB22C4336
:10AD3000C988848002838186038470BD002C014011
:10AD4000038C30B523F010021404250C0584038C09
:10AD50008288048B23F0200324F4E6452C040D881C
:10AD6000240C44EA05241D042B0C0D8992B243EAFD
:10AD700005134D88A4B243EA0513124D9BB2A842B5
:10AD800003D005F50065A84215D14D8923F0800355
:10AD90009BB243EA05134FF6BF751D408B8822F422
:10ADA000406245EA0315ABB28D8942EA8502CD893E
:10ADB00042EA850292B2C9888280048301870384B3
:10ADC00030BD00BF002C0140038C30B523F48072ED
:10ADD0001404250C0584038C8288848B23F400736F
:10ADE00024F073052C040D88240C2C431D042B0C1B
:10ADF0000D8992B243EA05234D8843EA0523124D9B
:10AE00009BB2A84203D005F50065A84215D14D8933
:10AE100023F400639BB243EA05234FF6FF351D4040
:10AE20008B8822F4405245EA0325ABB28D8942EA71
:10AE30000512CD8942EA051292B2C98882808483C4
:10AE40008187038430BD00BF002C0140038C30B5E6
:10AE500023F480521404250C0584038C8288858B8E
:10AE600094B225F4E64215042A0C0D8823F400530D
:10AE700042EA05221D042B0C0D8992B243EA0533E8
:10AE80004D8843EA05330A4D9BB2A84203D005F52D
:10AE90000065A84205D18D8924F4804444EA8514D4
:10AEA000A4B2C98884808283A0F84010038430BD96
:10AEB000002C014000214FF6FF7383800180C18088
:10AEC0004180017270470023038043808380C380E8
:10AED000038143818381C381704700230122038062
:10AEE00043808280C38003817047038819B199B27F
:10AEF00041F0010303E023F001010A04130C038075
:10AF00007047B0F8443029B16FEA43436FEA5341C8
:10AF10008AB201E059044A0CA0F8442070478389A2
:10AF20009BB20AB1194301E023EA01018181704714
:10AF3000038B23F0080213041A0C1143018370479A
:10AF4000038B23F4006213041A0C42EA01218BB232
:10AF500003837047838B23F0080213041A0C1143F8
:10AF600081837047838B23F4006213041A0C42EA36
:10AF700001218BB28383704781847047038B23F058
:10AF80000C0213041A0C0283038B9AB2114301833F
:10AF90007047038B23F4406213041A0C0283038B63
:10AFA0009AB242EA01218BB203837047838B23F06C
:10AFB0000C0213041A0C8283838B9AB2114381838F
:10AFC0007047838B23F4406213041A0C8283838BB3
:10AFD0009AB242EA01218BB283837047F8B50B889D
:10AFE0000D4604464988AA8843B92B89FFF7AAFD74
:10AFF000E9882046BDE8F840FFF7C0BF042B08D120
:10B000002B89FFF7D3FDE9882046BDE8F840FFF71C
:10B01000C0BF082B0E462F89008C3BD120F48073D3
:10B020001804030C2384A08B83B223F0F30343EAB8
:10B030000717374B208CBFB29C4280B247EA02020E
:10B0400012D003F500639C420ED0B4F1804F0BD0B8
:10B05000A3F598339C4207D003F580639C4203D04C
:10B0600003F580639C4207D120F4007040EA06217A
:10B070008BB243F4807305E020F4206041F48071CA
:10B0800040EA0103E9882046A2832384BDE8F84012
:10B09000FFF78CBF20F480531804030C2384A38B88
:10B0A000208C23F440731B051B0D43EA022242EA65
:10B0B0000733174A80B294429BB212D002F5006265
:10B0C00094420ED0B4F1804F0BD0A2F59832944246
:10B0D00007D002F58062944203D002F58062944268
:10B0E00007D120F4005040EA063291B241F4805278
:10B0F00005E047F6FF52024041F480510A43E988D7
:10B100002046A3832284BDE8F840FFF75ABF00BF62
:10B11000002C0140808E80B27047008F80B2704753
:10B12000808F80B27047B0F8400080B27047038AC9
:10B13000828911EA030092B203D011420CBF0020B1
:10B1400001207047C9438AB202827047038A30B532
:10B150000D460446EA8898B220F4405111432182FA
:10B16000A3892889A98823F4B05340EA0102688999
:10B1700023F00C0102430804030C1A4391B2A1818D
:10B18000A08AAA8983B223F4407187B01143A182B7
:10B1900001A800F0EBF81848A38984420CBF04987A
:10B1A000039819B200294FF019032A6803FB00F035
:10B1B00001DA510000E09100B0FBF1F16423B1FB32
:10B1C000F3F21201100903FB1011A08900B200284C
:10B1D00006DAC9003231B1FBF3F303F0070005E0F2
:10B1E00009013231B1FBF3F303F00F00024390B2D7
:10B1F000208107B030BD00BF00380140838919B1FC
:10B2000099B241F4005303E023F400510A04130CF3
:10B2100083817047C1F3421310B5012401F01F016F
:10B22000A34204FA01F101D10C3004E0022B01D158
:10B23000103000E01430036812B143EA010201E06B
:10B2400023EA0102026010BD838A9BB20AB119434E
:10B2500001E023EA0101818270470000034A044BA8
:10B2600002F188305A605860704700BF230167457B
:10B2700000200240024B1A6942F0800018617047BA
:10B2800000200240014BD860704700BF0020024000
:10B29000084BDA68D20709D4D868400708D4D968BF
:10B2A00011F0100F0CBF04200320704701207047DD
:10B2B000022070470020024010B50446FFF7E8FF67
:10B2C000012806D11CB1FFF7E3FF013CF8E7052098
:10B2D00010BD002C08BF052010BD000073B5002371
:10B2E00006464FF400500D460193FFF7E5FF042892
:10B2F0001AD10E4CAAB2206940F0010121614FF42D
:10B3000000503280FFF7D8FF042808D1023601969A
:10B31000019B2D0C1D804FF40050FFF7CDFF2169DC
:10B3200041F6FE720A4022617CBD00BF002002404F
:10B3300038B505464FF43020FFF7BEFF042812D180
:10B34000094C236943F002002061656121694FF4D3
:10B35000302041F040022261FFF7AEFF216941F643
:10B36000FD730B40236138BD00200240204B10B517
:10B370005A6802F00C01042903D0082905D01D4B9E
:10B3800001E01D4C2368036011E05C685968C4F358
:10B390008342941CC90301D4184A06E016495B682D
:10B3A0000A6813F4003F18BF520854430460104B5E
:10B3B0005968C1F3031212498C5C026822FA04F244
:10B3C00042605C68C4F302240C5D22FA04F48460D9
:10B3D0005C68C4F3C224095D22FA01F2C2605B68B2
:10B3E0000849C3F38133CB5CB2FBF3F2026110BDB9
:10B3F0000010024000127A004C01002000093D00BC
:10B400005801002054010020044B5A6909B110432F
:10B4100001E022EA00005861704700BF00100240BE
:10B42000044B9A6909B1104301E022EA00009861D7
:10B43000704700BF00100240044BDA6909B11043A5
:10B4400001E022EA0000D861704700BF001002400E
:10B45000044BDA6809B1104301E022EA0000D86029
:10B46000704700BF00100240044B1A6909B1104335
:10B4700001E022EA00001861704700BF001002409E
:10B48000024B5A6A42F080705862704700100240C6
:10B4900008B50B4B984207D14FF400100121FFF77C
:10B4A000E3FF4FF4001006E04FF480000121FFF7A6
:10B4B000DBFF4FF480000021BDE80840FFF7D4BF58
:10B4C00000540040F0B58688044687B026F03F005F
:10B4D0000D46010401A80E0CFFF748FF2C4A039902
:10B4E000B1FBF2F087B23E43A680238823F001022D
:10B4F00013041A0C22802B68264A93420AD85B0058
:10B50000B1FBF3F0013783B2BFB22784032B98BF9E
:10B51000042320E0EE884BF6FF72964204D103220A
:10B520005343B1FBF3F305E019225343B1FBF3F1AD
:10B5300041F4804399B20A054FF4967208BF41F076
:10B540000101504341F400434FF47A7190FBF1F054
:10B55000421C91B22184A383228891B241F001035D
:10B560002380208820F4816222F002010B04AA8843
:10B570006989180C41EA02032989AA89184380B213
:10B5800041EA0203208098B2208107B0F0BD00BFDD
:10B5900040420F00A086010041F288330021036081
:10B5A0004BF6FF724FF480438180C280018141815C
:10B5B00083817047038819B199B241F0010303E018
:10B5C00023F001010A04130C03807047038819B1AA
:10B5D00099B241F4807303E023F480710A04130CE0
:10B5E00003807047038819B199B241F4007303E0F6
:10B5F00023F400710A04130C03807047038819B107
:10B6000099B241F4806303E023F480610A04130CCF
:10B610000380704783889BB20AB1194301E023EA93
:10B6200001018180704701827047008AC0B2704773
:10B6300012B141F0010101E001F0FE010182704709
:10B6400002684FF6FE73134003602D4B00219842B1
:10B65000016041608160C16022D02A49884229D0BE
:10B66000294B984230D02949884237D0284B9842FC
:10B670003ED0284B984206D153F8681C41F4700024
:10B6800043F8680C70472449884206D151F87C0C75
:10B6900040F0706241F87C2C7047204B984206D1F4
:10B6A00053F8042C42F00F0143F8041C70471C4966
:10B6B000884206D151F8183C43F0F00041F8180CCC
:10B6C0007047184B984206D153F82C2C42F4706105
:10B6D00043F82C1C70471449884206D151F8403C6D
:10B6E00043F4704041F8400C7047104B984205D12C
:10B6F00053F8542C42F4702143F8541C704700BF97
:10B70000080002401C000240300002404400024099
:10B71000580002406C0002408000024008040240D1
:10B720001C04024030040240440402405804024019
:10B7300070B506688C680D6A26F4FF4222F0700628
:10B740000A6945EA04034C6913438A692343CC69B7
:10B7500013431C434B6A44EA03028B6A1A43324385
:10B760000260CB680A68496843608260C16070BD4E
:10B770000023036043608360C360036143618361AE
:10B78000C361036243628362704719B1016841F08B
:10B79000010303E002684FF6FE7313400360704735
:10B7A00003680AB1194301E023EA0101016070470F
:10B7B00041607047406880B270470000C3004CBFD2
:10B7C000014B024B586070470004024000000240E9
:10B7D00000B540F6D87320F00042C3F649739A4290
:10B7E00083B0014615DDB2F1FF4F03DBF5F7D8F862
:10B7F00003B000BD694600F095FB00F00302012A8A
:10B80000009801990ED0022A07D082B900F0A0FD5D
:10B81000EEE7002100F09CFDEAE700F099FD00F161
:10B820000040E5E701F040FC00F10040E0E70122C4
:10B8300001F03AFCDCE700BF30B5C0F3C754A4F117
:10B840007F031E2B83B0014621DC581C1DDBCD0F6E
:10B85000162B0CDD21F07F4323F4000040F40000A0
:10B86000963C00FA04F005B1404203B030BD1148E7
:10B8700050F825402046F5F795F8019021460198AB
:10B88000F5F78EF820F0004121B90020EDE7F5F73B
:10B8900057FBEAE720F07F4222F40003C0F3C750D1
:10B8A00043F40001C0F1960221FA02F0002DDCD031
:10B8B000DAE700BFD00A010800B540F6D87320F0DF
:10B8C0000042C3F649739A4283B0014616DDB2F1D5
:10B8D000FF4F03DBF5F764F803B000BD694600F0E5
:10B8E00021FB00F00300012815D002280BD0B8B9C5
:10B8F00000980199012201F0D7FBEDE70021002219
:10B9000001F0D2FBE8E700980199012201F0CCFB9D
:10B9100000F10040E0E70098019900F019FDDBE735
:10B920000098019900F014FD00F10040D4E700BF39
:10B9300070B58AB0064600F09BF8224C054694F993
:10B940000030013303D0304601F0B0FD10B9284675
:10B950000AB070BD304601F05BFD4FF07E51F5F747
:10B96000E5FA0028F3D0184A01210025304601925B
:10B9700000910895F4F75AFD02460B461348CDE9AD
:10B980000423CDE9022301F011FC94F90030CDE944
:10B990000601022B0BD0684601F006FC38B108986E
:10B9A00050B9DDE90601F4F7A7FF0546CFE701F03E
:10B9B00089FE21210160F2E701F084FE089A02600D
:10B9C000EFE700BF68010020D80A0108E00A01087B
:10B9D00000F002BA70B58AB0054600F04FFC224C68
:10B9E000064694F90030013308D0284601F05EFD88
:10B9F00020B128460021F5F77BFA10B930460AB08D
:10BA000070BD1A4A0121284600260091019208962D
:10BA1000F4F70CFD2478CDE90401CDE902017CB9ED
:10BA200000220023CDE90623684601F0BDFB88B162
:10BA30000898A0B9DDE90601F4F75EFF0646DDE7E8
:10BA40000020002102460B46F4F76EFE022CCDE9E1
:10BA50000601E9D101F036FE21230360E8E701F099
:10BA600031FE08990160E5E768010020E40A010859
:10BA7000F8B520F00043B3F17E5F044613D00BDC31
:10BA8000B3F17C5F14DAB3F10C5F00F3A48040F6ED
:10BA9000DB70C3F6C970F8BD0146F4F781FF0146BB
:10BAA000F5F73CF9F8BD002840F30E810020F8BD01
:10BAB0000028C0F20E8101464FF07E50F4F770FF6F
:10BAC0004FF07C51F5F776F8044600F0D7FB4EF6C0
:10BAD0000871064620F47F65C3F611012046F5F78C
:10BAE00069F847F60471C3F64F21F4F75BFF21466E
:10BAF000F5F760F841F24611C3F62451F4F750FF10
:10BB00002146F5F757F840F6A821C3F64E61F4F741
:10BB100049FF2146F5F74EF84BF29001C3F6A661B6
:10BB2000F4F73EFF2146F5F745F84AF6AB21C3F698
:10BB30002A61F4F737FF2146F5F73CF84CF22E6105
:10BB40000746C3F69D512046F5F734F843F26131BC
:10BB5000C3F63071F4F724FF2146F5F72BF845F2D0
:10BB60002D71C4F20101F4F71DFF2146F5F722F80B
:10BB70004DF23911C4F21901F4F712FF2146F5F71D
:10BB800019F84FF07E51F4F70DFF01463846F5F7EE
:10BB9000C5F83146F5F70EF825F00F05074629469A
:10BBA0002846F5F707F801462046F4F7F9FE29463E
:10BBB00004463046F4F7F6FE01462046F5F7AEF8A7
:10BBC00001463846F4F7EEFE2946F4F7EBFE01464F
:10BBD000F4F7E8FEF8BD0146F4F7ECFF4EF6087105
:10BBE000C3F611010546F4F7E5FF47F60471C3F605
:10BBF0004F21F4F7D7FE2946F4F7DCFF41F2461156
:10BC0000C3F62451F4F7CCFE2946F4F7D3FF40F6EF
:10BC1000A821C3F64E61F4F7C5FE2946F4F7CAFF22
:10BC20004BF29001C3F6A661F4F7BAFE2946F4F789
:10BC3000C1FF4AF6AB21C3F62A61F4F7B3FE2946E9
:10BC4000F4F7B8FF4CF22E610646C3F69D51284624
:10BC5000F4F7B0FF43F26131C3F63071F4F7A0FEA0
:10BC60002946F4F7A7FF45F22D71C4F20101F4F75C
:10BC700099FE2946F4F79EFF4DF23911C4F21901DD
:10BC8000F4F78EFE2946F4F795FF4FF07E51F4F756
:10BC900089FE01463046F5F741F801462046F4F7A3
:10BCA00089FF014642F26810C3F2A230F4F778FE31
:10BCB00001462046F4F774FE014640F6DA70C3F6FA
:10BCC000C970F4F76DFEF8BD40F6DB70C4F24900B0
:10BCD000F8BD4FF07E51F4F765FE4FF07C51F4F75C
:10BCE00069FF4EF60871C3F611010446F4F762FFCE
:10BCF00047F60471C3F64F21F4F754FE2146F4F7DA
:10BD000059FF41F24611C3F62451F4F749FE21468A
:10BD1000F4F750FF40F6A821C3F64E61F4F742FE57
:10BD20002146F4F747FF4BF29001C3F6A661F4F702
:10BD300037FE2146F4F73EFF4AF6AB21C3F62A61EF
:10BD4000F4F730FE2146F4F735FF0646204600F0B2
:10BD500095FA4CF22E610546C3F69D512046F4F744
:10BD600029FF43F26131C3F63071F4F719FE214621
:10BD7000F4F720FF45F22D71C4F20101F4F712FE31
:10BD80002146F4F717FF4DF23911C4F21901F4F707
:10BD900007FE2146F4F70EFF4FF07E51F4F702FE46
:10BDA00001463046F4F7BAFF2946F4F703FF42F2A2
:10BDB0006811C3F2A231F4F7F3FD01462846F4F707
:10BDC000F1FD0146F4F7EEFD014640F6DA70C4F2EB
:10BDD0004900F4F7E5FDF8BDF8B521F00044B4F1F1
:10BDE000FF4F034617DC20F00045B5F1FF4F064634
:10BDF00011DCB1F17E5F42D08F1707F0020040EAFC
:10BE0000D37775B9022F35D0032F08D140F6DB73F5
:10BE1000CCF2490303E01846F4F7C4FD0346184684
:10BE2000F8BDD4B1B4F1FF4F2DD0B5F1FF4F14D010
:10BE30002C1BE4153C2C18DC002952DB1846F4F7C7
:10BE40006DFF01F0E5FA01F0B7F9012F46D0022F9E
:10BE500035D0002F25D10346E1E7002E40F6DB73F5
:10BE60001CDBC3F6C9731846F8BD40F6DB70C3F699
:10BE7000C970EAE740F6DB73C4F24903CFE7BDE8D7
:10BE8000F84001F099B9B5F1FF4F2FD0022FF1D052
:10BE9000032FBBD0012F34D00023C0E7CBF6C973EA
:10BEA000BDE74BF62E51C3F2BB31F4F77BFD40F6F4
:10BEB000DB71C4F24901F4F773FD0346AFE74BF6BB
:10BEC0002E51C3F2BB31F4F76DFD014640F6DB7035
:10BED000C4F24900F4F764FD0346A0E700F1004313
:10BEE0009DE714F13C0FA9DA0020AEE7022F13D032
:10BEF000032F0CD0012F40F6DB7305D0C3F6497336
:10BF00008DE74FF000438AE7CBF6497387E74CF69D
:10BF1000E433CCF2160382E74CF6E433C4F21603A2
:10BF20007DE700BF2DE9F04F40F6D87320F00044C4
:10BF3000C3F649739C4289B006460D4640F38B8098
:10BF40004CF6E331C4F216018C4226DC4FF47861E2
:10BF50000028C3F6C97140F32B81F4F721FD4FF49B
:10BF60007D6224F00F04C3F6C9729442064600F0C5
:10BF7000818044F24341C3F23571F4F711FD01466B
:10BF800028603046F4F70CFD44F24341C3F23571AA
:10BF9000F4F706FD0127686061E04FF47867C4F2AA
:10BFA0004937BC4240F38180B4F1FF4F5BDA4FEA7E
:10BFB000E459A9F18609A4EBC9542046F4F7C0FF5F
:10BFC000F4F7A4FD0246014620460592F4F7E8FC8A
:10BFD0004FF08741F4F7EEFD0746F4F7B1FFF4F7B1
:10BFE00095FD0146044638460694F4F7D9FC4FF017
:10BFF0008741F4F7DFFD00210790F4F76FFF002879
:10C0000000F0F6800327204600210DF11808013FBB
:10C01000F4F764FF40B158F8044D00212046013F79
:10C02000F4F75CFF0028F6D1924B022000900193B8
:10C0300005A83B4629464A4600F066FA002E074608
:10C040000DDA95E80C0002F1004103F1004229608D
:10C050006A60474203E00023286000274B603846AF
:10C0600009B0BDE8F08F0146F4F79AFC002768603C
:10C070002860F4E74FF48841C3F23571F4F790FC7F
:10C080004AF20831C2F685610446F4F789FC01469C
:10C0900028602046F4F784FC4AF20831C2F6856134
:10C0A000F4F77EFC01276860D9E701F0B1F94FF69B
:10C0B0008411C3F622718046F4F77CFD4FF07C5169
:10C0C000F4F770FCF4F73CFF0746F4F71FFD4FF45C
:10C0D0007861C3F6C9718346F4F76CFD01464046AA
:10C0E000F4F75EFC44F243418146C3F23571584691
:10C0F000F4F760FD1F2F8246514648461FDC5E4B19
:10C100007A1E53F8223024F0FF029A4217D0F4F737
:10C1100047FC8046C5F8008041464846F4F740FC9D
:10C120005146F4F73DFC002E686098DA08F10048AB
:10C1300000F10041C5F8008069607F428FE7F4F7A5
:10C140002FFCE3158046C0F3C750191A0829E1DD1A
:10C150004FF48841C3F2357158460393F4F72AFD32
:10C16000824651464846F4F71BFC044621464846A1
:10C17000F4F716FC5146F4F713FC4AF208318146F5
:10C18000C2F685615846F4F715FD4946F4F708FCF8
:10C19000824651462046F4F703FC039BC0F3C75286
:10C1A0008046981A192841DCC5F80080A146B3E7FB
:10C1B000F4F7F8FB4FF47D6724F00F04C3F6C9775A
:10C1C000BC42064616D044F24341C3F23571F4F73F
:10C1D000E9FB014628603046F4F7E2FB44F24341B4
:10C1E000C3F23571F4F7DEFB4FF0FF37686036E7D6
:10C1F000032719E74FF48841C3F23571F4F7D2FBF6
:10C200004AF20831C2F685610446F4F7CBFB0146D9
:10C2100028602046F4F7C4FB4AF20831C2F6856173
:10C22000F4F7C0FB4FF0FF37686018E74FF4234185
:10C23000C2F685615846F4F7BDFC8046414620466B
:10C24000F4F7AEFB814649462046F4F7A9FB414688
:10C25000F4F7A6FB43F232110446C2F28D41584670
:10C26000F4F7A8FC2146F4F79BFB8246514648466A
:10C270004DE700BF6C0B0108EC0A010820F00042FA
:10C28000B2F1FF4FF8B50446034646D2002A42D029
:10C29000002852DBC415B2F5000F09D210F40005D6
:10C2A00053D15B0001351902FBD5C5F101002418FB
:10C2B00023F07F417F3C21F40006E20746F40000B2
:10C2C00048BF400043004FF08072002760109A4240
:10C2D0003C462CDD5B004FF400021825A6185108DF
:10C2E0009E4205F1FF3502DCB4189B1BBF185B00B2
:10C2F00062189A4202DC9B1A54187F185B004A08A5
:10C30000013DEBD113B107F001017F187C1004F15E
:10C310007C5303EBC0542046F8BD0146F4F74AFCB9
:10C3200001462046F4F73EFB04462046F8BD4FF098
:10C33000007403F17F431746CCE70146F4F730FB66
:10C340000146F4F7EBFC0446E5E70120AFE700BF48
:10C350002DE9F84320F00046B6F1485F05460F4648
:10C360005BDAF4F7EDFD002800F0CA802946284684
:10C37000F4F720FC4DF24E71CAF647510446F4F72B
:10C3800019FC47F2F641C3F20F11F4F70BFB2146FB
:10C39000F4F710FC4FF27C21C3F29341F4F700FB59
:10C3A0002146F4F707FC40F60151C3F2D071F4F7CF
:10C3B000F9FA2146F4F7FEFB40F66131C3F6B621E7
:10C3C000F4F7EEFA2146F4F7F5FB4AF6AB21C3F693
:10C3D0002A51F4F7E7FA2146F4F7ECFB80462046B1
:10C3E0004FF07C51F4F7E6FB414606462046F4F751
:10C3F000E1FB394604462846F4F7DCFB01462046BB
:10C40000F4F7CEFA01463046F4F7CAFA01464FF087
:10C410007E50F4F7C5FABDE8F8830146F4F7CAFB8D
:10C420004DF24E71CAF647510446F4F7C3FB47F28A
:10C43000F641C3F20F11F4F7B5FA2146F4F7BAFB4F
:10C440004FF27C21C3F29341F4F7AAFA2146F4F7A4
:10C45000B1FB40F60151C3F2D071F4F7A3FA2146C3
:10C46000F4F7A8FB40F66131C3F6B621F4F798FA69
:10C470002146F4F79FFB4AF6AB21C3F62A51F4F7A5
:10C4800091FA2146F4F796FB49F69913C3F699639E
:10C490009E428046A3DD0020C3F64870864227DC1A
:10C4A00006F17F464FF07E503146F4F779FA814627
:10C4B00020464FF07C51F4F77DFB3146F4F770FADB
:10C4C000414606462046F4F775FB394604462846A1
:10C4D000F4F770FB01462046F4F762FA0146304655
:10C4E000F4F75EFA01464846F4F75AFABDE8F883D5
:10C4F0004FF000090026C3F63879C3F69066D7E7F7
:10C500004FF07E50BDE8F8832DE9F04FDFB00C937B
:10C510000C9D224B689C0A91691ED61E48BF161DB1
:10C52000834653F82400F71027EAE7730890049134
:10C5300004980D93089DDC43DDF834C002EBC4027F
:10C5400041190792C0EB0C0750D47E18699BC7EBCA
:10C5500006090136002F03EB870522AC09F0010A1A
:10C56000C0F2FE822868F4F7D1FA0137B7422060A2
:10C570004FF004083AD0BAF1000F26D0002FC0F2D5
:10C58000F18255F80800F4F7C1FA0137B74244F8D0
:10C59000080008F1040818D128E000BF840E010843
:10C5A00055F80800F4F7B2FA013708F1040944F825
:10C5B000080013D455F80900F4F7A8FA0137B74278
:10C5C00044F8090009F1040810D0002FE8DA00202F
:10C5D000013708F1040944F80800EBD501370020C1
:10C5E000B74244F8090009F10408EED1089A002A7C
:10C5F000C0F2458508990C9E8D004AAB5C190395E5
:10C6000049AF02944FEA860A049A002AC0F2968241
:10C610000DF1880808EB860555F8041CAAF10403FF
:10C62000DBF80000C3F38009F4F7C4FA01460020E8
:10C63000F4F7B8F90424043D544580462BD0B9F1F1
:10C64000000F0DD055F8041DDBF80400F4F7B2FA22
:10C6500001464046F4F7A6F90824544580461AD00E
:10C6600055F8041C5BF80400F4F7A4FA01464046B0
:10C67000F4F798F90434804655F8081C5BF8040078
:10C68000F4F798FA01464046F4F78CF90434083D73
:10C6900054458046E4D1029847F8048F013687421A
:10C6A000B2D1039F0EA9CE190996089EB2005EABC7
:10C6B0009D18002E029255F8509C7DDD0DF5947C5E
:10C6C0004FF06E5148460DACA7180CEB0205F4F77D
:10C6D00071FAF4F735FCF4F719FA4FF0874101903D
:10C6E000F4F768FA01464846F4F75AF9F4F728FCDB
:10C6F0000EAC20600198014655F8040DF4F752F98C
:10C70000BC428146C7F3800156D0E9B14FF06E516B
:10C71000F4F750FAF4F714FCF4F7F8F94FF0874106
:10C720000190F4F747FA01464846F4F739F9F4F76F
:10C7300007FC019A0FAC2060114655F8040DF4F780
:10C7400031F9BC42814637D04FF06E514846F4F77C
:10C7500031FAF4F7F5FBF4F7D9F94FF08741804649
:10C76000F4F728FA01464846F4F71AF9F4F7E8FB1B
:10C770004146606055F8040DF4F714F94FF06E511E
:10C780008146F4F717FAF4F7DBFBF4F7BFF94FF043
:10C7900087418046F4F70EFA01464846F4F700F95F
:10C7A000F4F7CEFB4146A06055F8040DF4F7FAF813
:10C7B0000834BC428146C7D10799484600F0A2FE22
:10C7C0004FF078510546F4F7F5F900F025FE4FF0EB
:10C7D0008241F4F7EFF901462846F4F7E1F80746FD
:10C7E000F4F7AEFB8146F4F791F901463846F4F7C9
:10C7F000D7F807990746002940F33981721E0EAC1D
:10C80000079D54F82230C5F1080043FA00F101FAFF
:10C8100000F0C5F107041B1A43FA04F40DF1380CBB
:10C8200089444CF82230002C55DD002E09F1010915
:10C8300040F39481029D0EABDDF808C053F8042B41
:10C84000281F0DF1380E00250EEB0C01C0F38000FF
:10C8500022B1C2F5807243F8042C01258B4226D008
:10C8600060B10F9A0433002D40F0F38022B1C2F57D
:10C87000807543F8045C01258B4218D053F8042BD3
:10C88000002D40F0EC80C2F5807012B143F8040C2A
:10C89000012553F8042B002D40F0DB80C2F5807099
:10C8A000002AE9D001258B4243F8040CE6D1079910
:10C8B00000290DDD012900F0E280022908D1701E57
:10C8C0000DF1380E5EF8202002F03F034EF82030C4
:10C8D000022C00F0E08038460021F4F7FFFA00282F
:10C8E00000F0F3800898751EA84225DC029B0DF12C
:10C8F000380E0EEB03010B46DDF824C053F8042D6F
:10C90000CCEB0100011F6345C1F3800011D030B1B1
:10C9100053F8041DDDF824E00A43734509D0099F4C
:10C9200053F8040D53F8041D0243BB4242EA0102CE
:10C93000F6D1002A40F01A81089F0EAD781E55F8F6
:10C940002020002A40F0108105EB8004012354F8D8
:10C95000041D01330029FAD0F018771C87420B9090
:10C9600075DCDDF810E00D9D0B9B0C9C0EEB0702B7
:10C97000DDF808C0699F991B06EB05094AA8A619AE
:10C9800022AB07EB890900EB0C05571C8A0003EB6F
:10C990008601029506920591002659F8040FF4F7D6
:10C9A000B5F8059CA051049800285EDB22AD05EB8C
:10C9B0008702AAF10403C3F3800452F8041CDBF8D5
:10C9C00000000394141FF4F7F5F801460020F3F774
:10C9D000E9FF4FF00408D04505462DD0039971B109
:10C9E00054F8041DDBF80400F4F7E4F80146284687
:10C9F000F3F7D8FF4FF00808D04505461CD054F88F
:10CA0000041C5BF80800F4F7D5F801462846F3F754
:10CA1000C9FF08F10408054654F8081C5BF8080033
:10CA2000F4F7C8F801462846F3F7BCFF08F10408FC
:10CA3000083CD0450546E2D1DDF808E0069804360A
:10CA40004EF8045F01378642CDF808E0A5D10B9E71
:10CA50002CE6C2F1FF0243F8042C01250CE7C2F1D9
:10CA6000FF0543F8045C012513E70025E4E75ED1E8
:10CA7000701E0DF1380E5EF820301C12D3E6711EC8
:10CA80000DF1380C5CF82100022C00F07F024CF80C
:10CA900021207FF420AF39464FF07E50F3F780FF1E
:10CAA0000746002D3FF417AF07994FF07E5000F076
:10CAB00029FD01463846F3F773FF07463846002143
:10CAC000F4F70CFA00287FF40DAF0294079C384667
:10CAD0006142CDF8109000F015FD4FF087410546FA
:10CAE000F4F71AFA002800F0D2824FF06E5128466F
:10CAF000F4F760F8F4F724FAF4F708F84FF08741F8
:10CB00000746F4F757F801462846F3F749FFF4F7CC
:10CB100017FA0EA941F826003846F4F711FA079AD9
:10CB2000013608320EAC079244F8260034E04FF08C
:10CB30007C51F4F7F1F958B90024CCE64FF0000825
:10CB4000029847F8048F013687427FF45DADA8E56F
:10CB50000224002E09F101093FF76CAE0025A6E67C
:10CB6000002002E5002010E50123F5E6079A0EAE4D
:10CB700056F82530083ACDF8109002940792002B11
:10CB800040F08E8206EB85042E4654F8045D013E8B
:10CB9000083A002DF9D007924FF07E50079900F027
:10CBA000B1FC002E0446C0F2AC804FEA860AC6EB08
:10CBB000867B0EAF4FEA8B095744C9F100034AA99F
:10CBC000386801EB0A08C3F3800BF3F79FFF214697
:10CBD000F3F7F0FF4FF06E51C8F800002046F3F76E
:10CBE000E9FFA9F104096FF0030ACA45054631D0EF
:10CBF000BBF1000F0BD057F8040CF3F787FF294661
:10CC0000F3F7D8FF6FF0070A48F8040C1AE057F85A
:10CC10000A00F3F77BFF2946F3F7CCFF4FF06E5184
:10CC200048F80A002846F3F7C5FFAAF104040546B0
:10CC30003859F3F76BFF2946F3F7BCFFAAF1080A4E
:10CC400048F8040028464FF06E51F3F7B3FFCA4589
:10CC50000546DCD1701CDFF84C94DDF820A0039071
:10CC600000270596BAF1000FC0F20582002FC0F22E
:10CC70000282002600241AF0010F354620D0D8F891
:10CC80000010D9F80000F3F795FF01462046F3F7AE
:10CC900089FE0125AA45044626DB0426BD420FDD98
:10CCA00022E0BB4520DC58F8021059F80200F3F7E7
:10CCB00081FF01462046F3F775FEBD42044613DCB2
:10CCC00058F8061059F80600F3F774FF014620469D
:10CCD000F3F768FE05F1010B06F104020235DA45AF
:10CCE000044602F10406DCDA5EABDDF80CC003EBAF
:10CCF00087010137674541F8A04CA8F10408B1D17C
:10CD0000059E689C032C16D8DFE814F085011F01EE
:10CD10001F011B0000230299002900F00B81379CA2
:10CD2000369804F100420A9C00F1004503F10043EB
:10CD300025606260A360049D05F007005FB0BDE858
:10CD4000F08F002EE6DD06F1FF3836AF07EB8809DD
:10CD50004D4655F804290DF1D40AD5F808B010460F
:10CD600059460192F3F71EFE804641460198F3F7BB
:10CD700017FE01465846F3F715FE5545C9F38003E3
:10CD8000A860C5F8048044D0BBB155F80429D5F893
:10CD900008B0104659460192F3F704FE0199804607
:10CDA00008464146F3F7FCFD01465846F3F7FAFD05
:10CDB0005545C5F80480A8602BD02C4654F804399A
:10CDC000D4F808B0184659460193F3F7EBFD8046B6
:10CDD00041460198F3F7E4FD01465846F3F7E2FDBA
:10CDE000C4F80480A06055F804BC251FD5F808805D
:10CDF00058464146F3F7D6FD044621465846F3F718
:10CE0000CFFD01464046F3F7CDFD55456C60A86067
:10CE1000D3D1012E7FF77EAF4D4655F804B9C7EB4D
:10CE2000090ED5F808A058465146AEF10409F3F7AB
:10CE3000B9FD804641465846F3F7B2FD01465046DB
:10CE4000F3F7B0FDBD42C9F38009C5F80480A860BE
:10CE500043D0B9F1000F15D055F804A9D5F80890C2
:10CE600050464946F3F79EFD804641465046F3F74B
:10CE700097FD01464846F3F795FDBD42C5F804808D
:10CE8000A8602AD02C4654F804A9D4F8089050463B
:10CE90004946F3F787FD804641465046F3F780FD4B
:10CEA00001464846F3F77EFDC4F80480A06055F8BB
:10CEB000049C251FD5F8088048464146F3F772FDCB
:10CEC000044621464846F3F76BFD01464046F3F71A
:10CED00069FDBD426C60A860D4D1013607EB8607BE
:10CEE00008353E467A1B131F56F8041D0020C3F375
:10CEF0008007F3F757FDAE4203463FF40CAF3FB156
:10CF000056F8041DF3F74EFDAE4203463FF403AF5F
:10CF1000184656F8041C341FF3F744FD083E54F835
:10CF2000041CF3F73FFDAE42F3D1029903460029FA
:10CF30007FF4F5AEDDF828C036993798CCF80010AC
:10CF4000CCF80400CCF80830F5E60023002E29DBED
:10CF500036AF751C07EB85042546E21B55F8041D0A
:10CF6000A2F1040E0020CEF38008F3F71BFDBD42B2
:10CF7000034617D0B8F1000F06D055F8041DF3F79B
:10CF800011FDBD4203460DD0184655F8041C2C1F58
:10CF9000F3F708FD083D54F8041CF3F703FDBD4208
:10CFA000F3D103460299002967D003F10040DDF870
:10CFB00028C01946CCF800003698F3F7F1FC002E93
:10CFC000034621DD36AF07EB8606F51B2A1F37998E
:10CFD000C2F38007F3F7E6FC37ACB442034613D044
:10CFE00037B16168F3F7DEFC38ACB44203460BD0CE
:10CFF000184654F8041FF3F7D5FC54F8041FF3F750
:10D00000D1FCB442F5D10346029909B103F10043C2
:10D010000A9C63608FE6002E40DB36AF013607EBDB
:10D0200086000546C21B55F8041D0020141FF3F7A7
:10D03000B9FCBD42C4F38006034615D036B155F89D
:10D04000041DF3F7AFFCBD4203460DD0184655F85A
:10D05000041C2C1FF3F7A6FC083D54F8041CF3F73E
:10D06000A1FCBD42F3D10346029909B103F100438B
:10D070000A9C23605FE6002436E6184697E7DDF851
:10D0800030E0900003904FEA8E0AFFF70ABB284673
:10D09000F3F756FF0EAB43F826007DE50023E3E7E8
:10D0A0002E4679E5900E01082DE9F84320F0004363
:10D0B000B3F1485F04460F46904603DAF3F740FFAA
:10D0C000002859D021462046F3F774FD2146054635
:10D0D000F3F770FD4CF6D311C2F62E7106462846C2
:10D0E000F3F768FD42F63471C3F2D721F3F758FC29
:10D0F0002946F3F75FFD4EF61B71C3F23861F3F773
:10D1000051FC2946F3F756FD40F60151C3F6501184
:10D11000F3F746FC2946F3F74DFD48F68901C3F6BF
:10D120000841F3F73FFC8146B8F1000F27D04FF0DC
:10D130007C513846F3F73EFD494680463046F3F7CA
:10D1400039FD01464046F3F72BFC2946F3F732FD43
:10D150003946F3F725FC4AF6AB210546C3F62A61AA
:10D160003046F3F727FD01462846F3F71BFC01463E
:10D170002046F3F715FC04462046BDE8F883014637
:10D180002846F3F717FD4AF6AB21C3F62A61F3F7F9
:10D1900007FC3146F3F70EFD01462046F3F702FC8B
:10D1A00004462046BDE8F883002070470021002097
:10D1B000C7F6F871704700BF2DE9F04120F0004537
:10D1C000B5F1A14F044606460DDBB5F1FF4F00F364
:10D1D0009C80002840F6DB7440F3D480C3F6C97409
:10D1E0002046BDE8F0814FF6FF73C3F6DF639D4232
:10D1F00000F3A280B5F1445FC0F28E804FF0FF379C
:10D2000021462046F3F7D6FC01468046F3F7D2FCD0
:10D2100046F6D711C3F685410546F3F7CBFC4DF62C
:10D220005921C3F64B51F3F7BDFB2946F3F7C2FC76
:10D2300046F63531C3F68851F3F7B4FB2946F3F7C8
:10D24000B9FC42F66E61C3F6BA51F3F7ABFB29465F
:10D25000F3F7B0FC44F62511C3F61261F3F7A2FB15
:10D260002946F3F7A7FC4AF6AB21C3F6AA61F3F708
:10D2700099FB4146F3F79EFC4AF221218046CBF60A
:10D2800015512846F3F796FC4FF26B11C3F66E5119
:10D29000F3F786FB2946F3F78DFC48F29571C3F648
:10D2A0009D51F3F77DFB2946F3F784FC48F638617E
:10D2B000C3F6E351F3F774FB2946F3F77BFC4CF616
:10D2C000CD41C3F64C61F3F76BFB2946F3F772FCD3
:10D2D0007B1C0146404658D0F3F764FB2146F3F728
:10D2E00069FC494B53F82710F3F75AFB2146F3F733
:10D2F00057FB0146454850F82700F3F751FB002E35
:10D300003DDB04462046BDE8F0810146F3F74AFBC9
:10D3100004462046BDE8F0814FF2CA21C7F2491108
:10D32000F3F740FB4FF07E51F3F700FE00283FF487
:10D3300065AF2046BDE8F08100F06AF84FF6FF7156
:10D34000C3F697718D4204464FF6FF7228DCC3F690
:10D350002F72954246DC0146F3F724FB4FF07E51D5
:10D36000F3F71EFB4FF0804105462046F3F71AFB0A
:10D3700001462846F3F7D2FC0027044640E700F1B7
:10D3800000442DE7CBF6C9742AE7F3F70BFB2146DF
:10D39000F3F710FC01462046F3F702FB04461FE7B3
:10D3A000C4F21B02954214DC4FF07F51F3F7F8FAF8
:10D3B0004FF07F5105462046F3F7FCFB4FF07E51BE
:10D3C000F3F7F0FA01462846F3F7A8FC02270446D3
:10D3D00016E700202146CBF68070F3F79FFC032769
:10D3E00004460DE74FF07E51F3F7DAFA4FF07E5125
:10D3F00007462046F3F7D6FA01463846F3F78EFC87
:10D4000001270446FCE600BFBC0E0108CC0E010853
:10D4100020F00040704700BFF8B520F00046F50D41
:10D420007F3D162D014604461BDC002D074620DB00
:10D430004FF6FF73C0F27F0343FA05F606420ED0A3
:10D440004FF2CA21C7F24911F3F7ACFA0021F3F702
:10D450006DFD18B1002C1BDB27EA060421460846A7
:10D46000F8BDB6F1FF4FFAD3F3F79CFA0146084630
:10D47000F8BD4FF2CA21C7F24911F3F793FA002120
:10D48000F3F754FD0028E9D0002C07DB0024E5E782
:10D490004FF4000040FA05F56719DDE70021CBF6EF
:10D4A0008071002E18BF0C46D8E700BF08B90220D3
:10D4B0007047B0F1004FFAD0A0F500026FF00143C1
:10D4C0009A4201D80420704700F1FF419942F9D9EE
:10D4D0004FF6FE73421EC0F27F039A4201D803202A
:10D4E000704700F100414A1E9A42F8D9B0F1FF4F4F
:10D4F00005D010F5000F14BF002001207047012057
:10D50000704700BF38B530F00044034602460D4670
:10D510000FD0B4F1FF4F0ED2B4F5000F11D3E40DCC
:10D520006419FE2C33DC002C1BDD22F0FF4141EAA4
:10D53000C453184638BD0146F3F734FA034618467B
:10D5400038BD4FF09841F3F735FB43F6B041CFF6C5
:10D55000FF718D42034612DBC0F3C7540246193CEB
:10D56000DEE714F1160F21DA4CF2503295421946DB
:10D570000EDC44F26020C0F6A25000F023F844F222
:10D580006021C0F6A251F3F715FB0346D1E7194617
:10D590004FF2CA20C7F2491000F014F84FF2CA2126
:10D5A000C7F24911F3F706FB0346C2E722F0FF4337
:10D5B00004F1190043EAC0504FF04C51F3F7FAFA66
:10D5C0000346B6E701F0004120F0004008437047F1
:10D5D0002DE9F041274C84B025680746D5F848412D
:10D5E000002C41D066681F2E1CDD234810B94FF077
:10D5F000FF301FE04FF4C870039102920193AFF324
:10D60000008003990446029A019B0028EFD0D5F8C8
:10D610004861002060602660C5F84841C4F8880170
:10D62000C4F88C01656847B9A81C013544F820107E
:10D630006560002004B0BDE8F081012000FA05F02B
:10D64000D4F8886104EB85080643022FC8F88820C7
:10D65000C4F88861C8F80831E6D1D4F88C3143EABF
:10D660000002C4F88C21DFE705F5A674C5F848412F
:10D67000B8E700BFE40F01080000000000210A2203
:10D6800001F028B82DE9F84FDDF828B081468A4628
:10D6900098469AB193B11646002503E00FD0651C59
:10D6A000AE420BD97419640808FB04A748463946F2
:10D6B000D8470028F2DA2646AE42F3D8002738468B
:10D6C000BDE8F88F40F29853C2F200031868704723
:10D6D000114B124A70B5981A831018D0591E02EBDC
:10D6E00083040D4654F8042D01F00106904775B1EE
:10D6F00026B154F8040D8047013D08D054F8043D8C
:10D700009847013D54F8041D8847013DF6D1BDE816
:10D71000704003F06FBC00BF0C1001080810010836
:10D72000F8B5204F204C381B871017D07A1E23687D
:10D73000012502F001069847AF420FD02EB154F8F0
:10D74000041F02258847AF4208D060688047023531
:10D75000A268261D90470834AF42F6D1134F144CEF
:10D7600003F042FC3B1B9F1018D07D1E216805F082
:10D77000010601258847AF4211D02EB154F8040F9D
:10D7800002258047AF420BD0626890470235A368FC
:10D79000261D98470834AF42F6D1F8BDF8BDF8BD54
:10D7A000F8BD00BF001001080010010808100108B2
:10D7B000001001080F2A2DE9F00340F2A18041EA90
:10D7C00000039B0740F09E800C68A2F110050460E6
:10D7D0004B68AC4643608C68BCF10F0F8460CC682A
:10D7E000C5F30015C46000F1100301F110042BD93A
:10D7F00075B12568ACF1100C1D6065685D60A568A9
:10D800009D60E5681034DD601033BCF10F0F1BD94B
:10D81000276804F110061F60676803F110055F6058
:10D82000A768ACF1200C9F60E768DF6024691C6189
:10D83000776806F110046F60B7682033AF60F66850
:10D84000BCF10F0FEE60E3D8A2F1100828F00F032F
:10D8500002F00F0403F1100C032C00EB0C0301EB9E
:10D860000C0851D9211F4FEA9109444608EB890C55
:10D8700054F8046BC8EB0C010CF1040C1D46644514
:10D8800045F8046BC1F3800112D029B154F8041B90
:10D89000644545F8041B0BD0274657F8041B2E4659
:10D8A00046F8041B64686C603C1D351D6445F3D16B
:10D8B00009F1010C4FEA8C0902F0030208EB09019F
:10D8C0004B44D2B10D789A18DC4303F8015B14196C
:10D8D000934204F0010410D02CB111F8014F03F869
:10D8E000014B934209D04D781C4604F8015B8D78BA
:10D8F00002315D70631C9342F5D1BDE8F0037047BF
:10D900000346DEE70346DDE741462246D9E700BF8E
:10D91000F0B48407034600F08D80541E002A00F006
:10D920008780E507CEB211D41A4602F8016B134680
:10D930001546920710D0621E002C79D003F8016BB7
:10D9400014469A071D4607D0013CEDE7034603F84D
:10D95000016B9A071D46F7D1032C52D9CEB246EA85
:10D9600006270F2C47EA07432DD9A4F110021746CA
:10D970000F2FC2F300162B606B60AB60EB6005F1FC
:10D98000100216D93EB1103F136053609360D3600C
:10D9900010320F2F0DD9203F02F110061360536093
:10D9A0009360D360136153619361D36120320F2F71
:10D9B000F1D8A4F1100222F00F0204F00F0410328B
:10D9C000032C15441DD9271F3E462A46032E42F834
:10D9D000043BC7F380070DD927B1043E032E42F85C
:10D9E000043B07D9174647F8043B083E53603A1DED
:10D9F000032EF7D8231F23F00302131D04F00304A2
:10DA0000ED18ACB1C9B2EA432C1905F8011BA318F3
:10DA1000A54203F001020BD01AB105F8011BA54283
:10DA200006D02B4603F8011B69705D1CA542F8D196
:10DA3000F0BC7047054614468EE700BF830770B5FB
:10DA4000064614D10368A3F1013222EA030010F064
:10DA5000803F0CD1331D1A4653F8044BA4F1013515
:10DA600025EA040414F0803FF5D0104600E030466B
:10DA700003782BB1421C147810460132002CFAD1E5
:10DA800000F080F8304670BDC9B2F0B400294BD028
:10DA900082070FD00278002A71D0914242D0431CF5
:10DAA00005E013F8012B002A3BD091423AD09A07A7
:10DAB0001846F6D1036841EA0127A3F1013222EAB0
:10DAC000030212F0803F47EA07471CD17B40A3F1D5
:10DAD000013222EA030313F0803F14D1021D02E059
:10DAE00014F0803F0FD1104652F8043BA3F10136E9
:10DAF00087EA030426EA0303A4F1013513F0803F0B
:10DB000025EA0404ECD00278002A38D0914209D0EA
:10DB1000431C01E0914205D0184613F8012B002A5E
:10DB2000F8D11046F0BC704783070BD00278002A6A
:10DB3000F8D0431C03E0017801330029F2D09907A3
:10DB40001846F8D10168A1F1013323EA010212F06D
:10DB5000803F0AD1031D184653F8041BA1F101347C
:10DB600024EA010212F0803FF5D00378002BD9D0CF
:10DB7000421C1178104601320029FAD1D2E7104632
:10DB8000D0E700BF80EA0102844612F0030F4FD1B4
:10DB900011F0030F32D14DF8044D11F0040F51F87C
:10DBA000043B0BD0A3F101329A4312F0803F04BF33
:10DBB0004CF8043B51F8043B16D100BF51F8044B1C
:10DBC000A3F101329A4312F0803FA4F101320BD14C
:10DBD0004CF8043BA24312F0803F04BF51F8043BD1
:10DBE0004CF8044BEAD023460CF8013B13F0FF0F2E
:10DBF0004FEA3323F8D15DF8044B704711F0010F61
:10DC000006D011F8012B0CF8012B002A08BF704731
:10DC100011F0020FBFD031F8022B12F0FF0F16BF28
:10DC20002CF8022B8CF8002012F47F4FB3D17047F0
:10DC300011F8012B0CF8012B002AF9D1704700BF15
:10DC400020F0030110F00300C0F1000051F8043B84
:10DC500000F1040C4FEACC0C6FF000021CBF22FA5A
:10DC60000CF213434FF0010C4CEA0C2C4CEA0C4C18
:10DC7000A3EB0C0222EA030212EACC1204BF51F811
:10DC8000043B0430F4D013F0FF0F1FBF013013F436
:10DC90007F4F013013F47F0F18BF0130704700BF72
:10DCA000F0B4002A63D0344B04461B6814F8010B0F
:10DCB000571E1D186E7807F0010706F00305012DA9
:10DCC00058D011F8015B5E19767806F00306012E34
:10DCD00008BF2035401B4BD1002D49D0013A47D019
:10DCE0002FB314F8010B1D186E7806F00305012DF3
:10DCF00011F8015B08BF20305E19767806F0030644
:10DD0000012E08BF2035401B32D18DB3013A0ED110
:10DD10002EE011F8012B9E18767806F00306012EEE
:10DD200008BF2032801A23D112B36A1E20D014F803
:10DD3000010B1D186E7806F00305012D11F8015B2B
:10DD400008BF20305E19767806F00306012E08BF62
:10DD50002035401B0CD15DB114F8010B551E1A186B
:10DD6000567806F00302012AD3D12030D1E71046BD
:10DD7000F0BC70472030A4E76C01002041EA0003AA
:10DD80009B07F0B474D1032A72D90C4654F8045B93
:10DD9000161FA5F1013727EA050717F0803F034654
:10DDA000C6F3800C31D10346032E324643F8045BA0
:10DDB0002AD9BCF1000F0AD0214654F8045BA5F122
:10DDC000013626EA050616F0803F18D01DE02646EB
:10DDD00056F8045B2146A5F1013727EA050717F03D
:10DDE000803F12D143F8045B65683146A5F10136E6
:10DDF00026EA0506043A0C1D16F0803F05D1043AC8
:10DE0000032A43F8045BE2D821467AB30D78013A3D
:10DE100003F8015B9DB112F0010F1C462AD1234685
:10DE200022B311F8015F013A03F8015B3DB111F82B
:10DE3000015F013A65705C1C2346002DEFD1AAB149
:10DE400000219C18DA4303F8011BA218A34202F038
:10DE500001020BD01AB103F8011BA34206D01A46E7
:10DE600002F8011B5970531CA342F8D1F0BC704753
:10DE70000346CAE711F8015F1C4604F8015B013A4A
:10DE80002346002DCBD1DAE72DE9F00701273C46E8
:10DE900000254FF0FF3663198B4200EB060C0DD2C4
:10DEA0001CF804A010F80380D0452ED201241D4692
:10DEB0009F1B63198B4200EB060CF1D34FF0010A54
:10DEC0001760544600254FF0FF3C6319994200EB60
:10DED0000C080ED918F8048010F80390C1451AD91F
:10DEE00001241D46CCEB030A6319994200EB0C0890
:10DEF000F0D80CF101000136B0423CBFBA463046C2
:10DF0000C2F800A0BDE8F00770470BD001272E46ED
:10DF10003C46ED19BFE709D04FF0010AAC46544624
:10DF20005544D2E7BC4205D00134B4E7544505D08E
:10DF30000134CAE727461D460124ACE7A2461D4628
:10DF40000124C2E72DE9F04FADF2244D15460646F7
:10DF500089461046194607AA1C46FFF795FF07ABEE
:10DF600082460DF21C411A1D5C6008338B425460DE
:10DF7000F9D114B301232F78611E08A8A34240F8F9
:10DF8000271001EA030218D032B16A7802234F1E2B
:10DF9000A34240F8227010D0B046A4465C1C15F88D
:10DFA00003E0CE1A2A5D02330F1B634540F82E6052
:10DFB00040F82270F2D1464664460799284669180F
:10DFC000524600F045FC002840F0B6800AF1FF3EC2
:10DFD00005EB0E0CCDF808E0CAF1010E834604F102
:10DFE000FF38CDF80CC0CDF814E00746CDF810A0EE
:10DFF0004A460095019408E027B1079FBB4201D231
:10E000000199CB1B9B4400272246019CB0185C441D
:10E010000021A21A00F07CFB002840F08780002C31
:10E0200000F08480301910F8013C08A951F8233021
:10E03000002BE1D1049B9F4228BF3B46434527D29A
:10E04000DDF8009006EB0B0119F80350CA5C09EBF0
:10E050000300954266D1DD43454415F0010F0246A9
:10E0600013D00133434513D24078CD5C0132854251
:10E070000BD057E012F8010FCD5C854252D101332D
:10E0800012F8010FCD5C85424CD101334345F1D3E9
:10E09000DDF81090029B4F4528BF4B4639D2DDF882
:10E0A00008C0DDF8009006EB0B0519F80C1015F808
:10E0B0000C00814240F0C080DDF80CE009EB070A5B
:10E0C000CAEB0E01C80772461ED5DDF8089009F1AB
:10E0D000FF31DDF80C90685C19F801CC09F1FF32D2
:10E0E000844516D10B460FE012F8019C15F800E0AC
:10E0F0004A1EF1450DD10346013815F800C011F84C
:10E10000011C614505D10346581E524502F1FF31FD
:10E11000EAD101379F4200F29180079F019ABB44E8
:10E12000D71B71E7DDF814E0F3446BE7002009B07A
:10E130000DF5806DBDE8F08FCAEB0400504538BF87
:10E140005046CAF10102431C0AF1FF3C05EB0A07E5
:10E1500004F1FF3B019200944A460793B1464FF009
:10E16000000864463E46009909EB020008EB0107EF
:10E17000BA1A002100F0CCFA0028D7D1002FD5D050
:10E1800009EB070010F8013C08AA52F82300002808
:10E190004AD1DA4509EB08002AD210F80A30317862
:10E1A000994218BF534642D16FEA0A0303EB0B01B1
:10E1B000C9073246534618D50AF101035B4517D209
:10E1C000324612F8011F10F803E08E450DD02EE004
:10E1D00012F8011F10F803C08C4528D1013312F842
:10E1E000011F10F803E08E4521D101335B45EFD3C9
:10E1F000621C23469BD0295D025D914213D1E10749
:10E2000009D5631EE95CC25C914204D00BE0E95C75
:10E21000C25C914207D15A1E002B88D0A95C825C57
:10E22000023B9142F3D0079880443A469BE7DDF8E1
:10E2300004C0E0449844F8E7049B6AE706EB0B004F
:10E2400075E700BF2DE9F04F037889B080460D4691
:10E25000002B00F065810A789AB1844601310126CD
:10E2600002E011F8012B5AB1934214BF002606F0C8
:10E2700001061CF8013F0C46002BF2D1207820B992
:10E2800036B1404609B0BDE8F08F4FF00008F8E71E
:10E2900008F101002978FFF7F7FB641B0646002808
:10E2A000F3D0012C00F0B580A044404594BFC0EBF2
:10E2B000080701271F2C06D939462A462346FFF7AF
:10E2C00041FE8046DDE7214607AA2846FFF7DCFD30
:10E2D0000799039069182846039A00F0B9FA0028B4
:10E2E00040F09980DDF80CC0DDF80C900CF1FF3E99
:10E2F00005EB0E01C9F1010C8346CDF808E080461C
:10E300000491CDF814C03A46B146019508EB0406D5
:10E3100009EB02000021B21A00F0FAF90028B4D18A
:10E32000002EB2D0039B9B4528BF5B469C4227D959
:10E33000019D09EB030010F80820E95CE818914200
:10E340005FD1DD432D1915F0010F024609EB0801DD
:10E3500013D001339C4213D94078CD5C0132854201
:10E360000BD04EE012F8010FCD5C854249D101334C
:10E3700012F8010FCD5C854243D101339C42F1D8A4
:10E38000DDF80CE0029ADE4540F2CD80019B09EBFE
:10E390000805995CA85C814240F0C580DDF804A0C6
:10E3A000049BDA44CAEB0301C8071AD5029FDDF8C3
:10E3B00010C0791E685C1CF8017C0CF1FF338742A9
:10E3C00014D10A460DE013F801EC2F5C4B1EBE453C
:10E3D0000CD1024601382F5C11F8011CB94205D15D
:10E3E0000246501E534503F1FF31ECD10BF1010BF6
:10E3F000934500F29A80079A9044C2EB040B324690
:10E4000084E7059D05EB080B0BEB03084FF0000BB1
:10E41000F5E7804635E7DDF80CA00399CAEB040365
:10E42000534538BF5346CAF1010B581C06EB0A028C
:10E4300005EB0A08CDF808B03B4607904FF00009FD
:10E44000019201F1FF3B37468A4609EB0406F818B2
:10E450000021F21A00F05CF900287FF416AF002EBC
:10E460003FF413AF544598BF07EB09002CD9DDF8F2
:10E4700004E098F800001EF8093098424AD16FEA8B
:10E480000A021119C9074246534607EB090018D57D
:10E490000AF101039C4217D9424612F8011F10F8F5
:10E4A00003C08C450DD036E012F8011F10F803E0D0
:10E4B0008E4530D1013312F8011F10F803C08C458E
:10E4C00029D101339C42EFD8BBF1FF3F5B463FF4BB
:10E4D000F8AE15F80B1010F80B20914216D11BF076
:10E4E000010F0AD00BF1FF33E95CC25C914204D00A
:10E4F0000CE0E95CC25C914208D15A1E002B3FF44B
:10E50000E0AEA95C825C023B9142F2D00798814464
:10E5100033469AE75346DDF808E0F1449944F7E7BB
:10E520000C460126AAE6039A60E74E46C844A8E6D0
:10E5300040F29853C2F200031A6801235C3200F0E3
:10E5400001B800BFF0B4002825D0074638463E7811
:10E550000D46013715F8014B3CB1A642FAD1002B0C
:10E56000F4D1176007F8013C11E0C6B13D4600E068
:10E570001BB915F8016B0C46284614F8013B9E4266
:10E58000F6D136B1002105F8011C1060781EF0BCF0
:10E5900070473046F9E710680028D6D1F7E71660D3
:10E5A0003046F4E72DE9F00F494C82B0D4F800C0B2
:10E5B00001900F463C4614F8015B0CEB05004678D1
:10E5C000274606F00800C6B2002EF3D12D2D61D0EB
:10E5D0002B2D04BF244614F8015BB346002B41D118
:10E5E000302D43D00A239A46BBF1000F0CBF6FF0C9
:10E5F00000474FF00047B7FBFAF90AFB197000908B
:10E60000002080460CE0303DAB421BDD461C05D0AF
:10E61000C84539D835D00AFB0858012014F8015BE9
:10E620000CEB0506767806F00407FFB2002FEAD15E
:10E6300016F0030606D0012E14BF57263726AD1B51
:10E64000AB42E3DC431C2AD0BBF1000F01D0C8F180
:10E650000008002A31D0D0B94046116002B0BDE8B0
:10E66000F00F7047102BBED1302DBCD12578782DFE
:10E6700025D0582D23D043BB4FF0080A30255346F0
:10E68000B2E700988542C6DD4FF0FF30C6E740464E
:10E69000611EE2E714F8015B4FF0010B9EE7BBF14E
:10E6A000000F01990CBF6FF000404FF00040222393
:10E6B0000B60002AD2D0611ECFE74046CEE74FF074
:10E6C000100A6578534602348EE79A4630258BE768
:10E6D0006C01002070B440F29854C2F20004064667
:10E6E0000D462068134631462A4670BCFFF75ABFD4
:10E6F000024B13B1024800F005B87047000000005B
:10E70000D1D600080146002002460346FEF760BF4E
:10E710008307F0B4C9B200F09680531E002A00F0BF
:10E72000948002788A420BD0421CD8071AD512F086
:10E73000030F10461CD01478013B01328C4211D1DA
:10E74000F0BC7047002B7CD01278013B8A42F7D096
:10E7500014F0030F204604F1010209D02478013B94
:10E760008C42EDD012F0030F104602F10104E9D102
:10E77000032B3FD9046841EA012545EA054585EAAE
:10E780000407A7F1013222EA07021E1F041D12F03E
:10E79000803FC6F380072DD1032E334629D967B1B8
:10E7A0002668204685EA0602A2F1013626EA020220
:10E7B000043412F0803F19D01CE020462468061D66
:10E7C00085EA0402A2F1013424EA020212F0803F39
:10E7D00010D13468043B85EA0402A2F1013424EA32
:10E7E0000202341D12F0803F304603D1043B032B5C
:10E7F000E3D820465D1E23B303788B42A0D0431C90
:10E800000022E80714D51C781846012201338C42F7
:10E8100096D09542184603F1010402F102020ED08F
:10E820001B788B428CD020462478431C8C4287D0A6
:10E830009542184603F1010402F10202F0D10020D2
:10E840007EE718467CE7134692E7104678E700BF5C
:10E85000032AF0B431D941EA00039C072ED106689F
:10E860000F68151F031D0C1DBE42C5F3800C24D17B
:10E87000032D2A461FD9BCF1000F08D01E68256859
:10E880002146184604340433AE4211D015E0214627
:10E8900018461C680B68051D0E1D9C420DD13146A3
:10E8A00028462E680D68043A031D0C1DAE4204D1A3
:10E8B000043A032AEBD8214618461AB303780C7899
:10E8C000A3420AD1551E0022EB0714D510F8013FD0
:10E8D00011F8014F0122A3420DD0181B10E010F8CF
:10E8E000013F11F8014FA342F7D110F8013F11F891
:10E8F000014FA342F1D1AA4202F10202EFD100205E
:10E90000F0BC70471046FBE71E1E646464646464D8
:10E910001048498A8B8C8D84858687FF1048494A28
:10E920004B4C4D44454647FF2021222324252627D2
:10E9300048498A8B8C8DFF0048E900081CE90008D3
:10E9400028E9000810E90008202122232425262791
:10E9500048494A4B4C4DFF00CF1D00087D1D000863
:10E96000A11D0008691D00086F1D00086B1D00082F
:10E97000000000400008014001000000001C0000F1
:10E98000000000400008014002000000041C0000DC
:10E99000000000400008014004000000081C0000C6
:10E9A0000000004000080140080000000C1C0000AE
:10E9B000000400400008014040000000001D00006D
:10E9C000000400400008014080000000041D000019
:10E9D00000040040000C014001000000081D000080
:10E9E00000040040000C0140020000000C1D00006B
:10E9F000002C01400008014000010000001B010044
:10EA0000002C014000080140000800000C1B010020
:10EA100000080040000C014040000000001E000003
:10EA200000080040000C014080000000041E0000AF
:10EA300000080040000C014000010000081E00001A
:10EA400000080040000C0140000200000C1E000005
:10EA5000002C01400000004000040040000800407D
:10EA60000004080CD00732003200320032003200BD
:10EA700032003200C8006400000041455452313277
:10EA800033340000A3500008CB4F00087350000837
:10EA900029500008E14F0008C94F00080000803FDE
:10EAA00000000000A8AAAA3F0000803F0000803FAD
:10EAB000000080BFB0AA2ABF000080BF0000803FD6
:10EAC0000000803FB0AA2ABF000080BF0000803F46
:10EAD00000000000A8AAAA3F000080BF0000803FFD
:10EAE000000080BFB0AA2ABF0000803F0000803F26
:10EAF0000000803FB0AA2ABF0000803F0000803F96
:10EB000000000000A8AAAA3F000000000000803F0B
:10EB1000000080BFB0AA2ABF000000000000803FB4
:10EB20000000803FB0AA2ABF000000000000803F24
:10EB3000000080BF0000803F000080BF0000803FD9
:10EB4000000080BF000080BF0000803F0000803FC9
:10EB50000000803F0000803F0000803F0000803FB9
:10EB60000000803F000080BF000080BF0000803FA9
:10EB70000000000000000000000000000000803FD6
:10EB80000000000000000000000000000000803FC6
:10EB9000000000000000803F0000803F0000803F38
:10EBA000000080BF000080BF000000000000803F28
:10EBB000000000000000803F000080BF0000803F98
:10EBC0000000803F000080BF000000800000803F08
:10EBD000000000000000803F000080BF0000803F78
:10EBE000000080BF000000000000803F0000803F68
:10EBF0000000803F000000000000803F0000803FD8
:10EC000000000000000080BF000080BF0000000086
:10EC10000000000003010000FCEA000804000000FE
:10EC2000CCEB00080400000004EE00080201000024
:10EC3000A4ED000800010000000000000600000034
:10EC40009CEA00080600000044ED000801010000F5
:10EC50000000000004000000C4ED000806000000F1
:10EC6000C4EE00080800000024EF000808000000BF
:10EC7000C4EC00080800000044EE00080101000098
:10EC80000000000000010000000000000001000082
:10EC900000000000040000008CEB000806000000EB
:10ECA0002CEB000800010000000000000201000041
:10ECB000A4EF0008010100000000000000000000B7
:10ECC000000000000000803FF704353FF70435BF27
:10ECD0000000803F0000803FF70435BFF70435BFD8
:10ECE0000000803F0000803FF70435BFF704353F48
:10ECF0000000803F0000803FF704353FF704353FB8
:10ED00000000803F0000803F00000000000080BF46
:10ED1000000080BF0000803F000080BF00000000B6
:10ED2000000080BF0000803F000000000000803F26
:10ED3000000080BF0000803F0000803F0000000016
:10ED4000000080BF0000803FD0B35DBF0000003FE7
:10ED50000000803F0000803FD0B35DBF000000BFD7
:10ED6000000080BF0000803FD0B35D3F0000003F47
:10ED70000000803F0000803FD0B35D3F000000BF37
:10ED8000000080BF0000803F00000000000080BF46
:10ED90000000803F0000803F000000000000803F36
:10EDA000000080BF0000803F0000803F00000000A6
:10EDB000000000000000803F000080BF0000000055
:10EDC000000000000000803F000000000000803FC5
:10EDD000000080BF0000803F000080BF000080BFB7
:10EDE000000000000000803F000000000000803FA5
:10EDF0000000803F0000803F0000803F000080BF97
:10EE0000000000000000803F000080BF0000803F45
:10EE1000000080BF0000803F000080BF000080BF76
:10EE20000000803F0000803F0000803F0000803FE6
:10EE30000000803F0000803F0000803F000080BF56
:10EE4000000080BF0000803F0000803F000000BF46
:10EE50000000803F0000803F000000BF000080BF36
:10EE60000000803F0000803F000080BF0000003FA6
:10EE70000000803F0000803F0000003F0000803F16
:10EE80000000803F0000803F0000003F000080BF86
:10EE9000000080BF0000803F000080BF000000BF76
:10EEA000000080BF0000803F000000BF0000803FE6
:10EEB000000080BF0000803F0000803F0000003F56
:10EEC000000080BF0000803F000000BFD0B35D3F66
:10EED0000000803F0000803F000000BFD0B35DBF56
:10EEE0000000803F0000803F0000003FD0B35D3F46
:10EEF000000080BF0000803F0000003FD0B35DBF36
:10EF0000000080BF0000803F000080BF00000000C4
:10EF1000000080BF0000803F0000803F0000000034
:10EF20000000803F0000803F000080BF0000803F65
:10EF3000000080BF0000803F000080BF000080BF55
:10EF40000000803F0000803F0000803F0000803FC5
:10EF50000000803F0000803F0000803F000080BF35
:10EF6000000080BF0000803F000080BF0000803FA5
:10EF70000000803F0000803F000080BF000080BF95
:10EF8000000080BF0000803F0000803F0000803F05
:10EF9000000080BF0000803F0000803F000080BF75
:10EFA0000000803F0000803F0000000000000000E3
:10EFB000000080BF0000803F000000000000000053
:10EFC0000000803F24505542582C34312C312C30D5
:10EFD0003030332C303030312C3131353230302C30
:10EFE000302A31450D0A0024504D544B3235312C16
:10EFF0003131353230302A31460D0A002450554225
:10F00000582C34312C312C303030332C30303031DE
:10F010002C35373630302C302A32440D0A0024503B
:10F020004D544B3235312C35373630302A32430D82
:10F030000A0024505542582C34312C312C303030B9
:10F04000332C303030312C33383430302C302A32BD
:10F05000360D0A0024504D544B3235312C333834A0
:10F0600030302A32370D0A0024505542582C3431A2
:10F070002C312C303030332C303030312C3139328F
:10F0800030302C302A32330D0A0024504D544B328C
:10F0900035312C31393230302A32320D0A00B56226
:10F0A00006010300F00500FF19B56206010300F038
:10F0B0000300FD15B56206010300F00100FB11B568
:10F0C0006206010300F00000FA0FB56206010300BA
:10F0D000F00200FC13B56206010300F00400FE1705
:10F0E000B562060103000102010E47B56206010385
:10F0F000000103010F49B562060103000106011278
:10F100004FB562060103000112011E67B5620616C3
:10F11000080003070300510800008A41B562060891
:10F120000600C80001000100DE6A000000000000C7
:10F1300000C20100C4EF0008E7EF00080100000072
:10F1400000E10000FCEF00081EF0000802000000D3
:10F150000096000032F0000854F0000803000000A0
:10F16000004B000068F000088AF00008040000006E
:10F1700080250000A0F80008A0F80008414552547E
:10F180003132333400000000C3000108C700010819
:10F19000CC000108DD000108E6000108F1000108CB
:10F1A000FC00010807010108E5FF00081001010843
:10F1B000DFFF000819010108230101082E010108E1
:10F1C00034010108000000001500010819000108C1
:10F1D0001F00010825000108280001082F00010870
:10F1E0003200010837000108430001084600010809
:10F1F0004C000108530001085D0001086700010888
:10F20000700001087E0001088A00010891000108D1
:10F2100097000108A4000108AF000108BC00010824
:10F220000000000027FE00082BFE0008A18F000848
:10F2300052FE000857FE00089D9400086BFE00086F
:10F2400074FE0008E18D000891FE000896FE00089B
:10F25000E9920008C5FE0008A0F80008A98D000882
:10F26000CAFE0008D2FE0008BD8C0008E6FE0008B9
:10F27000F5FE00089D8C00080FFF0008A0F80008AC
:10F28000A58A000814FF000818FF0008F58B000885
:10F2900065FE000834FF00080D8E000847FF0008D7
:10F2A0004DFF0008F98E000868FF000870FF000895
:10F2B000AD8E00087FFF000884FF0008C58B0008A2
:10F2C000B1F7000894FF000895910008C2FF0008FC
:10F2D000B6FF0008D18A0008C9FF0008A0F800089E
:10F2E000998A0008A0F80008F1FF0008F9FF00085B
:10F2F00001000108090001081000010800000000D9
:10F30000303132333435363738394142434445465B
:10F310004748494A4B4C4D4E4F5051525354555605
:10F320005758595A004166726F333220434C492076
:10F3300076657273696F6E20322E322041707220B2
:10F3400031392032303134202F2030313A31323AC5
:10F35000353200417661696C61626C6520636F6D66
:10F360006D616E64733A0D0A0025730925730D0AE9
:10F370000053797374656D20557074696D653A201A
:10F380002564207365636F6E64732C20566F6C74F4
:10F390006167653A202564202A20302E31562028C6
:10F3A0002564532062617474657279290D0A0043E3
:10F3B00050552025644D487A2C206465746563742B
:10F3C00065642073656E736F72733A200025732035
:10F3D0000041434348573A202573002E25630043DC
:10F3E00079636C652054696D653A2025642C204949
:10F3F0003243204572726F72733A2025642C206369
:10F400006F6E6669672073697A653A2025640D0A14
:10F4100000536176696E672E2E2E000D0A526562CA
:10F420006F6F74696E672E2E2E004D757374206297
:10F430006520616E79206F72646572206F6620416D
:10F44000455452313233340D0A0043757272656E81
:10F45000742061737369676E6D656E743A20004540
:10F4600072726F723A20456E61626C6520616E64E3
:10F4700020706C756720696E204750532066697252
:10F4800073740D0A00456E61626C696E67204750A7
:10F490005320706173737468726F7567682E2E2EB7
:10F4A0000D0A00456E61626C656420666561747565
:10F4B0007265733A2000417661696C61626C652007
:10F4C00066656174757265733A2000496E76616C89
:10F4D00069642066656174757265206E616D652E64
:10F4E0002E2E0D0A0044697361626C65642000452C
:10F4F0006E61626C656420000D0A4C656176696E10
:10F500006720434C49206D6F64652E2E2E0D0A0036
:10F51000526573657474696E6720746F20646566E4
:10F5200061756C74732E2E2E0D0A00437572726510
:10F530006E74206D697865723A2025730D0A00415A
:10F540007661696C61626C65206D69786572733A89
:10F550002000496E76616C6964206D69786572205F
:10F56000747970652E2E2E0D0A004D697865722013
:10F5700073657420746F2025730D0A0043757272D1
:10F58000656E742070726F66696C653A2025640D33
:10F590000A0055736167653A0D0A6D6F746F7220CA
:10F5A000696E646578205B76616C75655D202D20E1
:10F5B00073686F77205B6F72207365745D206D6F69
:10F5C000746F722076616C75650D0A004E6F207342
:10F5D000756368206D6F746F722C20757365206180
:10F5E000206E756D626572205B302C2025645D0D88
:10F5F0000A004D6F746F7220256420697320736553
:10F60000742061742025640D0A00496E76616C696E
:10F6100064206D6F746F722076616C75652C20317B
:10F620003030302E2E323030300D0A005365747475
:10F63000696E67206D6F746F7220256420746F206F
:10F6400025640D0A006175782025752025750D0A41
:10F6500000496E76616C69642046656174757265F7
:10F6600020696E6465783A206D7573742062652038
:10F670003C2025750D0A0020256420256400437573
:10F680007272656E742073657474696E67733A2064
:10F690000D0A0025732073657420746F2000455295
:10F6A000523A2056616C75652061737369676E6D9F
:10F6B000656E74206F7574206F662072616E676569
:10F6C0000D0A004552523A20556E6B6E6F776E20D0
:10F6D0007661726961626C65206E616D650D0A000C
:10F6E00043757272656E7420436F6E6669673A2067
:10F6F000436F70792065766572797468696E6720EA
:10F7000062656C6F7720686572652E2E2E0D0A007B
:10F710006D697865722025730D0A00636D69782024
:10F72000256400636D697820256420302030203006
:10F7300020300D0A0066656174757265202D257391
:10F740000D0A00666561747572652025730D0A00E7
:10F750006D61702025730D0A007365742025732078
:10F760003D20004E4709004F4B0900437573746FED
:10F770006D206D697865723A200D0A4D6F746F7255
:10F780000954687209526F6C6C0950697463680996
:10F790005961770D0A002325643A09002573090091
:10F7A00053616E69747920636865636B3A0900720E
:10F7B00065736574006C6F6164004C6F61646564AF
:10F7C000202573206D69782E2E2E0D0A0057726F3A
:10F7D0006E67206E756D626572206F66206172675C
:10F7E000756D656E74732C206E6565647320696435
:10F7F000782074687220726F6C6C20706974636812
:10F80000207961770D0A004D6F746F72206E756DEF
:10F81000626572206D75737420626520626574770D
:10F8200065656E203120616E642025640D0A000D2F
:10F830000A456E746572696E6720434C49204D6FAE
:10F8400064652C2074797065202765786974272099
:10F85000746F2072657475726E2C206F7220276829
:10F86000656C70270D0A000D0A2320000D1B5B4BF1
:10F87000001B5B324A1B5B313B3148004552523A18
:10F8800020556E6B6E6F776E20636F6D6D616E6469
:10F890002C20747279202768656C70270008200876
:10F8A000006C6F6F7074696D65006D6964726300E0
:10F8B0006D696E7468726F74746C65006D617874D4
:10F8C00068726F74746C65006D696E636F6D6D61E5
:10F8D0006E64006D696E636865636B006D6178636B
:10F8E0006865636B006465616462616E6433645F64
:10F8F0006C6F77006465616462616E6433645F6835
:10F90000696768006E65757472616C336400646564
:10F91000616462616E6433645F7468726F74746C86
:10F9200065006D6F746F725F70776D5F7261746583
:10F9300000736572766F5F70776D5F7261746500DA
:10F9400072657461726465645F61726D00666C619A
:10F9500070735F7370656564006669786564776964
:10F960006E675F616C74686F6C645F64697200726B
:10F9700065626F6F745F6368617261637465720062
:10F98000736F667473657269616C5F6261756472CE
:10F9900061746500736F667473657269616C5F3161
:10F9A0005F696E76657274656400736F6674736503
:10F9B0007269616C5F325F696E766572746564004E
:10F9C0006770735F74797065006770735F626175EB
:10F9D00064726174650073657269616C72785F74DA
:10F9E0007970650074656C656D657472795F7072AD
:10F9F0006F76696465720074656C656D65747279A3
:10FA00005F706F72740074656C656D657472795F98
:10FA100073776974636800766261747363616C659F
:10FA200000766261746D617863656C6C766F6C747E
:10FA300061676500766261746D696E63656C6C7692
:10FA40006F6C7461676500706F7765725F61646386
:10FA50005F6368616E6E656C00616C69676E5F679D
:10FA600079726F00616C69676E5F61636300616CDE
:10FA700069676E5F6D616700616C69676E5F626F79
:10FA80006172645F726F6C6C00616C69676E5F625B
:10FA90006F6172645F706974636800616C69676E3E
:10FAA0005F626F6172645F796177007961775F632C
:10FAB0006F6E74726F6C5F646972656374696F6E88
:10FAC000006163635F6861726477617265006D6194
:10FAD000785F616E676C655F696E636C696E617497
:10FAE000696F6E006D6F726F6E5F746872657368B8
:10FAF0006F6C64006779726F5F6C70660067797213
:10FB00006F5F636D70665F666163746F72006779C3
:10FB1000726F5F636D70666D5F666163746F7200B4
:10FB20007069645F636F6E74726F6C6C657200797C
:10FB300061776465616462616E6400616C745F68C2
:10FB40006F6C645F7468726F74746C655F6E6575FA
:10FB50007472616C00616C745F686F6C645F666185
:10FB600073745F6368616E6765007468726F747444
:10FB70006C655F636F7272656374696F6E5F7661E7
:10FB80006C7565007468726F74746C655F636F7216
:10FB900072656374696F6E5F616E676C6500726336
:10FBA0005F726174650072635F6578706F0074687E
:10FBB000725F6D6964007468725F6578706F00725F
:10FBC0006F6C6C5F70697463685F726174650079F3
:10FBD000617772617465007470617261746500743C
:10FBE00070615F627265616B706F696E74006661EF
:10FBF000696C736166655F64656C617900666169F3
:10FC00006C736166655F6F66665F64656C617900E1
:10FC10006661696C736166655F7468726F74746C39
:10FC200065006661696C736166655F6465746563D0
:10FC3000745F7468726573686F6C64007273736963
:10FC40005F6175785F6368616E6E656C007961777E
:10FC50005F646972656374696F6E007472695F7561
:10FC60006E61726D65645F736572766F0067696D52
:10FC700062616C5F666C616773006163635F6C7087
:10FC8000665F666163746F720061636378795F6455
:10FC900065616462616E64006163637A5F6465617B
:10FCA0006462616E64006163635F756E61726D654D
:10FCB0006463616C006163635F7472696D5F706936
:10FCC000746368006163635F7472696D5F726F6C07
:10FCD0006C006261726F5F7461625F73697A650064
:10FCE0006261726F5F6E6F6973655F6C70660062F0
:10FCF00061726F5F63665F76656C006261726F5FF1
:10FD000063665F616C74006D61675F6465636C69F5
:10FD10006E6174696F6E006770735F706F735F7090
:10FD2000006770735F706F735F69006770735F70F7
:10FD30006F735F64006770735F706F73725F7000E2
:10FD40006770735F706F73725F69006770735F7065
:10FD50006F73725F64006770735F6E61765F7000CF
:10FD60006770735F6E61765F69006770735F6E6165
:10FD7000765F64006770735F77705F726164697546
:10FD800073006E61765F636F6E74726F6C735F6821
:10FD9000656164696E67006E61765F737065656446
:10FDA0005F6D696E006E61765F73706565645F6D2F
:10FDB0006178006E61765F736C65775F7261746500
:10FDC00000705F706974636800695F70697463686C
:10FDD00000705F726F6C6C00695F726F6C6C0070AA
:10FDE0005F79617700695F79617700705F616C743A
:10FDF00000695F616C7400645F616C7400705F6CBB
:10FE00006576656C00695F6C6576656C00645F6C37
:10FE10006576656C00705F76656C00695F76656C11
:10FE200000645F76656C0061757800666561747565
:10FE300072655F6E616D6520617578666C616720C3
:10FE40006F7220626C616E6B20666F72206C6973DA
:10FE50007400636D69780064657369676E2063750B
:10FE600073746F6D206D6978657200646566617585
:10FE70006C747300726573657420746F20646566BA
:10FE800061756C747320616E64207265626F6F744B
:10FE90000064756D70007072696E7420636F6E66B9
:10FEA0006967757261626C652073657474696E67E9
:10FEB0007320696E2061207061737461626C6520CB
:10FEC000666F726D0065786974006665617475723D
:10FED00065006C697374206F72202D76616C206FE1
:10FEE000722076616C0067707370617373746872EE
:10FEF0006F75676800706173737468726F75676897
:10FF00002067707320746F2073657269616C00687C
:10FF1000656C70006D6170006D617070696E672056
:10FF20006F66207263206368616E6E656C206F720D
:10FF3000646572006D69786572206E616D65206F11
:10FF400072206C697374006D6F746F7200676574F2
:10FF50002F736574206D6F746F72206F7574707578
:10FF6000742076616C75650070726F66696C6500EF
:10FF7000696E64657820283020746F203229007300
:10FF8000617665007361766520616E6420726562DA
:10FF90006F6F74006E616D653D76616C7565206F85
:10FFA0007220626C616E6B206F72202A20666F7205
:10FFB000206C6973740073686F772073797374654C
:10FFC0006D207374617475730076657273696F6EFA
:10FFD000004759524F00414343004241524F0053A2
:10FFE0004F4E415200475053004750532B4D41470D
:10FFF000004144584C333435004D5055363035307F
:020000040801F1
:10000000004D4D413834357800424D413238300092
:100010004E6F6E6500545249005155414450005195
:10002000554144580042490047494D42414C00590E
:1000300036004845583600464C59494E475F5749A7
:100040004E47005934004845583658004F43544FE6
:100050005838004F43544F464C415450004F43547E
:100060004F464C41545800414952504C414E450076
:1000700048454C495F3132305F4343504D0048455D
:100080004C495F39305F44454700565441494C3430
:100090000048455836480050504D5F544F5F534517
:1000A00052564F004455414C434F50544552005313
:1000B000494E474C45434F505445520043555354C5
:1000C0004F4D0050504D005642415400494E464C51
:1000D000494748545F4143435F43414C00534552B5
:1000E00049414C5258004D4F544F525F53544F505A
:1000F00000534552564F5F54494C5400534F465499
:1001000053455249414C004C45445F52494E4700CB
:100110004641494C534146450054454C454D455494
:10012000525900504F5745524D4554455200564183
:1001300052494F0033440000D1FF0008D6FF0008A9
:10014000DAFF0008EDFF0008DFFF0008E5FF000808
:10015000E9FF000800000000A1F80008020000000C
:10016000E01700200000000028230000AAF8000883
:1001700002000000E6180020B0040000A406000001
:10018000B0F8000802000000A418002000000000E1
:10019000D0070000BCF8000802000000A6180020EC
:1001A00000000000D0070000C8F8000802000000AE
:1001B000A818002000000000D0070000D3F80008B5
:1001C00002000000E818002000000000D007000036
:1001D000DCF8000802000000EA180020000000001F
:1001E000D0070000E5F8000802000000AA1800206F
:1001F00000000000D0070000F4F800080200000032
:10020000AC18002000000000D007000004F900082E
:1002100002000000AE18002000000000D00700001F
:100220000EF9000802000000B018002000000000D5
:10023000D007000022F9000802000000B2180020D8
:1002400032000000007D000031F9000802000000CB
:10025000B418002032000000F201000040F900084C
:1002600000000000EC180020000000000100000069
:100270004DF9000800000000ED180020000000000B
:100280006400000059F9000801000000EE18002089
:10029000FFFFFFFF010000006FF9000800000000F1
:1002A000FE180020300000007E00000084F90008E5
:1002B00004000000F4180020B004000000C2010097
:1002C00080F9000804000000F8180020B0040000C5
:1002D000004B000094F9000800000000FC1800200A
:1002E0000000000001000000AAF900080000000062
:1002F000FD1800200000000001000000C0F9000807
:1003000000000000F01800200000000004000000C1
:10031000C9F9000801000000F118002000000000E9
:1003200004000000D6F9000800000000E4180020D6
:100330000000000003000000E4F9000800000000D5
:10034000001900200000000001000000F7F900087B
:100350000000000001190020000000000200000061
:1003600006FA00080000000002190020000000004A
:100370000100000017FA000800000000D818002053
:100380000A000000C800000021FA00080000000078
:10039000D91800200A0000003200000034FA0008DA
:1003A00000000000DA1800200A00000032000000FF
:1003B00047FA000800000000DB18002000000000E1
:1003C0000900000059FA000800000000B6180020DB
:1003D000000000000800000064FA000800000000AF
:1003E000B718002000000000080000006EFA0008A6
:1003F00000000000B8180020000000000800000005
:1004000078FA000803000000BA1800204CFFFFFF34
:100410006801000089FA000803000000BC180020F1
:100420004CFFFFFF680100009BFA0008030000007A
:10043000BE1800204CFFFFFF68010000ABFA000867
:1004400001000000C0180020FFFFFFFF01000000B6
:10045000C1FA000800000000C118002000000000E0
:1004600005000000CEFA000802000000CA180020B3
:100470006400000084030000E4FA000800000000AB
:10048000C81800200000000080000000F4FA0008F6
:1004900002000000C218002000000000000100005F
:1004A000FDFA000802000000C418002064000000EB
:1004B000E80300000EFB000802000000C618002040
:1004C00064000000E803000020FB000800000000BA
:1004D0000817002000000000010000008FFC000849
:1004E0000000000074170020000000002000000041
:1004F0002FFB00080000000075170020000000001E
:10050000640000003BFB000800000000761700209C
:1005100001000000FA00000055FB00080000000088
:100520007717002000000000010000006AFB0008AF
:10053000000000007A170020000000009600000074
:1005400084FB000802000000781700200100000072
:10055000840300009EFB0008000000002717002015
:1005600000000000FA000000A6FB000800000000E8
:10057000281700200000000064000000AEFB000807
:1005800000000000291700200000000064000000A7
:10059000B6FB0008000000002A1700200000000041
:1005A00064000000BFFB0008000000002B170020C3
:1005B0000000000064000000CFFB00080000000005
:1005C0002C1700200000000064000000D7FB00088A
:1005D000000000002D170020000000006400000053
:1005E000DFFB0008020000002E170020E8030000D7
:1005F000D0070000EEFB000800000000BC17002040
:1006000000000000C8000000FDFB00080000000022
:10061000BD17002000000000C800000010FC00080A
:1006200002000000BE170020E8030000D007000011
:1006300022FC000802000000C01700206400000037
:10064000D00700003CFC000801000000EF1800206B
:1006500000000000040000004DFC00080100000044
:10066000C2170020FFFFFFFF010000005BFC000835
:1006700001000000C317002000000000010000007E
:100680006DFC000800000000C417002000000000FE
:10069000FF0000007AFC0008000000003617002070
:1006A00000000000FA00000089FC000800000000C3
:1006B00038170020000000006400000098FC0008CB
:1006C0000000000037170020000000006400000058
:1006D000A6FC0008000000004817002000000000F1
:1006E00001000000B5FC00080300000034170020E2
:1006F000D4FEFFFF2C010000C4FC00080300000032
:1007000032170020D4FEFFFF2C010000D2FC0008AD
:100710000000000039170020000000003000000039
:10072000E0FC0008050000003C170020000000006D
:1007300001000000EFFC0008050000004017002049
:100740000000000001000000FBFC000805000000A4
:1007500044170020000000000100000007FD000811
:100760000300000030170020B0B9FFFF5046000022
:1007700017FD0008000000000D1700200000000019
:10078000C800000021FD000800000000171700202D
:1007900000000000C80000002BFD00080000000061
:1007A0002117002000000000C800000035FD0008EF
:1007B000000000000E17002000000000C80000002C
:1007C00040FD000800000000181700200000000095
:1007D000C80000004BFD00080000000022170020A8
:1007E00000000000C800000056FD000800000000E6
:1007F0000F17002000000000C800000060FD000886
:10080000000000001917002000000000C8000000D0
:100810006AFD00080000000023170020000000000F
:10082000C800000074FD000802000000C617002088
:1008300000000000D007000082FD0008000000005A
:10084000CA170020000000000100000097FD00080A
:1008500002000000CC1700200A000000D0070000B2
:10086000A5FD000802000000CE1700200A000000CD
:10087000D0070000B3FD000800000000C9170020E9
:100880000000000064000000C1FD0008000000003E
:100890000A17002000000000C8000000C9FD000881
:1008A000000000001417002000000000C800000035
:1008B00093FA0008000000001E170020000000004E
:1008C000C8000000D1FD000800000000091700204A
:1008D00000000000C8000000D8FD00080000000073
:1008E0001317002000000000C800000082FA000872
:1008F000000000001D17002000000000C8000000DC
:10090000DFFD0008000000000B17002000000000C1
:10091000C8000000E5FD00080000000015170020D9
:1009200000000000C8000000A5FA00080000000058
:100930001F17002000000000C8000000EBFD0008A9
:10094000000000000C17002000000000C80000009C
:10095000F1FD000800000000161700200000000054
:10096000C8000000F7FD000800000000201700206C
:1009700000000000C8000000FDFD000800000000AD
:100980001017002000000000C800000005FE00084D
:10099000000000001A17002000000000C80000003E
:1009A0000DFE0008000000002417002000000000D9
:1009B000C800000015FE000800000000121700200B
:1009C00000000000C80000001BFE0008000000003E
:1009D0001C17002000000000C800000021FE0008D5
:1009E000000000002617002000000000C8000000E2
:1009F000524F4C4C3B50495443483B5941573B4163
:100A00004C543B506F733B506F73523B4E61765268
:100A10003B4C4556454C3B4D41473B56454C3B00B6
:100A200041524D3B00414E474C453B00484F5249D7
:100A30005A4F4E3B004241524F3B00564152494FA4
:100A40003B004D41473B0048454144465245453BEC
:100A5000004845414441444A3B0043414D535441C1
:100A6000423B0043414D545249473B0047505320BD
:100A7000484F4D453B0047505320484F4C443B00A6
:100A800050415353544852553B00424545504552FE
:100A90003B004C45444D41583B004C45444C4F575E
:100AA0003B004C4C49474854533B0043414C49425E
:100AB0003B00474F5645524E4F523B004F53442048
:100AC00053573B0054454C454D455452593B00004B
:100AD0000000004B000000CB61636F7366000000F4
:100AE000000000007371727466000000000FC93FBF
:100AF000000F494000CB9640000FC9400053FB4017
:100B000000CB164100ED2F41000F494100316241F9
:100B100000537B41003A8A4100CB9641005CA341DF
:100B200000EDAF41007EBC41000FC94100A0D5419E
:100B30000031E24100C2EE410053FB4100F20342AA
:100B4000003A0A420083104200CB164200141D42B4
:100B5000005C234200A5294200ED2F4200363642B8
:100B6000007E3C4200C74242000F4942A200000002
:100B7000F9000000830000006E0000004E0000003D
:100B8000440000001500000029000000FC000000E7
:100B90002700000057000000D1000000F500000011
:100BA00034000000DD000000C0000000DB00000099
:100BB0006200000095000000990000003C00000069
:100BC000430000009000000041000000FE00000013
:100BD0005100000063000000AB000000DE000000D8
:100BE000BB000000C500000061000000B70000006D
:100BF000240000006E0000003A00000042000000E7
:100C00004D000000D2000000E000000006000000DF
:100C1000490000002E000000EA000000090000006A
:100C2000D1000000920000001C000000FE00000047
:100C30001D000000EB0000001C000000B1000000DF
:100C400029000000A70000003E000000E8000000AE
:100C50008200000035000000F50000002E000000BA
:100C6000BB0000004400000084000000E900000018
:100C70009C0000007000000026000000B40000008E
:100C80005F0000007E00000041000000390000000D
:100C900091000000D6000000390000008300000031
:100CA0005300000039000000F40000009C00000028
:100CB000840000005F0000008B000000BD00000009
:100CC000F9000000280000003B0000001F000000A9
:100CD000F800000097000000FF000000DE000000A8
:100CE00005000000980000000F000000EF00000069
:100CF0002F000000110000008B0000005A000000CF
:100D00000A0000006D0000001F0000006D000000E0
:100D1000360000007E000000CF0000002700000029
:100D2000CB00000009000000B70000004F000000E9
:100D3000460000003F000000660000009E0000002A
:100D40005F000000EA0000002D00000075000000B8
:100D500027000000BA000000C7000000EB00000000
:100D6000E5000000F10000007B0000003D000000F5
:100D70000700000039000000F70000008A000000B2
:100D80005200000092000000EA0000006B0000002A
:100D9000FB0000005F000000B10000001F00000029
:100DA0008D0000005D0000000800000056000000FB
:100DB000030000003000000046000000FC000000BE
:100DC0007B0000006B000000AB000000F0000000A2
:100DD000CF000000BC000000200000009A000000CE
:100DE000F4000000360000001D000000A900000013
:100DF000E300000091000000610000005E000000C0
:100E0000E60000001B000000080000006500000074
:100E100099000000850000005F0000001400000041
:100E2000A000000068000000400000008D000000ED
:100E3000FF000000D8000000800000004D0000000E
:100E400073000000270000003100000006000000D1
:100E5000060000001500000056000000CA00000057
:100E600073000000A8000000C9000000600000003E
:100E7000E20000007B000000C00000008C000000C9
:100E80006B000000040000000700000009000000E3
:100E90000000C93F0000F0390000DA370000A2333B
:100EA0000000842E0000502B0000C2270000D0223A
:100EB0000000C41F0000C61B000044176937AC3196
:100EC00068212233B40F14336821A2333863ED3E16
:100ED000DA0F493F5E987B3FDA0FC93F00202020A0
:100EE00020202020202028282828282020202020DA
:100EF00020202020202020202020202020881010AA
:100F00001010101010101010101010101004040405
:100F100004040404040404101010101010104141C3
:100F200041414141010101010101010101010101B1
:100F300001010101010101011010101010104242C5
:100F40004242424202020202020202020202020281
:100F50000202020202020202101010102000000021
:100F60000000000000000000000000000000000081
:100F70000000000000000000000000000000000071
:100F80000000000000000000000000000000000061
:100F90000000000000000000000000000000000051
:100FA0000000000000000000000000000000000041
:100FB0000000000000000000000000000000000031
:100FC0000000000000000000000000000000000021
:100FD0000000000000000000000000000000000011
:100FE0004300000070010020F8B500BFF8BC08BC49
:100FF0009E467047F8B500BFF8BC08BC9E467047D7
:08100000F1E6000835010008CB
:0410080011010008CA
:10100C000403010103010100D90303012136000887
:10101C00010000010000803F000000000000000003
:10102C00DC05DC05DC05DC05DC05DC05DC05DC05AC
:10103C000000803F00000000200A010800000000B2
:10104C0001000000250A0108010000000200000058
:10105C002C0A01080200000003000000350A0108F8
:10106C0003000000040000003B0A0108040000001B
:10107C0005000000420A01080500000006000000FF
:10108C00470A01080600000007000000510A010889
:10109C0007000000080000005A0A010808000000C0
:1010AC0009000000630A0108090000000A000000A2
:1010BC006C0A01080A0000000B000000760A010807
:1010CC000B0000000C000000800A01080C0000005E
:1010DC000D0000008A0A01080D0000000E0000003F
:1010EC00920A01080E0000000F0000009A0A010885
:1010FC000F00000010000000A20A01081000000000
:10110C0011000000AB0A01081100000012000000E1
:10111C00B20A01081200000013000000BC0A01080A
:10112C001300000014000000C40A010814000000A1
:10113C001500000000000000FF000000000000008F
:10114C0000000000010203040607080900127A00DF
:10115C0000A24A0402040608000000000102030475
:10116C00010203040607080901000000DC0E010857
:10117C00000000005C040020C40400202C050020AA
:10118C000000000000000000000000000000000053
:10119C000000000000000000000000000000000043
:1011AC0000000000E00F010800000000000000003B
:1011BC000000000000000000000000000000000023
:1011CC000000000000000000000000000000000013
:1011DC000000000000000000000000000000000003
:1011EC0000000000000000000000000000000000F3
:1011FC0000000000000000000000000000000000E3
:10120C0000000000000000000000000000000000D2
:10121C0000000000000000000100000000000000C1
:10122C000E33CDAB34126DE6ECDE05000B00000086
:10123C0000000000000000000000000000000000A2
:10124C000000000000000000000000000000000092
:10125C000000000000000000000000000000000082
:10126C000000000000000000000000000000000072
:0C159C00000000000000000070010020B2
:0400000508000000EF
:00000001FF
